:100000000C94102B0D9411130D94E6120D94BB1249
:100010000D9490120D9465120D943A120D940F12D6
:100020000C94B4D80C94412B0C94412B0C94412B80
:100030000C94412B0C949EEB0C94412B0C94412B73
:100040000C94412B0C9433D10C94412B0C94412BE8
:100050000C94412B0C94412B0C94A4CF0D943C1385
:100060000C94412B0C94FAD70C94412B0C94412BFB
:100070000C94412B0C94412B0C94412B0C94412B50
:100080000C94412B0C94412B0C94412B0C94412B40
:100090000C94412B0C94412B0C94412B0C94412B30
:1000A0000C94412B0C94412B0C94412B0C94412B20
:1000B0000C94412B0C94412B0C94412B0C94412B10
:1000C0000C94412B0C94412B0C94412B0C94412B00
:1000D0000C94412B0C94412B0C94412B0C94412BF0
:1000E0000C94412B2E463146204624462A4668462B
:1000F000354639463F46434647464D4651465546A6
:1001000068465B465F46634631893189388938895C
:1001100038893F893F893F894C8946894689468984
:100120007CA881A886A890A89AA813A9A4A8ACA87E
:10013000B4A8BEA8C8A8D2A8E1A8EBA813A9F5A89E
:10014000FFA809A92ED834D845D850D858D86DD88A
:100150005CD86DD860D864D86DD86AD8084AD73BC7
:100160003BCE016E84BCBFFDC12F3D6C74319ABD86
:1001700056833DDA3D00C77F11BED9E4BB4C3E91AA
:100180006BAAAABE000000803F05A84CCDB2D44E99
:10019000B93836A9020C50B9918688083CA6AAAA9B
:1001A0002ABE000000803F000D94CC140D948613ED
:1001B0000D94790E0D946E100D949508434F4D4D8E
:1001C000554E49434154494F4E0044525952554EA1
:1001D000004552524F525300494E464F0045434846
:1001E0004F0020746F6F206C6F6E6720657874729B
:1001F0007573696F6E2070726576656E7465640ADA
:100200000020636F6C6420657874727573696F6E1B
:100210002070726576656E7465640A0047322F47F8
:10022000332062616420706172616D657465727300
:100230000A00536C6565702E2E2E00205A3A20005D
:1002400020593A200042656420583A20004C756CD1
:100250007A426F74204D696E692032204C434420ED
:1002600072656164792E00526573756D696E6720E1
:100270007072696E7400436C69636B20746F2072D6
:100280006573756D652E2E2E004E6F206D6F766531
:100290002E004D313235005072696E742074696DD4
:1002A000653A2000000125301D0C1E24311C0B185E
:1002B000232F1B0A17FFFF040806FF06222B1A41F3
:1002C00042043803FF3628294527444350726F748F
:1002D00065637465642050696E0A006D0046696C40
:1002E000616D656E7420757365643A2000537461A6
:1002F00074733A20002C204C6F6E67657374206A0B
:100300006F623A2000546F74616C2074696D653AB5
:10031000200053746174733A20002C204661696C8C
:1003200065643A20002C2046696E69736865643AFA
:1003300020005072696E74733A20005374617473B4
:100340003A20004578747275646572202573004CFC
:10035000756C7A426F74204D696E692032204C436F
:10036000442072656164792E00DD01D801D101CA93
:1003700001BC016F66660044454255473A006F6B09
:1003800000436F6F6C696E6720646F6E652E004866
:10039000656174696E6720646F6E652E0020573A40
:1003A000004578747275646572202573004C756C15
:1003B0007A426F74204D696E692032204C4344208C
:1003C00072656164792E0042656420646F6E652EEB
:1003D0000020573A004265642068656174696E6761
:1003E0002E0042656420636F6F6C696E672E004C4F
:1003F000756C7A426F74204D696E692032204C43CF
:1004000044204F66662E007A5F6D61783A20007A4C
:100410005F6D696E3A2000795F6D61783A200079EE
:100420005F6D696E3A2000785F6D61783A200078E0
:100430005F6D696E3A20005265706F7274696E6705
:1004400020656E6473746F70207374617475730AC1
:10045000004D31343520533C696E6465783E206F21
:100460007574206F662072616E67652028302D31AB
:10047000290A0020643A0020693A0020703A0043BB
:10048000290A0061626C656420286D696E207465BC
:100490006D702000436F6C642065787472756465BC
:1004A000732061726520004E6F2063617365206C5C
:1004B000696768740A0041637469766520457874D9
:1004C00072756465723A2000556E6B6E6F776E20A0
:1004D000636F6D6D616E643A20220000002000237E
:1004E00000260029002C002F00320000010000032C
:1004F0000106010901000000000000C0C00000006A
:10050000000000254300003F43000037432F2F2009
:10051000004361703A454D455247454E43595F503F
:1005200041525345523A310A004361703A434153B4
:10053000455F4C494748545F4252494748544E45ED
:1005400053533A300A004361703A544F47474C4581
:100550005F4C49474854533A300A004361703A535C
:100560004F4654574152455F504F5745523A300A13
:10057000004361703A4C4556454C494E475F4441F3
:1005800054413A310A004361703A5A5F50524F4227
:10059000453A310A004361703A4155544F4C455633
:1005A000454C3A310A004361703A5052494E545F0B
:1005B0004A4F423A310A004361703A50524F475213
:1005C0004553533A300A004361703A4155544F52F3
:1005D00045504F52545F54454D503A310A004361E3
:1005E000703A454550524F4D3A310A004649524DF6
:1005F000574152455F4E414D453A4D61726C696EAF
:1006000020204649524D574152455F564552534965
:100610004F4E3A312E312E352E3434204558545217
:10062000554445525F545950453A4165726F737451
:10063000727564657220534F555243455F434F4472
:10064000455F55524C3A68747470733A2F2F636F3C
:1006500064652E616C6570686F626A656374732E81
:10066000636F6D2F646966667573696F6E2F4D4198
:10067000524C494E2050524F544F434F4C5F5645B9
:100680005253494F4E3A312E30204D414348494E46
:10069000455F545950453A4C756C7A426F74204D01
:1006A000696E692032204C434420455854525544C9
:1006B00045525F434F554E543A3120555549443ABF
:1006C00038306665643464362D346431352D343504
:1006D00031322D613032652D3631623164633466DA
:1006E000623037320A0020706F736974696F6E2050
:1006F0006F7574206F662072616E67652E0A003F09
:1007000050726F626520001000C90210012C014078
:1007100001220170011801B0010E01F00104015025
:1007200002FA00B002F0003003E600D003DC0090D3
:1007300004D2007005C800A006BE000008B400B0D6
:1007400009AA00D00BA000600E960060118C00007A
:1007500015820020197800C01D6E00A0226400B030
:10076000275A00902C500000314600E0343C001025
:10077000383200903A2800603C1E00A03D140080F2
:100780003E0A00203F00001000AD0330016A015016
:10079000022B0170030A019004F500B005E500D0BA
:1007A00006D800F007CE001009C500300ABE005080
:1007B0000BB700700CB100900DAB00B00EA600D0CE
:1007C0000FA200F0109D00101299003013950050F8
:1007D00014920070158E0090168B00B0178700D011
:1007E000188400F0198100101B7E00301C7B005023
:1007F0001D7900701E7600901F7300B0207000D02D
:10080000216E00F0226B0010246900302566005034
:100810002663007027610090285E00B0295C00D03C
:100820002A5900F02B5600102D5400302E51005044
:100830002F4E0070304B0090314800B0324500D050
:10084000334200F0343E0010363B00303737005062
:1008500038330070392E00903A2900B03B2300D085
:100860003C1B00F03D1100103F0100F03F00002054
:10087000204E6F7A7A6C653A2000200068656174BA
:10088000206E6F7A7A6C652E0050726573732062E9
:100890007574746F6E20746F005052494E5420501E
:1008A00041555345440020204E6F7A7A6C653A20BA
:1008B00000200066696C616D656E742065787472E5
:1008C000756465005761697420666F720050524903
:1008D0004E54205041555345440020204E6F7A7AA3
:1008E0006C653A2000200066696C616D656E74204D
:1008F0006C6F6164005761697420666F72005052BA
:10090000494E54205041555345440020204E6F7AA3
:100910007A6C653A2000746F20636F6E74696E752F
:10092000652E2E2E00616E642070726573732062D6
:100930007574746F6E00496E736572742066696CAD
:10094000616D656E74005052494E542050415553AC
:1009500045440020204E6F7A7A6C653A20002000D2
:1009600066696C616D656E7420756E6C6F61640094
:100970005761697420666F72005052494E5420507E
:1009800041555345440020204E6F7A7A6C653A20D9
:10099000006368616E6765006F6620746865206635
:1009A000696C616D656E74005761697420666F7261
:1009B000207374617274005052494E542050415556
:1009C0005345440020204E6F7A7A6C653A2000200F
:1009D000004261636B004D696E696D756D205465F1
:1009E0006D70206973203132302E00486561746962
:1009F0006E67206661696C656400426564204C65C1
:100A000076656C696E6720004661696C6564207468
:100A10006F20656E61626C6520426564204C65766E
:100A2000656C696E670A00426564204C6576656C8A
:100A300020436F7272656374696F6E204D617472CA
:100A400069783A0053442063617264206F6B0A0036
:100A50006F70656E526F6F74206661696C65640AB1
:100A600000766F6C756D652E696E697420666169BC
:100A70006C65640A00534420696E6974206661697C
:100A80006C0A00436172642072656D6F7665640064
:100A90004361726420696E736572746564004F66A9
:100AA0006673657473206170706C6965640045726B
:100AB000723A20546F6F206661722100546F6F206C
:100AC0006661722066726F6D207265666572656E12
:100AD000636520706F696E740A0048617264636FA9
:100AE0006465642044656661756C74205365747434
:100AF000696E6773204C6F616465640A0028230087
:100B0000002823000064000000E8030000000096B5
:100B10004300009643000000410000C8410000C9A6
:100B2000420000C942A5C2DF440000D2432028632E
:100B3000616C63756C6174656429210A0020213D34
:100B40002000454550524F4D20435243206D69735C
:100B50006D61746368202D202873746F7265642939
:100B60002000290A002062797465733B2063726358
:100B700020002073746F7265642073657474696EED
:100B80006773207265747269657665642028002039
:100B90004D61726C696E3D563430290A0028454516
:100BA00050524F4D3D00454550524F4D2076657295
:100BB00073696F6E206D69736D617463682000578F
:100BC000726974696E6720746F2066696C653A207B
:100BD000006F70656E206661696C65642C204669E3
:100BE0006C653A20006F70656E206661696C6564A3
:100BF0002C2046696C653A200046696C6520736557
:100C00006C65637465640A002053697A653A200054
:100C100046696C65206F70656E65643A20006F7080
:100C2000656E206661696C65642C2046696C653A66
:100C300020002066696C653A20004E6F7720002204
:100C400020706F73002220706172656E743A22000A
:100C5000535542524F5554494E452043414C4C2028
:100C60007461726765743A22004B494C4C45442EBE
:100C70002000747279696E6720746F2063616C6CF8
:100C8000207375622D67636F64652066696C657398
:100C9000207769746820746F6F206D616E79206CA5
:100CA0006576656C732E204D4158206C6576656CB9
:100CB0002069733A00004D3234004D363030204206
:100CC00030004D3234004D3233202573006175748D
:100CD0006F25692E670043616E6E6F7420656E74B8
:100CE0006572207375626469723A2000022E2E00CC
:100CF0004D61696E0020643A0020693A0020703A24
:100D00000053657474696E672054726176656C2057
:100D1000416363656C65726174696F6E3A2000535C
:100D2000657474696E6720526574726163742041E2
:100D30006363656C65726174696F6E3A2000536518
:100D40007474696E67205072696E742041636365C4
:100D50006C65726174696F6E3A20005365747469D2
:100D60006E67205072696E7420616E6420547261E7
:100D700076656C20416363656C65726174696F6E42
:100D80003A2000204500205A0020204D39303720DD
:100D9000580053746570706572206D6F746F7220A7
:100DA00063757272656E74733A0A0020204D38358F
:100DB00031205A005A2D50726F6265204F6666735B
:100DC000657420286D6D293A0A00204400204900EE
:100DD00020204D3330342050002044002049002092
:100DE000204D3330312050005049442073657474D5
:100DF000696E67733A0A00204600204200204800CE
:100E000020204D3134352053004D61746572696185
:100E10006C2068656174757020706172616D6574B5
:100E20006572733A0A0020204D343230205300415D
:100E300075746F20426564204C6576656C696E67D9
:100E40003A0A00205A0020590020204D3230362026
:100E50005800486F6D65206F66667365743A0A00C6
:100E6000204500205A002059002058002042002030
:100E7000540020204D323035205300416476616E9D
:100E80006365643A20533C6D696E5F6665656472A4
:100E90006174653E20543C6D696E5F747261766565
:100EA0006C5F66656564726174653E20423C6D6985
:100EB0006E5F7365676D656E745F74696D655F6D98
:100EC000733E20583C6D61785F78795F6A65726B1C
:100ED0003E205A3C6D61785F7A5F6A65726B3E2096
:100EE000453C6D61785F655F6A65726B3E0A002004
:100EF000540020520020204D3230342050004163F5
:100F000063656C65726174696F6E2028756E6974B3
:100F1000732F7332293A20503C7072696E745F618E
:100F20006363656C3E20523C726574726163745FEA
:100F3000616363656C3E20543C74726176656C5FDE
:100F4000616363656C3E0A00204500205A00205909
:100F50000020204D3230312058004D6178696D7588
:100F60006D20416363656C65726174696F6E2028E2
:100F7000756E6974732F7332293A0A002045002078
:100F80005A0020590020204D3230332058004D6146
:100F900078696D756D20666565647261746573202E
:100FA00028756E6974732F73293A0A002045002052
:100FB0005A0020590020204D3932205800537465C2
:100FC00070732070657220756E69743A0A00202073
:100FD0004D3230302044300A0020204D3230302055
:100FE00044002044697361626C65640A0046696C60
:100FF000616D656E742073657474696E67733A0011
:1010000020204D3134392043203B20556E697473C4
:1010100020696E2043656C736975730A0020204750
:101020003231202020203B20556E69747320696E78
:10103000206D6D0A00205A3A0020593A0020436F73
:10104000756E7420583A0020453A00205A3A002024
:10105000593A00583A003A20007A5F6D696E3A209A
:10106000202D32207A5F6D61783A202035005A2099
:101070004F666673657420002569730025696D20CD
:10108000256973002569682025696D20256973002D
:10109000256964202569682025696D20256973000C
:1010A00025697920256964202569682025696D20D6
:1010B00025697300656E7175657565696E672022B7
:1010C000004572726F722077726974696E6720745E
:1010D0006F20454550524F4D210A00486F6D6520E5
:1010E0002573257325732066697273740020666901
:1010F0007273740A005A0059005800486F6D6520D9
:10110000000000000000003F4300003743576172B9
:101110006E696E673A20486F6D696E672042756D23
:10112000702044697669736F72203C20310A000296
:1011300002040000A0400000A040000000400000A9
:10114000254300004543000037430000F041000004
:10115000F0410000004100000000FF01014F666601
:10116000004F6E2000456E6473746F702061626F73
:1011700072740053746570732F6D6D004A65726BE5
:1011800000416363656C65726174696F6E005665DA
:101190006C6F63697479005A204F666673657400DA
:1011A000416476616E6365642053657474696E672B
:1011B00073005654726176206D696E0056547261E8
:1011C00076206D696E005654726176206D696E00EE
:1011D000566D696E00566D696E00566D696E0056EB
:1011E0006D6178204500566D6178204500566D612F
:1011F00078204500566D6178205A00566D61782040
:101200005A00566D6178205A00566D617820590059
:10121000566D6178205900566D6178205900566DE1
:101220006178205800566D6178205800566D6178BD
:101230002058004D6F74696F6E004573746570734C
:101240002F6D6D004573746570732F6D6D005A734B
:10125000746570732F6D6D005A73746570732F6DA4
:101260006D005973746570732F6D6D0059737465DB
:1012700070732F6D6D005873746570732F6D6D00F2
:101280005873746570732F6D6D004D6F74696F6E58
:101290000056652D6A65726B0056652D6A65726B26
:1012A0000056652D6A65726B00567A2D6A65726B01
:1012B00000567A2D6A65726B0056792D6A65726BDD
:1012C0000056792D6A65726B0056792D6A65726BCE
:1012D0000056782D6A65726B0056782D6A65726BC0
:1012E0000056782D6A65726B004D6F74696F6E00E1
:1012F0005072696E7420706175736564004D31328F
:1013000035004D6F766520617869730044697361BB
:10131000626C65207374657070657273004D38344B
:1013200000426564204C6576656C696E67004732E3
:10133000382058590A4D31303920533137350A4752
:101340003238205A0A4D31303920523134350A476B
:1013500031320A4732390A4D31303420533000419E
:1013600075746F20686F6D6500473238004D616994
:101370006E0025753A2530327500253032753A25D4
:101380003032750025756420253032753A253032AB
:10139000750000060900FE000000000001090008B9
:1013A000FE000005080806000040F0C8888898780C
:1013B00010050808060000C0F88888888888F805A5
:1013C00005050600012030F8302005080806000059
:1013D0002070F820202020E00509090600FF207079
:1013E000A8A8B8888870200509090600FFE080C019
:1013F000B0A8283028280509090600FFF8A8888821
:10140000888888A8F8050A0A0600FE205050505027
:1014100088A8A8887003030306000340A0400006C4
:101420000900FE070192032120FFFF08FF07FF00CC
:10143000000006000001070706020080808080800F
:101440000080030202060105A0A0050707060000B0
:101450005050F850F850500507070600002078A0BB
:101460007028F020050707060000C0C8102040982B
:10147000180507070600006090A040A890680203C6
:1014800003060104C04080030707060100204080D6
:101490008080402003070706010080402020204074
:1014A0008005050506000120A870A8200505050691
:1014B00000012020F820200203030602FFC0408024
:1014C000050101060003F8020202060200C0C00581
:1014D00005050600010810204080050707060000EA
:1014E0007088888888887003070706010040C0401C
:1014F000404040E0050707060000708808708080C3
:10150000F8050707060000F81020100808F0050786
:101510000706000010305090F8101005070706006D
:1015200000F880F008088870050707060000708042
:1015300080F0888870050707060000F80810202052
:1015400020200507070600007088887088887005CD
:1015500007070600007088887808087002050506ED
:101560000200C0C000C0C00206060602FFC0C000E4
:10157000C040800407070600001020408040201073
:10158000050303060002F800F804070706010080BF
:1015900040201020408005070706000070880810D2
:1015A00020002005070706000070880868A8A870BA
:1015B000050707060000708888F8888888050707EF
:1015C000060000F08888F08888F00507070600000C
:1015D00070888080808870050707060000F0888882
:1015E000888888F0050707060000F88080F0808072
:1015F000F8050707060000F88080F0808080050766
:1016000007060000708880B8888870050707060004
:1016100000888888F888888801070706020080808B
:1016200080808080800507070600003810101010A9
:1016300090600507070600008890A0C0A09088056C
:101640000707060000808080808080F80507070675
:10165000000088D8A88888888805070706000088C1
:1016600088C8A898888805070706000070888888B9
:10167000888870050707060000F08888F080808061
:1016800005070706000070888888A8906805070786
:10169000060000F08888F0A0908805070706000083
:1016A000788080700808F0050707060000F8202001
:1016B0002020202005070706000088888888888861
:1016C000700507070600008888888888502005076D
:1016D000070600008888888888A850050707060044
:1016E00000888850205088880507070600008888F1
:1016F0008850202020050707060000F80810204029
:1017000080F8030707060100E08080808080E00504
:1017100005050600018040201008030707060100A8
:10172000E02020202020E00503030600042050884C
:10173000050101060000F8020202060205804005CC
:101740000505060000700878887805070706000080
:101750008080B0C88888F00505050600007080808C
:1017600088700507070600000808689888887805CB
:1017700005050600007088F8807005070706000060
:101780003048E0404040400506060600FF7088886B
:101790007808700507070600008080B0C888888830
:1017A000010707060200800080808080800308080F
:1017B0000601FF200020202020A04004070706008B
:1017C00000808090A0C0A090030707060100C040E1
:1017D00040404040E0050505060000D0A8A8A8A8A4
:1017E000050505060000B0C88888880505050600BF
:1017F0000070888888700506060600FFF08888F06B
:1018000080800506060600FF7888887808080505A8
:1018100005060000B0C88080800505050600007040
:10182000807008F00407070600004040E040404098
:1018300030050505060000888888986805050506B6
:10184000000088888850200505050600008888A8C3
:10185000A85005050506000088502050880506069A
:101860000600FF888888780870050505060000F8DE
:10187000102040F803070706010020404080404048
:101880002001070706020080808080808080030797
:10189000070601008040402040408005020206000B
:1018A0000268900000000600000000000600000032
:1018B0000000060000000000060000000000060016
:1018C000000000000600000000000600000000000C
:1018D00006000000000006000000000006000000F6
:1018E00000000600000000000600000000000600E6
:1018F00000000000060000000000060000000000DC
:1019000006000000000006000000000006000000C5
:1019100000000600000000000600000000000600B5
:1019200000000000060000000000060000000000AB
:101930000600000000000600000000000600000095
:101940000000060000000000060000000000060085
:10195000000000000600000000000600000000007B
:101960000600000000000600000000000600000164
:101970000707060200800080808080800507070638
:1019800000002070A8A0A8702005070706000030FE
:101990004040E04050A805050506000088705070E2
:1019A00088050707060000885020F820F820010766
:1019B00007060200808080008080800508080600FD
:1019C000003048205050209060030101060107A01C
:1019D000050707060000F888B8B8B888F8050707B3
:1019E000060001700878887800F8050505060001F2
:1019F0002850A05028050303060001F80808020239
:101A0000020602064080050707060000F888A8883D
:101A100098A8F8050101060006F80404040600036E
:101A2000609090600507070600002020F820200045
:101A3000F804050506000360902040F00305050644
:101A40000003E020E020E0020202060206408005DA
:101A500008080600FF8888888898E88080050707BE
:101A600006000078989878181818020202060202F8
:101A7000C0C00202020602FF408003050506000303
:101A800040C04040E0050707060001708888887064
:101A900000F8050505060001A0502850A00507071D
:101AA0000600008890A858B8080805070706000037
:101AB0008890B848982038050808060000C040C043
:101AC00048D8380808050707060000200020408095
:101AD00088700508080600004020007088F8888893
:101AE0000508080600001020007088F8888805089E
:101AF000080600002050007088F88888050808064D
:101B000000006890007088F88888050808060000C2
:101B10005000708888F88888050808060000205062
:101B2000207088F888880507070600003860A0B88C
:101B3000E0A0B80508080600FF7088808088702043
:101B400060050808060000402000F880F080F805D5
:101B50000808060000081000F880F080F805080862
:101B6000060000205000F880F080F8050707060006
:101B7000005000F880F080F803080806010080405B
:101B800000E0404040E0030808060100204000E07B
:101B9000404040E003080806010040A000E040404B
:101BA00040E0030707060100A000E0404040E005D8
:101BB0000707060000704848E8484870050808060E
:101BC000000068900088C8A89888050808060000EA
:101BD000402070888888887005080806000010205A
:101BE00070888888887005080806000020500070FA
:101BF000888888700508080600006890007088884A
:101C00008870050808060000500070888888887071
:101C100005050506000188502050880508080600C3
:101C2000FF1070A8A8A8A87040050808060000408A
:101C30002088888888887005080806000010208899
:101C40008888888870050808060000205000888869
:101C500088887005080806000050008888888888F1
:101C6000700508080600001020885020202020055C
:101C700009090600FFC040704848704040E0040871
:101C8000080601FF609090A09090E080050808068B
:101C900000004020007008788878050808060000D9
:101CA0001020007008788878050808060000205089
:101CB00000700878887805080806000068900070B1
:101CC00008788878050707060000500070087888B3
:101CD00078050808060000205020700878887805EC
:101CE0000606060000D02878A0A8500506060600C3
:101CF000FF70808870206005080806000040200002
:101D00007088F880700508080600001020007088B0
:101D1000F880700508080600002050007088F880E0
:101D20007005070706000050007088F880700308EF
:101D30000806010080400040C04040E0030808065B
:101D4000010020400040C04040E0030808060100B8
:101D500040A00040C04040E0030707060100A0008B
:101D600040C04040E0050707060000A040A01078F2
:101D70008870050808060000689000B0C888888848
:101D80000508080600004020007088888870050853
:101D90000806000010200070888888700508080672
:101DA0000000205000708888887005080806000030
:101DB000689000708888887005070706000050004A
:101DC00070888888700505050600012000F800204D
:101DD0000507070600FF1070A8A8A87040050808AE
:101DE00006000040200088888898680508080600DA
:101DF00000102000888888986805080806000020E0
:101E000050008888889868050707060000500088F9
:101E1000888898680509090600FF102000888888CE
:101E2000F808700407070601FFC04060506040E0FA
:101E30000508080600FF50008888887808705A0056
:101E400059005800092000000000000000000000B8
:101E50000000007FFFE00000000000000000000024
:101E600000007000E0000000000000000000000022
:101E70000061F860000000000000000000000000A9
:101E800041F82000000000000000000000000040B9
:101E9000F020000000000000000000000000406092
:101EA000200000000000000000000000005801A019
:101EB0007F80000000000000004104005C63A0FF80
:101EC000C0000000000000002082005EF7A0FFC0FC
:101ED000000000000000002082005EF7A0FFC000AC
:101EE0000000000000004104005C63A07F8000004F
:101EF00000000000008208005801A07F8000000060
:101F000000000001041000406020FFC0000000003D
:101F100000000104100040F020FFC000000000009D
:101F2000000082080041F820FFC00000000000000F
:101F30000041040061F8603F000000000000000064
:101F40000000007000E01E0000000000000001FF23
:101F5000FF807FFFE00C0000000000000001FFFF99
:101F600080000000000000000000000000000000F1
:101F70007FFFE00000000000000000000000007093
:101F800000E0000000000000000000000000630C02
:101F900060000000000000000000000000470E206C
:101FA0000000000000000000000000004F0F2000B3
:101FB00000000000000000000000005F0FA0000013
:101FC000000000000000000000005E07A07F80000D
:101FD000000000000000410400406020FFC000003D
:101FE000000000000020820040F020FFC000000040
:101FF0000000000020820040F020FFC00000000030
:102000000000004104004060207F800000000000CC
:1020100000008208005E07A07F8000000000000032
:10202000010410005F0FA0FFC000000000000001CD
:102030000410004F0F20FFC00000000000000082CD
:102040000800470E20FFC00000000000000041040F
:1020500000630C603F000000000000000000000072
:102060007000E01E0000000000000001FFFF807F04
:10207000FFE00C0000000000000001FFFF800000F6
:10208000004578747275646572004D6F7665205AEC
:10209000004D6F76652059004D6F76652058004DD4
:1020A0006F76656D656E74004D6F766520302E31EC
:1020B0006D6D004D6F766520316D6D004D6F7665ED
:1020C0002031306D6D004D6F766520617869730049
:1020D0004578747275646572004D6F7665205A009C
:1020E0004D6F76652059004D6F7665205800746FEE
:1020F00020726573756D65005761697420666F7233
:10210000207072696E74005052494E5420504155EF
:102110005345440045787472756465206D6F72652F
:1021200000526573756D65207072696E740052455A
:1021300053554D45204F5054494F4E533A0020209F
:102140004E6F7A7A6C653A20002000506C6561739E
:102150006520776169742E2E2E0048656174696E62
:1021600067206E6F7A7A6C65005052494E54205049
:1021700041555345440000060900FE06018902FE50
:1021800020FFFE07FE06FE0000000600070106060F
:10219000060200808080800080030303060103A004
:1021A000A0A00507070600FF5050F850F850500552
:1021B00009090600FE2070A8A07028A87020060853
:1021C000080600FF40A848102048540805070706E5
:1021D00000FF6090906098906801030306020380FE
:1021E00080800207070602FF4080808080804002D6
:1021F00007070602FF804040404040800505050675
:1022000000008850F850880505050600002020F8D9
:1022100020200204040602FEC040408005010106A1
:102220000002F8020202060200C0C004060606010F
:102230000010102040808004060606010060909087
:1022400090906003060606010040C0404040E00454
:1022500006060601006090102040F0040606060104
:1022600000F020601010E005060606000010305057
:1022700090F810040606060100F080E01010E0045B
:1022800006060601006080E09090600406060601E4
:1022900000F0101020404004060606010060906027
:1022A0009090600406060601006090907010600235
:1022B0000505060200C0C000C0C00207070602FEF6
:1022C000C0C000C0404080050505060000186080C1
:1022D0006018050303060001F800F805050506006F
:1022E00000C0300830C0040707060100609010608D
:1022F0004000400506060600007090A8B0807005FA
:102300000606060000205088F888880506060600A4
:1023100000F088F08888F0040606060100609080CE
:10232000809060040606060100E090909090E00422
:102330000606060100F080E08080F0040606060133
:1023400000F080E080808004060606010060908036
:10235000B090600406060601009090F09090900303
:102360000606060100E040404040E0050606060083
:102370000038101010906004060606010090A0C0FE
:10238000A090900406060601008080808080F00501
:10239000060606000088D8A8A88888040606060154
:1023A0000090D0B0909090050606060000708888D6
:1023B000888870040606060100E09090E0808004A2
:1023C00007070601FF609090D0B060100406060673
:1023D0000100E09090E090900406060601006090F5
:1023E00040209060050606060000F82020202020EE
:1023F0000406060601009090909090600406060680
:102400000100909090F06060050606060000888844
:10241000A8A8D88805060606000088502020508805
:1024200005060606000088885020202004060606BF
:102430000100F010204080F0030606060100E08055
:10244000808080E004060606010080804020101095
:10245000030606060100E020202020E00503030615
:1024600000032050880501010600FEF80202020662
:102470000204804004040406010070909070040679
:10248000060601008080E09090E00404040601004C
:102490007080807004060606010010107090907025
:1024A00004040406010060B0C070040606060100C2
:1024B000205040E040400406060601FE6090907007
:1024C00010600406060601008080E09090900306EC
:1024D000060601004000C04040E00308080601FE77
:1024E000200060202020A040040606060100808015
:1024F000A0C0A090030606060100C040404040E096
:10250000050404060000D0A8A888040404060100FD
:10251000E09090900404040601006090906004062E
:10252000060601FEE09090E080800406060601FEAB
:10253000709090701010040404060100A0D08080F8
:1025400004040406010070C030E004060606010021
:102550004040E04050200404040601009090907038
:102560000404040601009090606005040406000065
:1025700088A8A85004040406010090606090040636
:10258000060601FE9090907090600404040601001D
:10259000F02040F003070706010020404080404043
:1025A000200107070602FF8080808080808003076B
:1025B00007060100804040204040800402020601DE
:1025C0000350A0FFFFFFFFFFFFFFFFFFFFFFFFFF25
:1025D000FFFFFFFFFFFFFFFFFFFFFFFFFFFFFFFF0B
:1025E000FFFFFFFF000000060007010606060200CD
:1025F0008000808080800406060601FF2070A0A075
:1026000070200507070600FF304840F04040F805FD
:102610000505060000A8508850A80506060600001B
:102620008850F820F8200107070602FF808080000C
:102630008080800407070601FF708060906010E0D2
:10264000030101060105A00607070600007884942F
:10265000A494847803050506010160A06000E005EC
:1026600005050600002850A05028040303060100B9
:10267000F01010040101060102F006070706000031
:102680007884B4A4A48478040101060105F004034D
:10269000030601026090600507070600FF2020F88E
:1026A000202000F803050506010140A02040E003BA
:1026B0000505060101C0204020C0020202060204F6
:1026C00040800405050601FF9090B0D08005060605
:1026D00006000078E8E86828280101010602028067
:1026E0000202020602FE408003050506010140C009
:1026F0004040E003050506010140A04000E005055B
:1027000005060000A0502850A00508080600FF405C
:10271000C04050703078100508080600FF40C040E7
:1027200050680810380508080600FFC0204030F047
:1027300030781004070706010020002060809060B8
:10274000050707060000402020507088880507070D
:10275000060000102020507088880507070600003A
:102760002050205070888805070706000028502058
:1027700050708888050707060000500020507088B8
:10278000880507070600002050205070888805063D
:102790000606000078A0F0A0A0B80408080601FE14
:1027A0006090808090602040040707060100402070
:1027B000F080E080F00407070601002040F080E090
:1027C00080F00407070601002050F080E080F0044C
:1027D00007070601005000F080E080F003070706BD
:1027E00001008040E0404040E00307070601002070
:1027F00040E0404040E003070706010040A0E04001
:102800004040E0030707060100A000E0404040E030
:102810000506060600007048E848487004070706E9
:10282000010050A090D0B09090040707060100402E
:10283000206090909060040707060100204060909F
:10284000909060040707060100205060909090600F
:1028500004070706010050A06090909060040707ED
:10286000060100500060909090600505050600008C
:1028700088502050880408080601FF1070B0B0D0BE
:10288000D0E08004070706010040209090909060FF
:10289000040707060100204090909090600407070D
:1028A00006010020509090909060040707060100F8
:1028B0005000909090906005070706000010208857
:1028C0005020202004060606010080E09090E08061
:1028D0000406060601006090A0A090A00407070669
:1028E000010040200070909070040707060100204E
:1028F000400070909070040707060100205000709F
:1029000090907004070706010050A000709090702E
:102910000406060601005000709090700407070638
:102920000100205020709090700504040600007093
:10293000A8B0780406060601FE708080702040046E
:10294000070706010040200060B0C07004070706BA
:10295000010020400060B0C070040707060100209D
:10296000500060B0C070040606060100500060B060
:10297000C070030707060100804000C04040E0032C
:102980000707060100204000C04040E0030707069B
:10299000010040A000C04040E0030606060100A080
:1029A00000C04040E004070706010030601070904E
:1029B000906004070706010050A000E0909090048A
:1029C000070706010040200060909060040707069A
:1029D000010020400060909060040707060100207D
:1029E00050006090906004070706010050A000604E
:1029F000909060040606060100500060909060050B
:102A000005050600002000F800200404040601006B
:102A100070B0D0E0040707060100402000909090BD
:102A20007004070706010020400090909070040792
:102A300007060100205000909090700406060601E1
:102A4000005000909090700409090601FE2040009B
:102A50009090907090600408080601FE8080E090DD
:102A600090E080800408080601FE5000909090706D
:102A7000906000002200250028002B002E0031006D
:102A8000340002010000050108010B0100002100D3
:102A9000240027002A002D0030003300010100002F
:102AA000040107010A0105050505070508080808CE
:102AB000020202020A0A08080404040401010101D6
:102AC00001010101030303030303030304070707D1
:102AD0000C0C0C0C0C0C0C0C020202020606060676
:102AE000060606060B0B0B0B0B0B0B0B0102102043
:102AF0002008081020401020408002010201080434
:102B000002010102040810204080804020100804C7
:102B10000201800402018040201008040201080420
:102B20000201010204081020408001020408102064
:102B3000408000000A0B02090C0D0E080703040177
:102B40000000000000000000000000000000000085
:102B50000000000000000000000000000000121152
:102B60001000000000000000000000000000000055
:102B7000000000000000000045303A20005A3A20D2
:102B800000593A2000583A20004D53312C4D533211
:102B90002050696E730A002042002050006F6B00C5
:102BA0005265776970696E670050726F62696E670F
:102BB000206661696C65640050726F62696E67209F
:102BC0006661696C65640050524F42452046414938
:102BD0004C20434C45414E204E4F5A5A4C450A001A
:102BE0005265776970696E670A0052657769706926
:102BF0006E670050726F62696E67206661696C650E
:102C0000640050726F62696E67206661696C65640A
:102C10000050524F4245204641494C20434C4541CB
:102C20004E204E4F5A5A4C450A00526577697069DA
:102C30006E670A0050726F62696E67206661696C28
:102C400065640A0050726F62696E67206661696C24
:102C5000656400205A3A200020593A2000426564F9
:102C600020583A20000A0A426564204C6576656C5B
:102C700020436F7272656374696F6E204D61747268
:102C800069783A00202B000A436F7272656374659D
:102C90006420426564204865696768742076732EF5
:102CA0002042656420546F706F6C6F67793A0A0038
:102CB000202B000A426564204865696768742054C7
:102CC0006F706F6772617068793A0A2020202B2D2F
:102CD0002D2D204241434B202D2D2B0A2020207CDE
:102CE00020202020202020202020207C0A204C2072
:102CF0007C20202020282B29202020207C20520AE4
:102D00002045207C20202020202020202020207CE6
:102D100020490A2046207C20282D29204E20282BBF
:102D200029207C20470A2054207C2020202020209D
:102D300020202020207C20480A2020207C202020C9
:102D400020282D29202020207C20540A2020207C8F
:102D500020202020202020202020207C0A2020202D
:102D60004F2D2D2046524F4E54202D2D2B0A20281A
:102D7000302C30290A004D65616E206F662073612A
:102D80006D706C656420706F696E74733A200020FA
:102D9000643A200020623A200045716E20636F651E
:102DA0006666696369656E74733A20613A20005201
:102DB000756E6E696E6720696E204452592D5255AA
:102DC0004E206D6F64650A00473239204175746F7B
:102DD00020426564204C6576656C696E670A002840
:102DE000422961636B00284629726F6E7400285275
:102DF000296967687400284C29656674003F4E7520
:102E00006D626572206F662070726F626520706FF0
:102E1000696E747320697320696D706C6175736974
:102E2000626C65202832206D696E696D756D292E82
:102E30000A003F2856296572626F7365206C6576BB
:102E4000656C20697320696D706C61757369626C63
:102E5000652028302D34292E0A007C3C3E5E2B3D17
:102E60003F2F5B5D3B2C2A225C0043616E6E6F74CA
:102E7000206F70656E207375626469722000456E04
:102E8000642066696C65206C6973740A004265672A
:102E9000696E2066696C65206C6973740A00466906
:102EA0006C652064656C657465643A0044656C65A6
:102EB00074696F6E206661696C65642C2046696C6C
:102EC000653A20006F70656E206661696C65642CE0
:102ED0002046696C653A200001050800FF060121C3
:102EE000023520FFFF07FF06FF090050221656801B
:102EF0008080800080153353A0A0A0025757505007
:102F0000F850F850500257572070A07028702013C6
:102F1000355580A040A02002475740A0A040A0A067
:102F20005025135380808012265640808080804038
:102F30001226568040404040800245559060F06027
:102F4000900255552020F820201133536040800412
:102F50004151F011335340E04002465610102040DA
:102F6000808012365640A0A0A0A04012365640C025
:102F7000404040E00246566090106080F0024656A5
:102F8000F020601090600246562060A0F0202002E1
:102F90004656F080E01090600246566080E09090C7
:102FA00060024656F0102020404002465660906075
:102FB000909060024656609090701060122555C047
:102FC000C000C0C0113656606000604080123656A6
:102FD000204080804020034353F000F0123656809A
:102FE000402020408012365640A02040004001582A
:102FF00058304898A8A8904030024656609090F00B
:103000009090024656E090E09090E0024656609024
:1030100080809060024656E090909090E002465684
:10302000F080E08080F0024656F080E080808002F0
:103030004656609080B090600246569090F0909016
:1030400090123656E040404040E002465670202044
:1030500020A04002465690A0C0A0A09002465680F4
:1030600080808080F002465690F0F090909002466A
:103070005690D0F0B0B0900246566090909090601C
:10308000024656E09090E08080014757609090D0D3
:10309000B06010024656E09090E090900246566074
:1030A0009040209060123656E0404040404002463A
:1030B00056909090909060024656909090906060EC
:1030C000024656909090F0F09002465690906060C4
:1030D0009090025656888850202020024656F010C4
:1030E000204080F0123656E080808080E002465614
:1030F000808040201010123656E020202020E0165C
:10310000325240A0014151F01622528040024454F4
:10311000709090700246568080E09090E012345497
:103120006080806002465610107090907002445487
:1031300060B0C060024656205040E0404001455516
:1031400060907010600246568080E0909090123639
:10315000564000C04040E01137572000202020A0FA
:1031600040024656808090E09090123656C0404013
:103170004040E0025454D0A8A8A8024454E09090E3
:103180009002445460909060014555E090E080804A
:103190000145557090701010024454A0D0808012E8
:1031A000345460C020C00246564040E040502002E7
:1031B000445490909070123454A0A0A040025454F3
:1031C00088A8A850024454906060900145559090A2
:1031D000709060024454F02040F002475730402085
:1031E000C020403022165680808080808002475761
:1031F000C02040304020C006425250A0FFFFFFFFD9
:10320000FFFFFFFFFFFFFFFFFFFFFFFFFFFFFFFFCE
:10321000FFFFFFFFFFFFFFFFFFFFFFFFFF09005062
:103220002216568000808080800146562070A0A023
:1032300070200246562050E04050A002555588703C
:103240005070880256568850F820F8202217578070
:103250008080008080800247577080E0907010E08E
:10326000173151A002565670A8C8C8A87014355519
:1032700060A06000E003435350A050123353E0209D
:1032800020143151E002565670E8D8E8D870173152
:1032900051E015335340A04012355540E04000E066
:1032A00014355540A02040E0143555C020C020C042
:1032B0001622524080014555909090E0800256566B
:1032C00078E8E8682828241151801122524080149F
:1032D000355540C04040E014355540A04000E00363
:1032E0004353A050A0024757808080A060F0200286
:1032F00047578080A0D010207002475780408060E0
:10330000A0F02012365640004080A04002475740AF
:10331000206090F0909002475720406090F090908D
:1033200002475760906090F0909002475750A0601D
:1033300090F0909002475790006090F09090024774
:103340005760906090F0909002465670A0A0F0A058
:10335000B0014757609080809060400247574020FE
:10336000F080E080F00247572040F080E080F002DB
:1033700047576090F080E080F00247579000F0805F
:10338000E080F01237578040E0404040E01237576D
:103390002040E0404040E012375740A0E04040402D
:1033A000E0123757A000E0404040E0025656704817
:1033B000E848487002475750A090D0B0909002471C
:1033C0005740206090909060024757204060909056
:1033D000906002475760906090909060024757500D
:1033E000A06090909060024757900060909090602D
:1033F000123353A040A002465670B0B0D0D0E002C5
:1034000047574020909090906002475720409090FE
:10341000909060024757609090909090600247575C
:103420009000909090906002575710208850202074
:103430002002465680E09090E0800246566090A0C0
:10344000A090A0024757402000709090700247570C
:10345000204000709090700247572050007090906C
:103460007002475750A0007090907002465650006E
:103470007090907002475760906070909070025406
:1034800054F068B07811355560808060400247572D
:1034900040200060B0C06002475720400060B0C0CC
:1034A0006002475760900060B0C06002465650000E
:1034B00060B0C060123757804000C04040E0123713
:1034C00057204000C04040E012375740A000C040A5
:1034D00040E0123656A000C04040E0024757A040EE
:1034E000A01070906002475750A000E090909002AA
:1034F000475740200060909060024757204000608E
:10350000909060024757609000609090600247572B
:1035100050A00060909060024656900060909060CD
:103520001235554000E0004002445470B0D0E00233
:1035300047574020009090907002475720400090DD
:10354000909070024757609000909090700246569D
:10355000900090909070014858204000909070909A
:10356000600147578080E090E080800147579000DD
:10357000909070906001050700FE0500FB01F220AD
:10358000FFFE05FE05FE020040021525808080003A
:1035900080053242A0A002556550F850F85001460F
:1035A000562070C030E0200255659010204048023F
:1035B000556560806890680512228080022535403C
:1035C000808080400225358040404080043343A005
:1035D00040A003334340E0400122324080043141A7
:1035E000E0021121800255650810204080024555F7
:1035F0006090909060022535C040404040024555A3
:10360000E0106080F0024555E0106010E002455582
:103610002060A0F020024555F080E010E002455502
:103620006080E09060024555F01020404002455512
:1036300060906090600245556090701060031323A5
:103640008000800214248000808002354520408064
:103650004020033343E000E00235458040204080B5
:10366000024555E0106000400255657088B8A870AA
:10367000024555609090F090024555E090E090E052
:103680000235456080808060024555E0909090E072
:10369000023545E080E080E0023545E080E0808052
:1036A0000245557080B090700245559090F0909012
:1036B000023545E0404040E0024555301010906032
:1036C00002455590A0C0A09002354580808080E0E2
:1036D00002556588D8A8888802455590D0B090904A
:1036E0000245556090909060024555E09090E080D2
:1036F000014656609090906010024555E09090E031
:103700009002455570806010E0023545E040404031
:103710004002455590909090600245559090A0A031
:103720004002556588A8A8A8500245559090609021
:10373000900245559090701060023545E020408021
:10374000E0022535C0808080C00255658040201091
:1037500008022535C0404040C005324240A0024129
:1037600051F005223280400244547090907002451E
:103770005580E09090E002344460808060024555BE
:10378000107090907002445460B0C06002354520C3
:1037900040E04040004656709090701060024555E1
:1037A00080E090909002152580008080800027376F
:1037B000400040404040800245558090A0E090028B
:1037C00015258080808080025464F0A8A8A8024457
:1037D00054E090909002445460909060004656E00F
:1037E0009090E080800046567090907010100234E7
:1037F00044A0C0808002445470C030E0023545408F
:10380000E0404020024454909090700244549090C4
:10381000A040025464A8A85050023444A04040A0E4
:10382000004656909090701060024454F02040F092
:103830000235456040804060021525808080808090
:10384000023545C0402040C005425250A0FFFFFF56
:10385000FFFFFFFFFFFFFFFFFFFFFFFFFFFFFFFF78
:10386000FFFFFFFFFFFFFFFFFFFFFFFFFFFF020064
:1038700040FFFFFFFFFFFFFFFFFFFFFFFFFFFFFF17
:10388000FFFFFFFFFFFFFFFFFFFFFFFFFFFFFFFF48
:10389000FFFFFFFFFFFFFFFFFFFFFFFFFFFFFFFF38
:1038A000FFFFFFFFFFFFFFFFFFFFFFFFFFFFFFFF28
:1038B000FFFFFFFFFFFFFFFFFFFFFFFFFFFFFFFF18
:1038C000FFFFFFFFFFFFFFFFFFFFFFFFFFFFFFFF08
:1038D00001060D00FE09016602D620FFFE0BFE0A5E
:1038E000FE0D0060221969808080808080800080C9
:1038F000183363A0A0A00357675050F850F85050F9
:103900000259692078A0A0702828F020025969483F
:10391000A85010204050A89002586840A0A040A095
:10392000989068281363808080113B6B2040408012
:1039300080808080404020113B6B804040202020D0
:10394000202040408006556520A870A820045565B9
:103950002020F82020113363604080065161F81167
:10396000336340E04002596908081010204040804D
:1039700080025969205088888888885020025969B7
:103980002060A02020202020F80259697088880833
:1039900010204080F8025969F80810207008088843
:1039A00070025969101030505090F8101002596987
:1039B000F88080B0C80808887002596970888080D3
:1039C000F088888870025969F8081010202040405B
:1039D000400259697088888870888888700259699F
:1039E00070888888780808887011386840E040003E
:1039F0000040E04011386840E04000006040800234
:103A00005969081020408040201008045464F800D0
:103A100000F80259698040201008102040800259A7
:103A200069708888081020200020025969708888F1
:103A300098A8A8B080780259692050888888F888AA
:103A40008888025969F048484870484848F0025947
:103A500069708880808080808870025969F0484849
:103A60004848484848F0025969F8808080F08080D2
:103A700080F8025969F8808080F080808080025947
:103A800069708880808098888870025969888888E1
:103A900088F888888888123969E040404040404072
:103AA00040E002596938101010101010906002594F
:103AB00069888890A0C0A090888802596980808019
:103AC0008080808080F80259698888D8A8A8888872
:103AD000888802596988C8C8A8A89898888802590F
:103AE00069708888888888888870025969F0888811
:103AF00088F080808080015A6A70888888888888E9
:103B0000A87008025969F0888888F0A09088880217
:103B10005969708880807008088870025969F82097
:103B200020202020202020025969888888888888C1
:103B300088887002596988888888505050202002EF
:103B4000596988888888A8A8A8A8500259698888CF
:103B50005050205050888802596988885050202041
:103B6000202020025969F808101020404080F811E8
:103B70003B6BE0808080808080808080E00259699B
:103B8000808040402010100808113B6BE02020206E
:103B9000202020202020E00853632050880151611C
:103BA000F82A226280400256667008788898680277
:103BB0005969808080F088888888F002566670880D
:103BC0008080887002596908080878888888887811
:103BD0000256667088F88088700259693048404003
:103BE000F0404040400058687088888878088870A5
:103BF000025969808080B0C88888888812386840F7
:103C000000C040404040E0004A6A100030101010F0
:103C10001090906002596980808090A0C0A0908828
:103C2000123969C040404040404040E0025666D0F2
:103C3000A8A8A8A888025666B0C8888888880256AE
:103C400066708888888870005868F0888888F08056
:103C50008080005868788888887808080802566646
:103C6000B0C88080808002566670886010887002BC
:103C700058684040F0404040483002566688888886
:103C80008898680256668888885050200256668850
:103C900088A8A8A85002566688502020508800584E
:103CA000688888889868088870025666F8102040EE
:103CB00080F8015B6B1820202020C02020202018D5
:103CC000221969808080808080808080015B6BC049
:103CD000202020201820202020C008536348A890CE
:103CE000FFFFFFFFFFFFFFFFFFFFFFFFFFFFFFFFE4
:103CF000FFFFFFFFFFFFFFFFFFFFFFFFFFFFFFFFD4
:103D0000FF0D0060221969800080808080808080A3
:103D10000358682070A8A0A0A870200259693048F4
:103D20004040E0404048B00356668870505070886C
:103D300002596988885050F820F82020221969809B
:103D40008080800080808080124A6A6090806090CD
:103D500090601090601A3262A0A00359697088A820
:103D6000D8C8D8A88870045767700878887800F891
:103D70000356662850A0A05028045363F80808167C
:103D80003161E00359697088E8D8D8E8D888700AAA
:103D90005161F8174464609090600357672020F8E1
:103DA000202000F807356540A02040E00735654039
:103DB000A04020C02A2262408000586888888888F5
:103DC00098E8808002596978E8E8E8E868282828B7
:103DD000262161C0202262408007356540C04040F6
:103DE000E0045767708888887000F8035666A05012
:103DF000282850A0025A6A40C04040E008182838DD
:103E000008025A6A40C04040E01028081038025AA0
:103E10006A40A04020A048182838080259692000AC
:103E200020204080888870025A6A402000205088F4
:103E300088F88888025A6A10200020508888F888FC
:103E400088025A6A30480020508888F88888025AC8
:103E50006A28500020508888F88888025A6A505092
:103E60000020508888F88888025A6A205020205004
:103E70008888F8888802596958A0A0A0B0E0A0A05E
:103E8000B8005B6B708880808080808870204002E2
:103E90005A6A402000F88080F08080F8025A6A1048
:103EA0002000F88080F08080F8025A6A304800F8DC
:103EB0008080F08080F8025A6A505000F88080F0CC
:103EC0008080F8123A6A804000E04040404040E084
:103ED000123A6A204000E04040404040E0124A6A06
:103EE000609000E04040404040E0123A6AA0A000EC
:103EF000E04040404040E0025969F0484848E84806
:103F00004848F0025A6A2850008888C8A8988888CB
:103F1000025A6A40200070888888888870025A6A2D
:103F200010200070888888888870025A6A3048009B
:103F300070888888888870025A6A2850007088883B
:103F400088888870025A6A505000708888888888EB
:103F5000700355658850205088015B6B08709898F5
:103F6000A8A8A8C8C87080025A6A4020008888881B
:103F700088888870025A6A10200088888888888813
:103F800070025A6A30480088888888888870025A87
:103F90006A50500088888888888870025A6A102081
:103FA000008888502020202002596980F088888865
:103FB000F0808080025969609090A0A0908888B0BD
:103FC0000259694020007008788898680259691081
:103FD0002000700878889868025969304800700895
:103FE000788898680259692850007008788898681D
:103FF000025969505000700878889868025A6A30EF
:10400000483000700878889868025666702870A05A
:10401000A8500058687088808088702040025969D4
:104020004020007088F88088700259691020007064
:1040300088F88088700259693048007088F8808854
:10404000700259695050007088F880887012396980
:10405000804000C040404040E0123969204000C02C
:1040600040404040E0124969609000C040404040FC
:10407000E0123969A0A000C040404040E0025A6A06
:104080005020601070888888887002596928500014
:10409000B0C888888888025969402000708888885C
:1040A00088700259691020007088888888700259C9
:1040B00069304800708888888870025969285000E3
:1040C0007088888888700259695050007088888884
:1040D0008870035767202000F800202001586808E6
:1040E0007098A8A8C8708002596940200088888804
:1040F0008898680259691020008888888898680222
:1041000059693048008888888898680259695050F1
:1041100000888888889868005B6B102000888888F1
:104120009868088870005A6A8080B0C88888C8B0CB
:104130008080005B6B505000888888986808887081
:10414000000000000000000000000000000000006F
:10415000000000000000000000000000000000005F
:104160000000000C000000000000000C0000000037
:10417000000000120000000000000023000000000A
:1041800000000021000000000000004C8000000042
:104190000000005E8000000000000092400000006F
:1041A000000000A1400000000000012120000000EC
:1041B0000000027F900000000000020010000000DC
:1041C000000007FFF80000000000040008000000E5
:1041D00000000800040000000000080006000000C5
:1041E00000001000020000000000301E010000006E
:1041F0000000207F81000000000041FFE0800000FF
:10420000000043FCF08000000000873B7840000085
:1042100000018EDBFC60000000010FEBCC200000F1
:1042200000021FEDB610000000021FDEB6100000F5
:10423000000439CD7F080000000436E0FF080000CC
:1042400000087EC0BB84000000187F005D8600006F
:1042500000107FC0ED82000000203CC07301000010
:1042600000203B337F01000000701BE77E038000CD
:1042700000C81DEEDE04C00000880FDEDC04400034
:1042800001240FDF3C092000012607DBF81920007C
:10429000027203E7F0139000025101FFE022900048
:1042A0000489007F802448000904801E00482400FF
:1042B0000BFE400000DFF400100040000080020010
:1042C0001FFFFFFFFFFFFE000000000000000000D6
:1042D00000000000000000000000000000000000DE
:1042E0001022103C3C0E1F0010221004221104006A
:1042F0001022100822110400102210083C110400A2
:10430000102210102211040010221020221104008B
:104310001E1C1E3C3C0E04000000000000000000BB
:10432000000000000000000000000000000000008D
:10433000000000000000000000000000000000007D
:10434000000000000000000000000000000000006D
:10435000000000000000000000000000000000005D
:10436000000000000000000000000000000000004D
:1043700000000000000000000000000000000A0033
:104380003B20454550524F4D20496E6465783A2098
:10439000005570646174696E67207A6F6666736534
:1043A0007420696E20454550524F4D3A200006005A
:1043B00006000600060006000600060006000600CD
:1043C0003FC01F800F00060006000F001F803FC087
:1043D00006000600060006000600060006000600AD
:1043E000060007F8000C0C0010020020010060011C
:1043F000804000804003E04001C040008040000059
:104400004000006000002000001000000C0C0007BD
:10441000F80001FE000303000400800800401800BB
:10442000601000207C0020380020100020000020B8
:104430000000200000600000400000800303000135
:10444000FE00FFFFFF7F80FFC0FFC0FFC07F807FB7
:1044500080FFC0FFC0FFC03F001E000C005A204F6D
:104460006666736574004D6F76652058004D6F76F3
:10447000652059004D6F7665205A00457874727535
:10448000646572004B494C4C45442E200024F4D402
:104490003050C38E20C2A24017828B7011127A91C5
:1044A0000D816CD90AA861E108C7586607615143BC
:1044B000061E4B5D05C145A7041A411104093D982C
:1044C00003713931034036DB0265339102D4305435
:1044D00002802E1D02632CEE01752AC501B028A0B2
:1044E00001102781018F2564012B244B01E0223428
:1044F00001AC211F018D200D01801FFC00841EEDE9
:1045000000971DDF00B81CD200E61BC600201BBCB4
:1045100000641AB200B219A8000A19A0006A18991A
:1045200000D117910040178B00B516840031167E1C
:1045300000B31579003A157300C7146F0058146A58
:1045400000EE1366008813630025135E00C7125B3C
:10455000006C12570015125400C111510070114F18
:104560000021114B00D61049008D10470046104421
:104570000002104200C00F4000800F3E00420F3C7E
:1045800000060F3B00CB0E3800930E37005C0E3553
:1045900000270E3400F30D3200C10D3100900D30B4
:1045A00000600D2E00320D2D00050D2C00D90C2BB6
:1045B00000AE0C2900850C29005C0C2700350C2767
:1045C000000E0C2600E80B2400C40B2400A00B23D3
:1045D000007D0B23005A0B2100390B2100180B2002
:1045E00000F80A1F00D90A1E00BB0A1E009D0A1D02
:1045F00000800A1D00630A1C00470A1B002C0A1BCE
:1046000000110A1A00F7091A00DD091900C4091976
:1046100000AB091900920917007B091800630917FC
:10462000004C09160036091600200916000A091563
:1046300000F5081500E0081400CC081400B80814B0
:1046400000A4081400900813007D0812006B0813E2
:1046500000580812004608120034081100230811FF
:10466000001208110001081100F0071000E0071007
:1046700000D0071000C0071000B0070F00A10710FE
:104680000091070E0083070F0074070F0065070EE7
:104690000057070E0049070E003B070D002E070EBE
:1046A0000020070D0013070D0006070D00F9060C8A
:1046B00000ED060D00E0060C00D4060C00C8060C48
:1046C00000BC060C00B0060C00A4060B0099060CFA
:1046D000008D060B0082060B0077060B006C060BA4
:1046E0000061060A0057060B004C060A0042060A43
:1046F0000038060A002E060A0024060A001A060AD6
:10470000001006090007060A00FD050900F4050966
:1047100000EB050900E2050900D9050900D00509EB
:1047200000C7050900BE050900B5050800AD05086C
:1047300000A50509009C050800940508008C0508E3
:1047400000840508007C050800740508006C050756
:1047500000650508005D050700560508004E0507C1
:104760000047050700400508003805070031050728
:10477000002A050700230507001C0506001605078B
:10478000000F0507000805060002050700FB0406E8
:1047900000F5040700EE040600E8040600E2040742
:1047A00000DB040600D5040600CF040600C9040699
:1047B00000C3040600BD040600B7040600B10405EA
:1047C00000AC040600A6040600A00405009B040635
:1047D0000095040500900406008A04050085040580
:1047E00000800406007A04050075040500700405C5
:1047F000006B04050066040500610405005C040507
:104800000057040500520405004D04050048040546
:1048100000430405003E0404003A04050035040585
:1048200000300404002C04050027040400230405C0
:10483000001E0404001A04040016040500110404F8
:10484000000D04040009040500040404000004042D
:1048500000FC030400F8030400F4030400F0030464
:1048600000EC030400E8030400E4030400E0030494
:1048700000DC030400D8030400D4030400D00304C4
:1048800000CC030400C8030300C503030024F404A0
:10489000D9201BC40C5C0E9804C4095F0265077123
:1048A00001F405F900FB04B30048048700C1036963
:1048B000005803550003034500BE023A008402314C
:1048C0000053022A002902250004022000E4011CF2
:1048D00000C8011900AF01170098011400840113EA
:1048E00000710110006101100051010E0043010D23
:1048F0000036010B002B010B0020010B00150109F4
:10490000000C01090003010800FB000800F3000887
:1049100000EB000700E4000600DE000600D80006F9
:1049200000D2000600CC000500C7000500C200054B
:1049300000BD000400B9000400B5000400B100048B
:1049400000AD000400A9000400A5000300A20003BC
:10495000009F0004009B00030098000300950002E4
:104960000093000300900003008D0002008B000301
:10497000008800020086000200840003008100021B
:10498000007F0002007D0002007B0002007900022F
:10499000007700010076000200740002007200013E
:1049A00000710002006F0002006D0001006C000247
:1049B000006A000100690002006700010066000152
:1049C0000065000100640002006200010061000156
:1049D00000600001005F0002005D0001005C00015A
:1049E000005B0001005A000100590001005800015D
:1049F000005700010056000100550001005400015D
:104A0000005300000053000100520001005100015A
:104A100000500001004F0001004E0000004E000158
:104A2000004D0001004C0001004B0000004B000154
:104A3000004A000100490001004800000048000150
:104A4000004700010046000000460001004500004C
:104A50000045000100440001004300000043000144
:104A6000004200000042000100410000004100013E
:104A700000400001003F0000003F0001003E000038
:104A8000003E0001003D0000003D0001003C000030
:104A9000003C0000003C0001003B0000003B000126
:104AA000003A0000003A000100390000003900011E
:104AB0000038000000380000003800010037000016
:104AC000003700010036000000360000003600010B
:104AD0000035000000350000003500010034000002
:104AE00000340000003400010033000000330000F7
:104AF00000330001003200000032000000320001EB
:104B000000310000003100000031000100300000E1
:104B10000030000000300001002F0000002F0000D6
:104B2000002F0000002F0001002E0000002E0000CA
:104B3000002E0001002D0000002D0000002D0000BF
:104B4000002D0001002C0000002C0000002C0000B3
:104B5000002C0001002B0000002B0000002B0000A7
:104B6000002B0001002A0000002A0000002A00009B
:104B7000002A00010029000000290000002900008F
:104B80000029000000290001002800000028000082
:104B90000028000000280000002800010027000075
:104BA0000027000000270000002700000027000168
:104BB000002600000026000000260000002600005D
:104BC000002600010025000000250000002500004F
:104BD0000025000000250000002500010024000041
:104BE0000024000000240000002400000024000134
:104BF0000023000000230000002300000023000029
:104C00000023000000230000002300010022000018
:104C1000002200000022000000220000002200000C
:104C200000220001002100000021000000210000FE
:104C300000210000002100000021000000210001EF
:104C400000200000002000000020000000200000E4
:104C500000200000002000000020000000200001D3
:104C6000001F0000001F0000001F0000001F0000C8
:104C7000001F0000001F0000001F0001001E0000B8
:104C8000001E0000001E0000001E0000004D383411
:104C900020582059205A2045004572723A204D492B
:104CA0004E54454D5020424544004D494E54454DCB
:104CB0005020747269676765726564004572723A64
:104CC000204D494E54454D50204531004572723AB1
:104CD000204D494E54454D50204530004572723AA2
:104CE000204D415854454D5020424544004D4158B7
:104CF00054454D502074726967676572656400455C
:104D000072723A204D415854454D5020453100456E
:104D100072723A204D415854454D50204530004D57
:104D200036303020486F74656E6420746F6F206376
:104D30006F6C6420746F206368616E6765206669BC
:104D40006C616D656E740A004B64200023646566B7
:104D5000696E65202044454641554C545F004B69BF
:104D6000200023646566696E6520204445464155F0
:104D70004C545F004B70200023646566696E6520AB
:104D80002044454641554C545F00504944204175EC
:104D9000746F74756E652066696E697368656421E9
:104DA0002050757420746865206C617374204B709A
:104DB0002C204B6920616E64204B6420636F6E73FE
:104DC00074616E74732066726F6D2062656C6F77AC
:104DD00020696E746F20436F6E66696775726174C7
:104DE000696F6E2E680A00504944204175746F74D3
:104DF000756E65206661696C6564212074696D65F6
:104E00006F75740A00504944204175746F74756E53
:104E100065206661696C6564212054656D706572FA
:104E2000617475726520746F6F20686967680A0025
:104E3000204B643A2000204B693A2000204B703A06
:104E400020000A20436C6173736963205049442039
:104E50000A002054753A2000204B753A2000206D3E
:104E600061783A2000206D696E3A200020643A2073
:104E70000020626961733A2000526573656E643A7E
:104E800020005344207072696E74696E67206279E5
:104E9000746520004E6F74205344207072696E74E4
:104EA000696E670A00290A002062797465733B20E5
:104EB000637263200053657474696E677320537462
:104EC0006F72656420280020496E76616C696420E9
:104ED00065787472756465722000205A002059004C
:104EE000580020204D61783A2000205A00205900B7
:104EF000580020204D696E3A20004F6E20004F660A
:104F00006600536F667420656E6473746F70733AD5
:104F10002000021FFFFFFFFFFFFF600000000001F5
:104F2000FF400000000000FF8000000000007F83C1
:104F3000CF00000C303F87FF80000C301F86798047
:104F4000000C000F8C30C7838C30E78C30CFC7CC7F
:104F500031F38C30DCECEC33B98C30D86C6C331919
:104F60008C30D06C0C33198C30D86C0C33198C30DD
:104F7000DC6C0E3B198C30CF7C079F198C30C77CC2
:104F8000038F1940000000000002600000000000D4
:104F9000061FFFFFFFFFFFF82020506C616E6E655B
:104FA0007242756666657242797465733A200020B4
:104FB00046726565204D656D6F72793A2000436FCA
:104FC0006D70696C65643A204E6F76203231203204
:104FD0003031370A00207C20417574686F723A20A6
:104FE00028416C657068204F626A6563747320495C
:104FF0006E632E2C204C756C7A426F742047697456
:10500000205265706F7369746F7279290A004E6F50
:1050100076203231203230313731333A32393A3535
:105020003600204C61737420557064617465643A75
:105030002000312E312E350A004D61726C696E00F0
:1050400020536F6674776172652052657365740AC8
:1050500000205761746368646F67205265736574DC
:105060000A002042726F776E206F7574205265734C
:1050700065740A002045787465726E616C20526513
:105080007365740A00506F77657255700A00737407
:105090006172740A006572726F7220777269746946
:1050A0006E6720746F2066696C650A004572726FC6
:1050B000723A00456E6473746F7073202563202507
:1050C0006320256320256300205A3A0020593A00C6
:1050D00020583A00656E6473746F70732068697449
:1050E0003A20006563686F3A00446F6E6520736113
:1050F00076696E672066696C652E0A004D3239004C
:10510000526573746F7265206661696C7361666560
:10511000004D3530320A4D353030004C6F6164201F
:1051200073657474696E67730053746F726520736E
:10513000657474696E677300416476616E6365645B
:105140002053657474696E6773004D61696E005019
:1051500072696E742061626F727465640041626F7F
:105160007574204669726D77617265004E6F2053C9
:10517000442063617264005072696E742066726FBD
:105180006D2053440053746F70207072696E740008
:10519000526573756D65207072696E74005061752B
:1051A0007365207072696E7400436F6E666967750F
:1051B000726174696F6E0054656D706572617475AB
:1051C0007265004D6F76656D656E74004368616E43
:1051D00067652066696C616D656E740054756E65F7
:1051E00000496E666F2073637265656E0020746F90
:1051F0006F206C6F6E6720657874727573696F6E5F
:105200002070726576656E7465640A0020636F6C49
:105210006420657874727573696F6E20707265763C
:10522000656E7465640A00202F002042403A002019
:10523000403A004E6F204C696E65204E756D626578
:1052400072207769746820636865636B73756D2C71
:10525000204C617374204C696E653A200053544FA2
:10526000505045442E20005072696E746572207350
:10527000746F707065642064756520746F2065724A
:10528000726F72732E20466978207468652065728B
:10529000726F7220616E6420757365204D393939E3
:1052A00020746F20726573746172742E20285465A7
:1052B0006D706572617475726520697320726573B3
:1052C00065742E205365742069742061667465725C
:1052D0002072657374617274696E67290A004E6F7B
:1052E00020436865636B73756D2077697468206C03
:1052F000696E65206E756D6265722C204C617374E9
:10530000204C696E653A2000636865636B73756D48
:10531000206D69736D617463682C204C6173742017
:105320004C696E653A20004C696E65204E756D6261
:105330006572206973206E6F74204C617374204C09
:10534000696E65204E756D6265722B312C204C6143
:105350007374204C696E653A20004D313130004D38
:105360003331004D383420582059205A20450053FD
:10537000442072656164206572726F720A00446F26
:105380006E65207072696E74696E672066696C65FF
:105390000A004B494C4C45442E20004B494C4C20B4
:1053A000636175736564206279204B494C4C2062BF
:1053B0007574746F6E2F70696E0A004B494C4C45C2
:1053C000442E20004B494C4C20636175736564206A
:1053D000627920746F6F206D75636820696E6163F8
:1053E000746976652074696D65202D20637572720D
:1053F000656E7420636F6D6D616E643A2000506C51
:1054000065617365207265736574005052494E542E
:1054100045522048414C544544005072696E7465B1
:10542000722068616C7465642E206B696C6C28292D
:105430002063616C6C6564210A006265640A002C5B
:105440002073797374656D2073746F707065642157
:10545000204865617465725F49443A2000544845AC
:10546000524D414C2052554E4157415920424544DE
:1054700000546865726D616C2052756E6177617958
:1054800000544845524D414C2052554E41574159C8
:1054900020453100544845524D414C2052554E4113
:1054A0005741592045300048656174696E67206630
:1054B00061696C6564204245440048656174696EA9
:1054C00067206661696C65640048656174696E6730
:1054D000206661696C65640048656174696E672067
:1054E0006661696C6564204530005A204F666673BA
:1054F000657400466C6F7700466C6F770046616E8E
:105500002073706565640046616E20737065656424
:105510000042656400426564004E6F7A7A6C6500F3
:105520004E6F7A7A6C6500537065656400537065E0
:105530006564004D61696E00416D617820450041F0
:105540006D6178204500416D6178205A00416D61A0
:1055500078205A00416D6178205900416D617820B2
:105560005900416D6178205800416D6178205800E4
:10557000412D74726176656C00412D74726176659F
:105580006C00412D7265747261637400412D726507
:10559000747261637400416363656C0041636365A9
:1055A0006C004D6F74696F6E00436F6F6C646F7742
:1055B0006E0046616E2073706565640046616E2002
:1055C00073706565640042656400426564004E6FF7
:1055D0007A7A6C65004E6F7A7A6C65004D61696EFF
:1055E000004E414E494E495459494E46CDCCCC3DD2
:1055F0000AD7233C17B7D13877CC2B329595E624C0
:105600001FB14F0A000020410000C84200401C4664
:1056100020BCBE4CCA1B0E5AAEC59D74D40095D892
:1056200011241FBECFEFD1E2DEBFCDBF00E00CBF23
:1056300014E0A0E0B2E0EEE9F3E402E00BBF02C048
:1056400007900D92A232B107D9F725E1A2E2B4E0AA
:1056500001C01D92AF34B207E1F716E5CEE1D6E501
:1056600000E006C022970109FE010BBF0F944F21F5
:10567000CC31D10780E00807A9F70E94D4E60D9449
:10568000BE210C9400002F923F924F925F926F9236
:105690007F928F929F92AF92BF92CF92DF92EF92C2
:1056A000FF920F931F93CF93DF93CDB7DEB7C05711
:1056B000D1090FB6F894DEBF0FBECDBF0091B01078
:1056C00020E6029F80011124005D104F8091F704B5
:1056D00080FF1AC0E3EEF0E584917F013FEFE31A0B
:1056E000F30A811102C0780104C00E94E148F70169
:1056F000F3CFD7018D917D01882319F00E94E148F5
:10570000F8CF8AE00E94E1481092B6041092B504E6
:105710008FE38093F6041092F5041092F404109233
:105720003C0410923D0410923E0410923F04F80194
:1057300080810F5F1F4F8032D1F38E34B1F48181AD
:1057400090ED980F9A3020F08D3211F08B3269F481
:105750003296DF0131962C9120532A30D0F3CD01BF
:10576000FC01019620812032D9F3F093EE04E093FE
:10577000ED047F01BFEFEB1AFB0A10816AE270E0D3
:10578000C7010F948F21009739F0DC0111978C919C
:105790008032E1F311961C921D3429F0143519F072
:1057A000173409F0CAC0F7014E2F9F2F8191803224
:1057B000D9F380538A3008F0C0C01093F6042091CA
:1057C000F4043091F504E42FF92F6AE0AF014F5F44
:1057D0005F4F629FC001639F900D1124208130E0D4
:1057E00020533109820F931F218120532A3030F03A
:1057F0009093F5048093F4049A0103C09C01FA018C
:10580000E5CFD9012F5F3F4F4C914032D1F31D348A
:10581000D1F48E31910591F03CF48731910571F00E
:105820008C31910581F40AC08537910564F0873782
:10583000910524F0803AE3E09E0729F4B093B60482
:10584000A093B5047AC01092B6041092B504D0901B
:10585000ED0441E050E0FD0131962C91222309F442
:105860006CC02132A1F41D3491F48032910579F499
:10587000F093B604E093B50463E270E0CF010F94B7
:105880008F21009709F459C0DC011C9256C00FEB20
:10589000020F0A31A0F59F01F90160812F5F3F4F90
:1058A0006032D1F320ED260F2A3040F023ED260F91
:1058B000223020F06B3211F00C94DA419F01602FFE
:1058C00070E0DB01B595A795B595A795B595A7951A
:1058D000A45CBB4F07707A01002E01C0EE0C0A9445
:1058E000EAF7FC90FE28FC922115310511F02D19E4
:1058F00001C020E0DB01AE5DBB4F2C930AC02091BC
:10590000B5043091B604232B21F4B093B604A093D0
:10591000B504208121542A3110F4DF019CCFDF012E
:1059200031966C9160536A30D0F39D01F9012F5F7D
:105930003F4F60816032D1F3F0CF8091F6048D3417
:1059400011F40C943135843511F40C94864187346C
:1059500011F00C94C0418091F4049091F5048A31C7
:10596000910509F43DC7A4F48430910544F48230D4
:1059700091050CF01EC197FF2AC00C94D7418430CA
:10598000910509F4A6C60C9709F4E8C60C94D74112
:105990008E31910509F4BFC73CF48C31910509F4AF
:1059A000A8C70CF424C7AAC78B35910511F40C9431
:1059B00028358C35910511F40C942D358A359105D7
:1059C00011F00C94D7411092F3040C94D7418091BC
:1059D0005302882311F40C94D7410E946F8880E40D
:1059E00094E00E94744A0E94EA4E8091F70483FD7D
:1059F0008FC0C0904C04D0904D04E0904E04F090C5
:105A00004F0420910A0F30910B0F40910C0F5091D1
:105A10000D0FC701B6010F94F019882309F478C05F
:105A20008091D604811138C0609151027091520268
:105A3000882777FD8095982F0F94F6199B01AC016C
:105A40006091690470916A0480916B0490916C0478
:105A50000F94F01987FF20C0C0920A0FD0920B0F4D
:105A6000E0920C0FF0920D0FE3EEF0E584918F01C0
:105A70000F5F1F4F882321F00E94E148F801F6CF05
:105A8000E1E0F2E084918F010F5F1F4F882321F046
:105A90000E94E148F801F6CFC0904C04D0904D042C
:105AA000E0904E04F0904F0420910A0F30910B0FBC
:105AB00040910C0F50910D0FC701B6010F94531E6A
:105AC00020E030E048E453E40F947A20181604F5FF
:105AD000C0920A0FD0920B0FE0920C0FF0920D0FB4
:105AE000E3EEF0E584918F010F5F1F4F882321F0D3
:105AF0000E94E148F801F6CFE2EEF1E084918F01D7
:105B00000F5F1F4F882321F00E94E148F801F6CF74
:105B1000209140043091410440914204509143044B
:105B20006091FE0E7091FF0E8091000F9091010F19
:105B30000F94F01981111DC0209144043091450447
:105B400040914604509147046091020F7091030FF9
:105B50008091040F9091050F0F94F019811109C0E5
:105B600060910A0270910B0280910C0290910D02DB
:105B70001AC06091A6027091A702882777FD8095D0
:105B8000982F0F94F61920910A0230910B02409140
:105B90000C0250910D020F94551A2AE037ED43E2A2
:105BA0005CE30F94551A0F9422020E94D34A0C947E
:105BB000D74120915302222311F40C94D74111E0D4
:105BC000029709F010E00E946F8882E50E94504C15
:105BD000882309F44AC10E94F2496B017C0140907C
:105BE000FE0E5090FF0E6090000F7090010F2091FC
:105BF000020F3091030F4091040F5091050F2EAB0F
:105C00003FAB48AF59AF8091400490914104A091BF
:105C10004204B09143048AAF9BAFACAFBDAF2091BB
:105C2000440430914504409146045091470426961F
:105C30002CAF3DAF4EAF5FAF269720E030E0A9011B
:105C4000C701B6010F94F019882309F428C5A301F0
:105C500092016AAD7BAD8CAD9DAD0F94F0198111B1
:105C60000FC02EA93FA948AD59AD26966CAD7DADAC
:105C70008EAD9FAD26970F94F019882309F40FC5B8
:105C800020E030E0A901C701B6010F94F019881F88
:105C90008827881F181759F080E090E0A0E8BFEB34
:105CA00062968CAF9DAFAEAFBFAF62970AC020E0E7
:105CB00030E040E85FE362962CAF3DAF4EAF5FAFA0
:105CC0006297A30192016AAD7BAD8CAD9DAD0F943F
:105CD000531E2A966CAF7DAF8EAF9FAF2A972EA929
:105CE0003FA948AD59AD26966CAD7DAD8EAD9FAD4B
:105CF00026970F94531E2E966CAF7DAF8EAF9FAF3D
:105D00002E972A962CAD3DAD4EAD5FAD2A97CA01B8
:105D1000B9010F94551A4B015C012E962CAD3DAD87
:105D20004EAD5FAD2E97CA01B9010F94551A9B0174
:105D3000AC01C501B4010F94541E0F94BF202296EC
:105D40006CAF7DAF8EAF9FAF229720E030E040E098
:105D50005FE30F94551A4B015C01A7019601C7013F
:105D6000B6010F94551A6B017C01A5019401C50180
:105D7000B4010F94551A9B01AC01C701B6010F94F1
:105D8000531E0F94BF209B01AC0162966CAD7DAD9C
:105D90008EAD9FAD62970F94551A4B015C012AADF1
:105DA0003BAD4CAD5DADC301B2010F94541E20E07C
:105DB00030E040E05FE30F94551A6B017C012E96B2
:105DC0006CAD7DAD8EAD9FAD2E97905822962CADCB
:105DD0003DAD4EAD5FAD22970F94301F9B01AC01DE
:105DE000C501B4010F94551A9B01AC01C701B6015E
:105DF0000F94541EA30192010F94531E6B017C015A
:105E000026962CAD3DAD4EAD5FAD26976EA97FA910
:105E100088AD99AD0F94541E20E030E040E05FE380
:105E20000F94551A2B013C0122962CAD3DAD4EAD81
:105E30005FAD22972A966CAD7DAD8EAD9FAD2A9752
:105E40000F94301F9B01AC01C501B4010F94551A8A
:105E50009B01AC01C301B2010F94541E2EA93FA9AE
:105E600048AD59AD0F94531E14C089E40E94504CA4
:105E7000882329F00E94F2496B017C0103C0C12CE8
:105E8000D12C76018AE40E94504C8823F9F00E94BC
:105E9000F24926966CAF7DAF8EAF9FAF269720E07C
:105EA00030E0A901C701B6010F94F01981111EC09D
:105EB00020E030E0A90126966CAD7DAD8EAD9FADA2
:105EC00026970F94F019811111C0E9C320E030E04A
:105ED000A901C701B6010F94F019882309F4DFC3A3
:105EE00026961CAE1DAE1EAE1FAE2697D701C6016C
:105EF000B0588EAB9FABA8AFB9AF26962CAD3DADD9
:105F00004EAD5FAD269750582AAF3BAF4CAF5DAF5B
:105F10009C01AD01BC01CD010F94551A4B015C01F0
:105F20002AAD3BAD4CAD5DADCA01B9010F94551A18
:105F30009B01AC01C501B4010F94541E0F94BF2006
:105F4000A2966CAF7DAF8EAF9FAFA2978091FE0EF1
:105F50009091FF0EA091000FB091010F2A968CAF87
:105F60009DAFAEAFBFAF2A97A7019601BC01CD018F
:105F70000F94541E62966CAF7DAF8EAF9FAF629749
:105F80002091020F3091030F4091040F5091050FA3
:105F90002E962CAF3DAF4EAF5FAF2E9726962CAD11
:105FA0003DAD4EAD5FAD26972E966CAD7DAD8EAD01
:105FB0009FAD2E970F94541E66966CAF7DAF8EAF3B
:105FC0009FAF66978091400490914104A091420454
:105FD000B09143046A968CAF9DAFAEAFBFAF6A97E6
:105FE00062962CAD3DAD4EAD5FAD6297BC01CD016B
:105FF0000F94531E6B017C012091440430914504A1
:1060000040914604509147046E962CAF3DAF4EAF81
:106010005FAF6E9766962CAD3DAD4EAD5FAD6697AA
:106020006E966CAD7DAD8EAD9FAD6E970F94531E89
:106030004B015C018091060F9091070FA091080F12
:10604000B091090FAA968CAF9DAFAEAFBFAFAA9724
:106050009C01AD01609148047091490480914A040B
:1060600090914B040F94531E22966CAF7DAF8EAF70
:106070009FAF229720910A0F30910B0F40910C0F88
:1060800050910D0FAE962CAF3DAF4EAF5FAFAE97B8
:1060900060914C0470914D0480914E0490914F0496
:1060A0000F94531EA6966CAF7DAF8EAF9FAFA69791
:1060B000A70196016EA97FA988AD99AD0F94551AD5
:1060C0002B013C01A50194016AAD7BAD8CAD9DAD6A
:1060D0000F94551A9B01AC01C301B2010F94541ED9
:1060E0002B013C01A50194016EA97FA988AD99AD52
:1060F0000F94551A4B015C01A70196016AAD7BAD67
:106100008CAD9DAD0F94551A9B01AC01C501B40136
:106110000F94531EA30192010F94C71E6B017C01C3
:1061200020E030E0A9010F94F01987FF0AC02BEDA1
:106130003FE049EC50E4C701B6010F94541E6B01D7
:106140007C01112351F02BED3FE049EC50E4C701F5
:10615000B6010F94531E6B017C0120E030E0A901D1
:10616000C701B6010F94F019811128C06A962CADB1
:106170003DAD4EAD5FAD6A972A966CAD7DAD8EADEF
:106180009FAD2A970F94F019811118C06E962CAD0F
:106190003DAD4EAD5FAD6E972E966CAD7DAD8EADC7
:1061A0009FAD2E970F94F019811108C06BEDC62E8C
:1061B0006FE0D62E69ECE62E60E4F62EA2962CADAA
:1061C0003DAD4EAD5FADA297C701B6010F94551A14
:1061D0009B01AC010F94551A4B015C0122962CAD2A
:1061E0003DAD4EAD5FAD2297CA01B9010F94551A6E
:1061F0009B01AC01C501B4010F94541E0F94BF2044
:106200004B015C012FE632E143E85AE30F94F019A9
:1062100087FD41C2C501B4010F94C91F0F949D1F92
:106220001B016115710519F422242394312CB1014D
:1062300080E090E00F94F4194B015C019B01AC01EC
:10624000C701B6010F94301F2A966CAF7DAF8EAF99
:106250009FAF2A97A501940122966CAD7DAD8EADBE
:106260009FAD22970F94301FA2966CAF7DAF8EAF7B
:106270009FAFA297A5019401A6966CAD7DAD8EADA2
:106280009FADA6970F94301FA6966CAF7DAF8EAFD3
:106290009FAFA6972A962CAD3DAD4EAD5FAD2A9728
:1062A000CA01B9010F94551A20E030E040E05FE3E5
:1062B0000F94551A9B01AC0160E070E080E89FE309
:1062C0000F94531E6A966CAF7DAF8EAF9FAF6A97E7
:1062D000AA968CAD9DADAEADBFADAA9789879A87C2
:1062E000AB87BC87AE962CAD3DAD4EAD5FADAE97E6
:1062F0002D873E874F87588B6091A6027091A70229
:10630000882777FD8095982F0F94F61920910A021F
:1063100030910B0240910C0250910D020F94551ACE
:106320002AE037ED43E25CE30F94551A6E966CAFAA
:106330007DAF8EAF9FAF6E970E94FB4DDC01CB010E
:1063400088539F4FAF4FBF4F22968CAF9DAFAEAFDC
:10635000BFAF22974EA85FA868AC79ACA1E0B0E0CF
:106360002C96BFAFAEAF2C9749E1B42E2C962EAD34
:106370003FAD2C972215330508F049C10F941D0C31
:106380000E94FB4D22962CAD3DAD4EAD5FAD2297E8
:10639000621B730B840B950B97FD11C00E94FB4D84
:1063A000DC01CB0188539F4FAF4FBF4F22968CAF7C
:1063B0009DAFAEAFBFAF229780E00F94F805BA94BF
:1063C00009F449C06A962CAD3DAD4EAD5FAD6A97FC
:1063D0006AAD7BAD8CAD9DAD0F94551A6B017C0100
:1063E0002A962CAD3DAD4EAD5FAD2A97B201C301EB
:1063F0000F94551AA70196010F94541E162FA72E1D
:10640000982E892E6A962CAD3DAD4EAD5FAD6A9744
:10641000B201C3010F94551A6B017C012A962CAD71
:106420003DAD4EAD5FAD2A976AAD7BAD8CAD9DADF8
:106430000F94551A9B01AC01C701B6010F94531E6E
:106440002B013C01812F9A2DA92DB82D8AAF9BAF2E
:10645000ACAFBDAF59C02C96AEADBFAD2C97BD0152
:1064600080E090E00F94F4192A962CAD3DAD4EAD2E
:106470005FAD2A970F94551A4B015C010F942D1FA5
:106480006B017C01C501B4010F94B5204B015C0187
:10649000A70196016EA97FA988AD99AD0F94551AF1
:1064A0002B013C01A501940126966CAD7DAD8EAD0E
:1064B0009FAD26970F94551A9B01AC01C301B20101
:1064C0000F94541E2B013C01A50194016EA97FA9D4
:1064D00088AD99AD0F94551A4B015C01A701960147
:1064E00026966CAD7DAD8EAD9FAD26970F94551A57
:1064F0009B01AC01C501B4010F94531E6AAF7BAF81
:106500008CAF9DAF39E1B32E9201A30162966CADC1
:106510007DAD8EAD9FAD62970F94541E69837A83D3
:106520008B839C832AAD3BAD4CAD5DAD66966CAD67
:106530007DAD8EAD9FAD66970F94541E6D837E83A7
:106540008F839887A2962CAD3DAD4EAD5FADA297DF
:1065500069857A858B859C850F94541E69877A8717
:106560008B879C87A6962CAD3DAD4EAD5FADA697B3
:106570006D857E858F8598890F94541E6D877E87E3
:106580008F87988BCE0101960E94744AC090EC04CC
:1065900089819A81AB81BC818E8B9F8BA88FB98FAB
:1065A0008D819E81AF81B8858A8F9B8FAC8FBD8F87
:1065B00089859A85AB85BC858E8F9F8FA8A3B9A34B
:1065C000AE01425E5F4FBE01665E7F4FCE014696D2
:1065D0000E9412546E96ECACFDAC0EAD1FAD6E97E2
:1065E0009E01235F3F4FAE01425E5F4FBE01665E7C
:1065F0007F4FCE0146960E946BF42C96EEADFFAD18
:106600002C9731962C96FFAFEEAF2C97AFCEC09063
:10661000EC048091400490914104A0914204B09117
:1066200043048E8B9F8BA88FB98F809144049091E7
:106630004504A0914604B09147048A8F9B8FAC8F8C
:10664000BD8F8091480490914904A0914A04B09173
:106650004B048E8F9F8FA8A3B9A3AE01425E5F4FFC
:10666000BE01665E7F4FCE0146960E9412546E9622
:10667000ECACFDAC0EAD1FAD6E972CE434E0AE017A
:10668000425E5F4FBE01665E7F4FCE0146960E941E
:106690006BF40E94D34A0E94EA4E0C94D741ECEA74
:1066A000F0E584918F010F5F1F4F882321F00E9436
:1066B000E148F801F6CFECE1F2E084918F010F5F41
:1066C0001F4F882311F40C94D7410E94E148F80130
:1066D000F4CF80E50E94504C882329F00E94B249F3
:1066E0004B015C0103C0812C912C540183E50E9475
:1066F000504C882361F00E94F24920E030E04AE7E4
:1067000054E40F94551A0F949D1F4B015C010E9495
:10671000466480910E02811105C060E082E392E040
:106720000E9462550E94EA4EC0905C04D0905D04C5
:10673000E0905E04F0905F04C80CD91CEA1CFB1CBE
:106740000E94FB4D6C197D098E099F0997FD02C0BF
:106750000C94D74180E00F94F805F2CF0E949A87FD
:1067600081110C94D74180E50E94504C882319F088
:106770000E94C24901C060E06EA383E50E94504CB4
:10678000882319F00E94C24901C06CE06AA384E525
:106790000E94504C882319F00E94C24901C063E056
:1067A0006E8B82E50E94504C882319F00E94F249BA
:1067B00004C060E070E080ED90E469837A838B83AD
:1067C0009C839E012A5E3F4FAE014F5F5F4FBE012B
:1067D0006E5D7F4FCE0186960E9440EE0C94D741AD
:1067E00081E0809353021092EB040C94D7410E94F5
:1067F0009A8781110C94D74180E50E94504C8823E0
:1068000021F00E94C249462F01C040E06091060F6E
:106810007091070F8091080F9091090F00E010E030
:1068200020E231E409831A832B833C8300E010E0EB
:1068300025E333E40D831E832F83388700E010E0C7
:1068400020EA31E409871A872B873C8700E010E0B3
:1068500020EC3FE70D871E872F87388B413071F181
:10686000423021F51E8A1F8A188E198E20E030E0F2
:1068700040EA51E40F94541E7B018C0120E030E08B
:1068800047E353E40F947A20181624F4E12CF12CFA
:1068900007E313E4A701B8014AA35BA36CA37DA39C
:1068A000BE016A5E7F4FCE01829611C020E030E0CB
:1068B00040EA51E40F94F01987FF0BC01E8A1F8A2B
:1068C000188E198EBE016A5E7F4FCE0109960E9416
:1068D00039EE1E8A1F8A188E198EAE014A5E5F4FEE
:1068E000BE016B5F7F4FCE0101960E9435EE0C9486
:1068F000D74180E00E9434970C94D74181E0809387
:10690000F10E24982C9A0E94A4AF1092F10E249AB2
:106910002C980C94D74120E030E0A9016091FE0E44
:106920007091FF0E8091000F9091010F0F94541EF3
:10693000182F88E5AF966FAFAF97E0967FAFE097DF
:10694000E1969FAFE1970E94504CAF966FADAF9725
:10695000E0967FADE097E1969FADE197882321F027
:106960000E94F2499B0102C09B01812FA901BC0139
:106970004E8B5F8B688F798F20E030E0A9016091AA
:10698000020F7091030F8091040F9091050F0F94E7
:10699000541E5B018C0189E50E94504C882321F034
:1069A0000E94F2495B018C01A501B80149835A8319
:1069B0006B837C834090540450905504609056043F
:1069C000709057042091500430915104409152042A
:1069D000509153046E897F89888D998D0F94531E31
:1069E0006B017C012FE632E143E85AEB0F947A20E9
:1069F00087FF02C00C94D74122E430E045E253E423
:106A0000C701B6010F94F019181614F40C94D7416D
:106A1000A3019201B501C8010F94531E6B017C01C3
:106A200021E338E040EC50EC0F947A2087FF02C05D
:106A30000C94D74122E430E04FE353E4C701B601A0
:106A40000F94F019181614F40C94D7410C94EB41E0
:106A500081E08093F3040C94D7410E9427F10C94B9
:106A6000D7418091F4049091F5048837910511F491
:106A70000C94583D0CF0CDC08D34910509F48CC3B5
:106A80000CF056C08931910509F48CC21CF5843193
:106A9000910509F444C27CF48131910509F434C2B2
:106AA0002CF4029708F4ADC10C94D741429709F435
:106AB0008BC60C94D7418631910509F438C20CF489
:106AC00032C28731910509F438C2489709F44BC2A4
:106AD0000C94D7418F31910509F4D9C294F48B31CC
:106AE000910509F47BC20CF46BC28C31910509F459
:106AF00079C24E9711F00C94D7410E9478C50C943E
:106B0000D7418A32910509F4EEC22CF4809709F43A
:106B100073C20C94D7418B34910509F439C38C347A
:106B2000910511F00C94D7410E940D890C94D74126
:106B30008A36910509F492C59CF58435910509F4CE
:106B400043C6CCF48135910509F425C634F48E345E
:106B5000910509F425C30C94D7418235910509F4B8
:106B600030C68335910511F00C94D74181E08093B4
:106B7000F2040C94D7418C35910509F441C634F4E4
:106B80008535910509F423C60C94D74188369105C3
:106B900009F418C48936910509F4F5C40C94D74159
:106BA0008237910509F4B1C6ACF48D36910509F42C
:106BB0002BC534F48B36910509F46DC50C94D7417F
:106BC0008E36910509F44BC48F36910509F458C4EB
:106BD0000C94D7418537910509F49CC64CF4833752
:106BE000910511F00C94D7410E941E490C94D74195
:106BF0008637910509F496C68737910511F00C94F4
:106C0000D74181E08093F10E24982C9AE7E3F4E0D9
:106C10008CC68F3231E0930711F40C94883F0CF04E
:106C200074C08C3C910511F40C943B3EBCF58B393F
:106C3000910509F4C2C4D4F48D37910509F43BC51C
:106C40005CF48937910511F00C94D7411092ED0E48
:106C50001092B7040C94D7418C38910509F479C48B
:106C60008139910509F42AC70C94D741883C9105D4
:106C700009F499C734F48E3B910509F4DBC40C94F4
:106C8000D741893C910509F4D6C78B3C910511F099
:106C90000C94D7410E94334C0C94D7418D3D910503
:106CA00011F40C94863EA4F48E3C910509F4E9C7D6
:106CB0000CF4E4C7833D910511F40C94833E8C3DA4
:106CC000910511F00C94D7410E945C4C0C94D74173
:106CD0008C3251E0950711F40C94893E4CF4823EBD
:106CE000910511F00C94D7410E9422F40C94D741E5
:106CF0008D32B1E09B0711F40C94B23E8E3291407C
:106D000011F40C94323F0C94D741843FF1E09F077B
:106D100011F40C94993FE4F5803931E0930711F4B4
:106D20000C948B3FECF48E3551E0950711F40C94E4
:106D3000EE403CF48033914011F40C94B53E0C9439
:106D4000D7418F35E1E09E0711F40C941F41833643
:106D5000914011F00C94D741ECEAF0E50C945F41BE
:106D6000823921E0920711F40C94923F14F40C94B0
:106D70008E3F843A41E0940711F40C94963F8C3A8C
:106D8000914011F00C94D7410E94676C0C94D7414C
:106D90008835A2E09A0711F40C94BB3FB4F4863F07
:106DA000E1E09E0711F40C949F3F14F40C949C3F77
:106DB000873F21E0920711F40C94A23F8C3192405E
:106DC00011F40C94B03F0C94D7418B3843E09407F6
:106DD00011F40C94B5404CF48335934011F00C94AD
:106DE000D7410E94797B0C94D741803AB3E09B074E
:106DF00009F440C1873E934011F40C9474410C9403
:106E0000D7410091B5041091B60480E50E94504C22
:106E1000882369F00E94B2496B017C01BB24B394C2
:106E2000611571058105910531F4B12C04C0B12CB7
:106E3000C12CD12C760183E50E94504C8823F9F0B7
:106E40000E94F24920E030E04AE754E40F94551ADA
:106E50000F949D1F6B017C01B11013C0611571056A
:106E60008105910571F40115110559F0D8018C9136
:106E7000882339F061E0C8010E94525507C0BB2049
:106E800091F360E086E792E00E94625581E0809392
:106E90000C090E9446640E94EA4EC114D104E10428
:106EA000F104D1F080905C0490905D04A0905E04A9
:106EB000B0905F048C0C9D1CAE1CBF1C0E94FB4D4F
:106EC000681979098A099B0997FF1AC080910C09F2
:106ED00081110C943F4214C080910C09882321F049
:106EE00080E00F94F805F8CF8091981260E0882335
:106EF00019F087E692E002C08DE492E00E946255AC
:106F000010920C090C94D74160E089E892E00E944D
:106F1000625517981698159814980C94D7410E94AA
:106F20002DC30C94D7410E948A600C94D7411092D3
:106F30009812109299120C94D741E091B504F091F7
:106F4000B6048081882329F0803209F410823196BA
:106F5000F8CF40E061E08091B5049091B6040E94C2
:106F600028760C94D74119821A821B821C821E8AB1
:106F70001F8A188E198E8091DE04882341F040E02C
:106F8000BE016F5F7F4FCE0146960E9426DD809145
:106F90009912882319F081E0809398120E9416E6D6
:106FA0000C94D741109298120E940D8982E992E0C8
:106FB00090939109809390090E94AE720C94D741EE
:106FC00080919912882311F40C94D74183E50E9493
:106FD000504C81110C9444420C94D7410E9461E4BE
:106FE0000C94D74140E060E08091B5049091B604E4
:106FF0000E9428760C94D7418091981281110E94AA
:1070000046640091B5041091B60480E50E94784B67
:10701000882321F00E94E349F82E01C0F12C8091D1
:107020009912882311F40C94D7414F2D61E0C801C7
:107030000E94287683E50E94504C882381F00E94AC
:10704000C249AB01BC0140933B1550933C15609382
:107050003D1570933E158AE894E10E944985809120
:107060009912882319F081E080939812F1100C9402
:10707000D74194CF8091B5049091B60421E020933C
:10708000971240E060E00E9428760C94D7418EE68B
:1070900092E10E9403506E8B7F8B888F998FBE0187
:1070A0006F5F7F4FCE0146960E94947860E0CE01DC
:1070B00001960E945255E3EEF0E584918F010F5F37
:1070C0001F4F882321F00E94E148F801F6CFBE014E
:1070D0006F5F7F4F87E992E00E940E8C8AE00E94EA
:1070E000E1480C94D74183E50E94504C882311F469
:1070F0000C94D7410E94D249E82E80E50E94504C62
:10710000811110C081E0E11001C080E08093F10E98
:10711000882321F024982C9A0C94D741249A2C98F7
:107120000C94D74180E50E94504C882341F00E9486
:10713000C24977FF02C00C94D7418B0102C00DE019
:1071400010E0802FE4EAF2E09491891739F031964B
:10715000B2E0EC3CFB07C1F70C945442ECEAF0E5DA
:1071600084918F010F5F1F4F882321F00E94E14817
:10717000F801F6CFECECF2E084918F010F5F1F4F26
:10718000882311F40C94D7410E94E148F801F4CF10
:107190000E9416E60C94D7410F9453090C94D741E2
:1071A00083E50E94504C882359F00E94C2496E34F6
:1071B000710531F48EE692E10E94DCE50C94D74132
:1071C0001E8A1F8A188E198EEBE3F3E084918F01DB
:1071D0000F5F1F4F882321F00E94E148F801F6CF8E
:1071E000E2E3F3E084918F010F5F1F4F882321F0CA
:1071F0000E94E148F801F6CF60917B1270917C12F9
:1072000080E090E04AE00E949FA6E5E2F3E08491EE
:107210008F010F5F1F4F882321F00E94E148F80182
:10722000F6CF60917D1270917E1280E090E04AE08E
:107230000E949FA6EAE1F3E084918F010F5F1F4F48
:10724000882321F00E94E148F801F6CF80917B125B
:1072500090917C1220917D1230917E12821B930BB3
:1072600040916E12415021E030E0423010F020E0B9
:1072700030E0BC01621B730B80E090E04AE00E94AA
:107280009FA68AE00E94E148E2E1F3E084918F0149
:107290000F5F1F4F882321F00E94E148F801F6CFCD
:1072A00080917F1290918012A0918112B0918212F0
:1072B0008E8B9F8BA88FB98FBE016F5F7F4FCE01E2
:1072C00046960E949478E5E0F3E084918F010F5F89
:1072D0001F4F811104C08E010F5F1F4F04C00E9419
:1072E000E148F801F2CFF80181918F01882319F06C
:1072F0000E94E148F8CF8091831290918412A0916E
:107300008512B09186128E8B9F8BA88FB98FBE018C
:107310006F5F7F4FCE0146960E949478E5EFF2E0D2
:1073200084918F010F5F1F4F811104C08E010F5F89
:107330001F4F04C00E94E148F801F2CFD8018D919F
:107340008D01882319F00E94E148F8CF8AE00E945D
:10735000E148EDEEF2E084918F010F5F1F4F88232B
:1073600021F00E94E148F801F6CFEDEDF2E08491C2
:107370008F010F5F1F4F882321F00E94E148F80121
:10738000F6CF20E030E04AE754E460918712709134
:1073900088128091891290918A120F94301F42E0D6
:1073A0000E949EE4EBEDF2E084918F010F5F1F4F8E
:1073B000882321F00E94E148F801F6CF8AE00E947C
:1073C000E148F5C788E690E00E94BCDF8111EFC775
:1073D0008091F70483FF01C0EAC783E50E94504C07
:1073E000882309F4E4C70E94F2490F94981F709310
:1073F000AC0E6093AB0E80E00E94C7570E94F2492A
:1074000020E030E040E752E40F94F01918163CF009
:107410000F94530960E08FE493E00E9462550E944C
:10742000F2492091690430916A0440916B045091B3
:107430006C040F947A2018160CF0B9C785EE92E010
:107440009F938F9383E493E09F938F931F920E9467
:107450007F870F900F900F900F900F90A8C78EE42A
:107460000E94504C882309F4A2C70E94C24960932D
:10747000600470936104809362049093630497C7DF
:1074800083E50E94504C882321F00E94D249C82EE7
:1074900001C0C12CC092F704E3EEF0E584918F01A6
:1074A0000F5F1F4F882321F00E94E148F801F6CFBB
:1074B000E7E7F3E084918F010F5F1F4F882321F0EE
:1074C0000E94E148F801F6CFCC2099F129E6E22E9E
:1074D00023E0F22E00E010E020E0D12CC601002EC7
:1074E00002C0959587950A94E2F780FF17C099240A
:1074F0009394920E222319F08CE20E94E148F70146
:1075000025913491F90184915901FFEFAF1ABF0A17
:10751000882329F00E94E1489501F4CF922E0F5F55
:107520001F4F22E0E20EF11C0530110571F0292DEC
:10753000D5CFE3E7F3E084918F010F5F1F4F8823DE
:1075400021F00E94E148F801F6CF8AE00E94E1486C
:107550002EC78091F70483FD2AC783E50E94504C13
:10756000882309F424C70E94F2490F94981F6739B1
:10757000710514F066E970E07093A80E6093A70E91
:107580000E947C5714C789E690E00E94BCDF8111FD
:107590000C947145EEE7F3E084918F010F5F1F4F6C
:1075A000882321F00E94E148F801F6CF0F946C0582
:1075B0008AE00E94E1480C94714583E50E94504C9A
:1075C000882309F4F4C60E94D249809368048D335D
:1075D00018F08CE3809368040E94FB4D6B017C01E2
:1075E0002091680430E0A8EEB3E00F94441EC60E6C
:1075F000D71EE81EF91EC0926404D0926504E09282
:107600006604F0926704D3C68DE690E00E94BCDF6A
:107610008111CDC68091F70483FDC9C683E50E9420
:10762000504C8EAB811155C782E50E94504C8111A0
:1076300050C7BDC68091F70483FDB9C683E50E949B
:10764000504C23968FAF239781110C94FD4382E514
:107650000E94504C81110C94FD43A9C683E50E9401
:10766000504C882339F00E94C2498B016F3F71054D
:1076700019F010F00FEF10E080E50E94504C8111DE
:1076800005C0109391110093901191C60E94D249A8
:1076900081118DC6F6CF80E50E94504C811105C046
:1076A000109291111092901182C60E94C249672BCC
:1076B00009F07DC6F5CF8CE40E94784B882319F041
:1076C0000E94F24904C060E070E080E090EC6AA79C
:1076D0007BA78CA79DA78AE50E94504C882319F0B0
:1076E0000E94F24903C060E070E0CB0120E030E08E
:1076F00040E251E40F94541E6EA37FA388A799A77C
:1077000088E50E94504C882319F00E94F24903C07A
:1077100060E070E0CB0120E030E040E251E40F9403
:10772000541E6AA37BA38CA39DA389E50E94504CA1
:10773000882319F00E94F24903C060E070E0CB0199
:1077400020E030E04FE353E40F94541E20E030E09B
:1077500040E251E40F94531E6E8B7F8B888F998F7C
:1077600019821A821B821C828091DE0481111FC63D
:10777000C12CE12C8E010F5F1F4F9E012A5E3F4FEF
:10778000AE014E5D5F4FBE016A5D7F4FCE018A96AE
:107790000E9450DE0CC60F94DA090E9446640E94D3
:1077A000254A109291111092901168EE73E080E0DA
:1077B00090E00F94570E60E08FEE93E00E946255C8
:1077C000F6C51092F204F3C50E94D1F3F0C583E52B
:1077D0000E94784B882309F4EAC50E94F24920E010
:1077E00030E04AE754E40F94551A0F949D1F6093BC
:1077F0007104709372048093730490937404D7C5DA
:107800001FE1A12E13E0B12E05EA14E0912CD50161
:107810008D915D010E94784B882309F46DC0B3E01F
:107820009B1263C00E94F2496B017C0120E030E0B2
:1078300040EA51E40F94F01987FF4EC0A70196016A
:107840006091B1047091B2048091B3049091B4043A
:107850000F94301F2B013C019B01AC016091A104EE
:107860007091A2048091A3049091A4040F94551ADE
:107870006093A1047093A2048093A3049093A40442
:10788000A3019201609191047091920480919304FC
:10789000909194040F94551A6093910470939204FC
:1078A0008093930490939404609181047091820476
:1078B00080918304909184040F94F419A3019201A0
:1078C0000F94551A0F949D1F609381047093820446
:1078D0008093830490938404C092B104D092B20444
:1078E000E092B304F092B40407C00E94F249F80198
:1078F000608371838283938393940C5F1F4FF4E0C2
:107900009F1285CF0E94266552C50E9446640E9440
:10791000E87B4DC560E08091B5049091B6040E946B
:10792000525545C50E94A64B42C584918F010F5FF9
:107930001F4F882321F00E94E148F801F6CFEFE2C3
:10794000F4E084918F010F5F1F4F882321F00E9484
:10795000E148F801F6CF1E9B03C000E013E002C02F
:107960000BEF12E0D8018D918D01882319F00E9450
:10797000E148F8CF8AE00E94E148E7E2F4E0849130
:107980008F010F5F1F4F882321F00E94E148F8010B
:10799000F6CF379B03C000E013E002C00BEF12E00C
:1079A000F80181918F01882319F00E94E148F8CFF6
:1079B0008AE00E94E148EFE1F4E084918F010F5FDB
:1079C0001F4F882321F00E94E148F801F6CF1D9B4C
:1079D00003C000E013E002C00BEF12E0D8018D916C
:1079E0008D01882319F00E94E148F8CF8AE00E94B7
:1079F000E148E7E1F4E084918F010F5F1F4F882396
:107A000021F00E94E148F801F6CF029B03C000E09C
:107A100013E002C00BEF12E0F80181918F0188237F
:107A200019F00E94E148F8CF8AE00E94E148EFE0B7
:107A3000F4E084918F010F5F1F4F882321F00E9493
:107A4000E148F801F6CF1C9903C000E013E002C042
:107A50000BEF12E0D8018D918D01882319F00E945F
:107A6000E148F8CF8AE00E94E148E7E0F4E0849141
:107A70008F010F5F1F4F882321F00E94E148F8011A
:107A8000F6CF019B03C000E013E002C00BEF12E051
:107A9000F80181918F01882319F00E94E148F8CF05
:107AA0008AE00E94E1481092F10E249A2C987FC43B
:107AB00081E08093ED0E8093B70479C483E50E9442
:107AC000504C882319F00E94C24902C060E070E067
:107AD0008B01112702301105C8F0ECEAF0E5849122
:107AE0008F010F5F1F4F882321F00E94E148F801AA
:107AF000F6CFE1E5F4E084918F010F5F1F4F8823FB
:107B000009F455C40E94E148F801F5CF88E40E94C9
:107B1000504C8823A9F00E94C249683771053CF097
:107B20006332F1E07F072CF062E271E002C068E7A7
:107B300070E0F801EE0FFF1FE054FB4F718360838C
:107B400086E40E94504C882399F00E94C2496F3FFE
:107B5000710519F014F06FEF70E0F801EE0FFF1FE0
:107B6000E454FB4F77FF02C060E070E071836083F4
:107B700082E40E94504C882309F419C40E94C2492F
:107B80006530710534F0683871052CF067E870E0F5
:107B900002C065E070E0F801EE0FFF1FE854FB4FF4
:107BA0007183608304C488EC90E00E94BCDF811183
:107BB000FEC384E40E94784B8823D1F10E94F249ED
:107BC00011E020E030E0A9010F94F019811101C00B
:107BD00010E01093C904112359F10091C80410E07A
:107BE0000E94F249F801EE0FFF1FEE0FFF1FEC534A
:107BF000FB4F608371838283938320E030E0A9018F
:107C00006091C4047091C5048091C6049091C7042A
:107C10000F94F01981110CC080E090E0A0E4B0E472
:107C20008093C4049093C504A093C604B093C70482
:107C30000E942F4ABCC30FE113E037E9E32E31E184
:107C4000F32ED8018D918D010E94784B882349F045
:107C50000E94F2490F949D1FF70160837183828314
:107C60009383F4E0EF0EF11C23E00332120749F78F
:107C70000E946B489CC30E946D8199C30E94D74BA0
:107C800096C39FE1892E93E0992E2EEFA22E2EE02F
:107C9000B22E02EF1EE0712CD4018D914D010E9495
:107CA000784B882311F10E94F2496B017C01F801A5
:107CB00020813181428153810F94531E9B01AC017D
:107CC000D5016D917D918D919C910F94541EF5017C
:107CD0006083718382839383D801CD92DD92ED928C
:107CE000FC921397872D0E94DD4A7394B4E0AB0E8B
:107CF000B11C0C5F1F4FE3E07E12CECF0E94166CCA
:107D00000E94E87B54C30E944CE551C30E94FCDFF3
:107D10004EC383E50E94504C882319F00E94C2494B
:107D200002C064E071E07F8B6E8B80E50E94504C56
:107D3000882339F00E94C2496938F3E17F0730F4A3
:107D400002C068EE73E07A83698304C088E893E137
:107D50009A838983BE016A5E7F4FCE0101960F949C
:107D6000AC0D25C30E94D68122C380E50E94784BCA
:107D7000882351F00E94F2496093D2047093D30497
:107D80008093D4049093D50489E40E94784B88238F
:107D900081F00E94F2492CEA35EC47E25EE30F9451
:107DA000551A6093CE047093CF048093D0049093BF
:107DB000D10484E40E94784B882381F00E94F24928
:107DC0002CEA35EC47E25EE30F94301F6093CA045F
:107DD0007093CB048093CC049093CD04E3EEF0E554
:107DE00084918F010F5F1F4F882321F00E94E1488B
:107DF000F801F6CF4091D2045091D3046091D4049D
:107E00007091D5048BE794E00E9430E52CEA35ECC4
:107E100047E25EE36091CE047091CF048091D0047C
:107E20009091D1040F94301FAB01BC0187E794E01F
:107E30000E9414E52CEA35EC47E25EE36091CA0447
:107E40007091CB048091CC049091CD040F94551A7D
:107E5000AB01BC0183E794E00E9414E58AE00E9434
:107E6000E148A5C283E50E94784B182F882371F062
:107E70000E94F2490F94981F70935202609351022E
:107E800021E0672B09F020E02093D60480E50E94D2
:107E9000784B882369F08091510290915202892B8E
:107EA00019F00E94E34901C081E08093D6047FC2AB
:107EB00011117DC2E3EEF0E584918F010F5F1F4F3A
:107EC000882321F00E94E148F801F6CF8091D60482
:107ED000882319F06DEF72E002C06AE073E084E974
:107EE00094E00E940E8C609151027091520283E8DE
:107EF00094E00E9420A8EFE7F4E084918F010F5FE7
:107F00001F4F882309F453C20E94E148F801F5CFBE
:107F10000E94DFD84CC20E94466449C281E00E94A0
:107F20004BF045C280E00E944BF041C20E949B632F
:107F30003EC20E9434E03BC20E942B6738C20E94BE
:107F4000AB6535C283E50E94784B882319F00E9407
:107F5000E34901C081E091E089270E94E77C27C2C4
:107F600083E50E94784B882309F421C20E94E349EB
:107F70008093120F1CC20E949A87882319F081E017
:107F80000E94349785E40E94784B882319F00E9460
:107F9000F24904C060E070E080E090EC6AAB7BAB3B
:107FA0008CAB9DAB8AE50E94504C882319F00E944F
:107FB000F24904C060E070E080E291E46EA77FA720
:107FC00088AB99AB88E50E94504C882319F00E9439
:107FD000F24904C060E070E080E291E46AA77BA708
:107FE0008CA79DA789E50E94504C882319F00E9418
:107FF000F24904C060E070E085E393E46EA37FA3E0
:1080000088A799A785E50E94784B882319F00E94DC
:10801000F24904C060E070E088EC92EC6AA37BA3B4
:108020008CA39DA38CE40E94784B882319F00E94B6
:10803000F24903C060E070E0CB016E8B7F8B888FCC
:10804000998F82E40E94504C882321F00E94C249FB
:10805000F62E02C085E0F82ED0906E128091DE04DC
:1080600081117DC0CC24C394EF2C8E010E5D1F4F77
:108070009E012A5D3F4FAE01465D5F4FBE01625DCE
:108080007F4FCE01C2960E9450DE882309F467C05C
:1080900081E080930C0911E080910C09882309F498
:1080A0004AC060E08F2D0F94E00D8091DD0488239D
:1080B000F1F11093D80440E050E0BA0185EC9EE560
:1080C0000E94815680910C09882321F081E00F9451
:1080D000F805F8CF1092D9041092DA041092DB045C
:1080E0001092DC041092DD040E94C7570F9487029F
:1080F0001093D80440E050E0BA0185E19DE50E946C
:1081000081560E94FB4D685370458F4F9F4F60937F
:10811000D9047093DA048093DB049093DC0410920A
:10812000DD0410930C0961E08F2D0F94E00D81E0C8
:108130000F94F805B1CF00E010E028E432E40983A1
:108140001A832B833C838091DE04882341F04F2DDA
:10815000BE016F5F7F4FCE0146960E9426DD21E073
:10816000D21225C10E9416E622C188E50E94784BF2
:108170008823F1F00E94C2498B01222717FD209528
:10818000322F0093DF041093E0042093E104309336
:10819000E204DB012FEF30E00F94492120ED37E0BE
:1081A00040E050E00F94181EB9018EE20E9458A8DA
:1081B0008AE50E94784B882329F00E94C24981E019
:1081C0000E9452CF85E40E94784B882309F4EFC0C7
:1081D0000E94C24982E00E9452CFE9C083E50E941A
:1081E000784B811104C00FE113E0F12C0EC010E0B8
:1081F0000E94D249682F812F17D61F5F1530C1F713
:10820000F2CFF394B4E0FB1669F0D8018D918D01A3
:108210000E94784B8823A9F30E94D249682F8F2DA2
:1082200003D6EFCF82E40E94784B882329F00E9486
:10823000D249682F84E0F8D50E9493A7B8C083E59F
:108240000E94504C8823C1F10E94D249813031F004
:10825000823091F50FE113E0F12C20C00FE113E023
:10826000F12CF80181918F010E94504C882331F04C
:108270000E94D2494FEF682F8F2D57D5F394F4E029
:10828000FF12EFCF82E40E94504C8823A9F00E9495
:10829000D24912C0F394B4E0FB16A1F3D8018D913A
:1082A0008D010E94504C8823A9F30E94D249482F87
:1082B0006FEF8F2D3AD5EECF0E9493A778C08491AF
:1082C0008F010F5F1F4F882319F07BD7F801F7CF7D
:1082D000E7EAF4E084918F010F5F1F4F882309F4D0
:1082E00066C06FD7F801F6CF81E0809353021092F9
:1082F000EB0483E50E94784B811103C00E9469E67C
:1083000056C00E94E349811152C0F8CFF090F404A6
:10831000FF2001F1E3EEF0E584918F010F5F1F4F25
:10832000882319F04ED7F801F7CF84E54AD76F2D8F
:1083300070E080E090E04AE00E949FA680E241D792
:108340000EE013E0F80181918F01882309F4FDC844
:1083500038D7F8CF1092EC04E3EEF0E584918F016A
:108360000F5F1F4F882319F02CD7F801F7CF60E07B
:1083700070E086EB94E00E9420A88AE022D717C024
:10838000E3EEF0E584918F010F5F1F4F882319F012
:1083900018D7F801F7CF6091ED047091EE0488ECE6
:1083A00094E00E940E8C82E20CD78AE00AD70E94E9
:1083B0002BA797C32091B5043091B604232B39F431
:1083C0009F01215031093093B6042093B50420E079
:1083D00030E00C945F2C80E00E9437630E940D4FC8
:1083E00083E50E94784B882309F447C0ECD721E04D
:1083F000482FBE016F5F7F4FCE0146960E9445AC6D
:108400006B017C019B01AC010F940021811130C0F4
:108410002CEA35EC47E257E36E897F89888D998D88
:108420000F94541EAB01BC0185E492E00E9414E558
:108430002CEA35EC47E257E369817A818B819C8194
:108440000F94541EAB01BC0180E492E00E9414E53D
:108450002CEA35EC47E257E3C701B6010F94541EEE
:10846000AB01BC018BE392E00E9414E58AE0A9D63F
:108470000E94F44E0E94E87B9ACF81E0B8CF80E062
:108480000F94F8050C945E377DD7AB01BC01409387
:108490003B1550933C1560933D1570933E158AE84B
:1084A00094E10E94498583CF802F0E9439A86E2DC8
:1084B000802F0E94C24DF12CB701802F0E9458A836
:1084C0000830110509F073CFF0929111E0929011EC
:1084D0006ECF88D70F94981F7093AC0E6093AB0E3D
:1084E00080E00E94C7577ED720E030E040E752E4AA
:1084F0000F94F019181644F00F94530960E08DEAB8
:1085000093E00E94625502C00E9416E66091AB0E95
:108510007091AC0E882777FD8095982F0F94F619EF
:108520002091690430916A0440916B0450916C046D
:108530000F947A2018160CF05AC185EE92E09F93A2
:108540008F9381EA93E09F938F931F920E947F877E
:108550000F900F900F900F900F9081E080938D02FD
:108560001AAE1BAE1CAE1DAE22961CAE1DAE1EAECC
:108570001FAE229710E027961FAE27973CE32B965D
:108580003FAF2B974CE12F964FAF2F9756E4639652
:108590005FAF6397D12CE12C90E8F92E0FEB812C83
:1085A000912C54016091AB0E7091AC0E882777FD31
:1085B0008095982F0F94F619762E672E582E492EF7
:1085C000262F372F482F592F6D2D7E2D8F2D902F31
:1085D0000F94F0198823C9F02091690430916A043E
:1085E00040916B0450916C04672D762D852D942D50
:1085F0000F94F019182F111F1127111F8EA988230E
:1086000041F0112331F011E0E0C07D2C6E2C5F2C85
:10861000402E0E94FB4D6B017C01DC01CB012296B8
:108620002CAD3DAD4EAD5FAD2297821B930BA40BDD
:10863000B50BB7FD38C0D701C60188519C4FAF4F6D
:10864000BF4F22968CAF9DAFAEAFBFAF22970F94B6
:108650006C05EDE9F3E084911F019FEF291A390AB7
:10866000882319F0AED5F101F6CF81149104A1044D
:10867000B104A9F0C501B40168517C4F8F4F9F4FE1
:108680006C197D098E099F0928EE33E040E050E027
:108690000F94F61DCA01B9010E9410A702C08FE312
:1086A00090D58AE08ED580E00F94F8050E94EA4EBE
:1086B000A09169042396AFAF239720906A0430906D
:1086C0006B0400916C042A2F322D432D502F672DFF
:1086D000762D852D942D0F94531E9F7720E030E04A
:1086E00040E251E481149104A104B10429F40F94EF
:1086F000F01987FD05C006C00F947A20181614F4EF
:1087000046015701112309F446C02AAD3BAD4CADDB
:108710005DAD211531054105510541F0D701C60177
:10872000821B930BA40BB50BB7FD35C023962FAD61
:108730002397322D432D502F27966FAD27972B96D9
:108740007FAD2B972F968FAD2F9763969FAD639735
:108750000F94531E20E030E040EC5FE30F94F019DB
:1087600087FD51CFD701C601805A9541AF4FBF4F0A
:108770008AAF9BAFACAFBDAF23969FAD2397279633
:108780009FAF27972B962FAE2B972F963FAE2F9705
:1087900063960FAF639780918D028823B1F08114A7
:1087A0009104A104B10429F4D72CE62CF52C042D56
:1087B000F9CEA8EECA1AA3E0DA0AE108F108C8184F
:1087C000D908EA08FB08F7FCEFCF80918D028823D7
:1087D00009F4EDCD60E0112329F081E893E00E94D7
:1087E0006255E5CD8FE893E00E946255E0CDFEA989
:1087F000F111B3CE80EF92E0A2CEF4D50F94981F82
:108800006739710514F066E970E07093A80E609303
:10881000A70E0E947C57E6D520E030E040EA50E405
:108820000F947A20181614F40E9416E66091A70E91
:108830007091A80E882777FD8095982F0F94F619D0
:1088400020916D0430916E0440916F04509170043A
:108850000F94F01960E087FF03C082EE93E002C03E
:1088600085ED93E00E94625581E080938D028091B6
:10887000EC048093C8041AAE1BAE1CAE1DAE22964B
:108880001CAE1DAE1EAE1FAE22971EAA27961FAEAF
:108890002797BCE32B96BFAF2B97ECE12F96EFAF5A
:1088A0002F97F6E46396FFAF6397C12CD12C00E8B5
:1088B000E02E8FEBF82E812C912C54016091A70EA5
:1088C0007091A80E882777FD8095982F0F94F61940
:1088D000162F072F782E692E262F372F482F592F26
:1088E000B601C7010F94F019882321F120916D047E
:1088F00030916E0440916F0450917004612F702F7D
:10890000872D962D0F94F019881F8827881F8EAB0E
:1089100023962FAD2397222389F0882379F0809125
:108920008D02882309F443CD60E087EC93E00E9438
:1089300062553DCD1C2D0D2D7E2C6F2C0E94FB4DC4
:108940006B017C01DC01CB0122962CAD3DAD4EAD1F
:108950005FAD2297821B930BA40BB50BB7FD38C0FC
:10896000D701C60188519C4FAF4FBF4F22968CAFA5
:108970009DAFAEAFBFAF22970F946C05E1EDF3E072
:1089800084912F019FEF491A590A882319F019D4AD
:10899000F201F6CF81149104A104B104A9F0C5013C
:1089A000B40168517C4F8F4F9F4F6C197D098E0920
:1089B0009F0928EE33E040E050E00F94F61DCA0115
:1089C000B9010E9410A702C08FE3FBD38AE0F9D35C
:1089D00080E00F94F8050E94EA4E20906D043090DC
:1089E0006E0440906F04509070049101A201612FB9
:1089F000702F872D962D0F94531E9F7720E030E027
:108A000040EA50E481149104A104B10429F40F94C4
:108A1000F01987FD05C006C00F947A20181614F4CB
:108A200046015701AEA9AA2309F43FC02AAD3BADC8
:108A30004CAD5DAD211531054105510541F0D70122
:108A4000C601821B930BA40BB50BB7FD2EC0910181
:108A5000A20127966FAD27972B967FAD2B972F9668
:108A60008FAD2F9763969FAD63970F94531E20E0B1
:108A700030E040EC5FE30F94F01987FD50CFD70151
:108A8000C601805A9541AF4FBF4F8AAF9BAFACAF85
:108A9000BDAF27962FAE27972B963FAE2B972F96DD
:108AA0004FAE2F9763965FAE639780918D028823B8
:108AB00009F435CF81149104A104B10429F4C12E25
:108AC000D02EE72CF62CFACE98EEC91A93E0D90AEC
:108AD000E108F108C818D908EA08FB08F7FE1FCF1B
:108AE000EECFC059DF4F0FB6F894DEBF0FBECDBF3B
:108AF000DF91CF911F910F91FF90EF90DF90CF907A
:108B0000BF90AF909F908F907F906F905F904F90AD
:108B10003F902F900895CF93DF932FB7F89494E070
:108B20008902E0011124FE01EA59F14F608171814F
:108B3000828193812FBF0F94F619CD5ED04F28818B
:108B400039814A815B810F94551ADF91CF91089545
:108B5000CF92DF92EF92FF920F931F93CF93DF9309
:108B60007C016A01EB0100E010E00C151D0571F0BD
:108B70006991D701ED91FC910190F081E02DC70141
:108B80001995892B19F00F5F1F4FEFCFC801DF91A7
:108B9000CF911F910F91FF90EF90DF90CF900895AC
:108BA000089580E090E0089580E00895FC01E60FCC
:108BB000F11D849190E0982F88273196E4918E0FD3
:108BC000911D08950895DC011696ED91FC9117977B
:108BD00012968C911297481B15968C91483018F07C
:108BE000E80FF11D4770869586958695489F402D24
:108BF0001124E40FF11D362F377080E890E002C099
:108C0000959587953A95E2F7669566956695E60F90
:108C1000F11D3081222311F0832B02C08095832324
:108C20008083089581E00895089590E0FC013197D4
:108C3000E231F10508F04CC0EE58FF4F0D9443218E
:108C4000809180008F7703C0809180008F7D80931A
:108C50008000089580918000877FF9CF84B58F7759
:108C600002C084B58F7D84BD08958091B0008F7758
:108C700003C08091B0008F7D8093B00008958091F3
:108C800090008F7707C0809190008F7D03C0809106
:108C90009000877F8093900008958091A0008F7747
:108CA00007C08091A0008F7D03C08091A000877FC6
:108CB0008093A0000895809120018F7707C0809154
:108CC00020018F7D03C080912001877F8093200148
:108CD00008953FB7F8948091BC119091BD11A09177
:108CE000BE11B091BF1126B5A89B05C02F3F19F04A
:108CF0000196A11DB11D3FBF6627782F892F9A2F9E
:108D0000620F711D811D911D42E0660F771F881F44
:108D1000991F4A95D1F708956091690470916A048A
:108D200080916B0490916C04089567FD44C081307C
:108D300061F028F08230D9F0833059F13CC06623CD
:108D400011F0A19A6DC0A1986BC09FB7662329F05E
:108D5000F89480910801806804C0F894809108011B
:108D60008F77809308019FBF47FF35C057C09FB7DB
:108D7000662329F0F89480910801806404C0F89477
:108D8000809108018F7B809308019FBF47FF29C016
:108D900046C09FB7662329F0F89480910801886047
:108DA00004C0F89480910801877F809308019FBFD9
:108DB00047FF27C038C047FD36C0813061F028F03A
:108DC000823079F08330E9F00895442311F0A09ABD
:108DD0000895A0980895442311F0A29A0895A298A6
:108DE00008959FB7442329F0F89480910801806288
:108DF00004C0F894809108018F7D809308019FBF83
:108E000008959FB7442329F0F89480910801806168
:108E1000F4CFF894809108018F7EEFCF08950895E4
:108E200047FFD3CF08950895643079F028F4613076
:108E300041F0623041F00895683051F0603141F006
:108E4000089540E003C040E004C041E060E002C09B
:108E500041E061E06ACFF894823041F52091090148
:108E6000247015989FB7662329F0F89480910B0120
:108E7000846004C0F89480910B018B7F80930B0178
:108E80009FBF429A8BE090E00197F1F742989FB71D
:108E9000222329F0F89480910B01846004C0F89497
:108EA00080910B018B7F80930B019FBF7894089575
:108EB00024E08202C0011124FC01EA59F14F4081F3
:108EC000518162817381FC01ED5DF04F40835183DC
:108ED00062837383E091990EF0919A0E828993894F
:108EE000A489B5898093760E9093770EA093780E1F
:108EF000B093790E089580E00EDE6093EF067093D4
:108F0000F0068093F1069093F20681E004DE609310
:108F1000F3067093F4068093F5069093F60682E0CC
:108F2000FADD6093F7067093F8068093F906909344
:108F3000FA0608958091980E9FB780FF09C0F894B3
:108F400080910B018D7F80930B019FBF8FEF08C035
:108F5000F89480910B01826080930B019FBF81E0A8
:108F600080938E028091980E9FB781FF09C0F8947C
:108F700080910B01816080930B019FBF8FEF08C030
:108F8000F89480910B018E7F80930B019FBF81E04D
:108F900080938F028091980E9FB782FF09C0F8944A
:108FA00080910B018B7F80930B019FBF8FEF08C0D7
:108FB000F89480910B01846080930B019FBF81E046
:108FC000809390028091980E9FB783FF09C0F89418
:108FD00080910B01806480930B019FBF8FEF08C0CD
:108FE000F89480910B018F7B80930B019FBF81E0F0
:108FF0008093910208954F925F926F927F92AF9209
:10900000BF92CF92DF92EF92FF920F931F93CF9375
:10901000DF938C01EB01FC0147A050A461A472A472
:10902000AFA0B8A4C9A4DAA49501A601C301B201F6
:109030000F94F01987FF40C0A3019201C301B20150
:109040000F94551A2B013C01F80183A994A9A5A9F5
:10905000B6A9BC01CD0190589B01AC010F94541EE0
:10906000F80127A530A941A952A90F94551A9B01CF
:10907000AC01C301B2010F94531E0F94BF207B01BA
:109080008C019B01AC01B501C6010F94F01987FF5B
:1090900002C0750186019701A801B501C6010F94B0
:1090A000F019882349F0A701B8014FA358A769A771
:1090B0007AA7888181608883DF91CF911F910F917A
:1090C000FF90EF90DF90CF90BF90AF907F906F9028
:1090D0005F904F9008958F929F92AF92BF92CF92E0
:1090E000DF92EF92FF920F931F93CF93DF9300D005
:1090F0001F92CDB7DEB757E9852E51E1952E65EA6F
:10910000A62E64E0B62E05E714E0C12CD12C760122
:10911000C394F40161917191819191914F01F50195
:1091200021913191419151915F0129833A834B8380
:109130005C830F94F41929813A814B815C810F94EF
:10914000551A0F949D1FF801619371938193919328
:109150008F01C616D706E806F90610F46B017C01EC
:10916000F7EA8F16F1E19F06A1F66FEF7FEFCB01D3
:10917000A70196010F94F61D2093B9103093BA10F1
:109180004093BB105093BC100F900F900F900F9016
:10919000DF91CF911F910F91FF90EF90DF90CF90D3
:1091A000BF90AF909F908F9008958EBD0DB407FE35
:1091B000FDCF08958FEF8EBD0DB407FEFDCF8EB5A8
:1091C00008959091C00095FFFCCF8093C60008954C
:1091D000EF92FF921F93CF93DF931F92CDB7DEB72D
:1091E000182FEFEFF6E084917F012FEFE21AF20AD9
:1091F000882329F09983E5DFF7019981F4CFE12FE6
:10920000F92F84917F019FEFE91AF90A882319F059
:10921000D8DFF701F6CFE6EEF6E084917F01AFEFFD
:10922000EA1AFA0A882319F0CCDFF701F6CF0F907B
:10923000DF91CF911F91FF90EF900895CF93DF932F
:10924000ECEEF5E08491EF012196882319F0B9DF67
:10925000FE01F8CFEEEDF5E08491EF012196882331
:1092600019F0AFDFFE01F8CFE7ECF5E08491EF01F4
:109270002196882319F0A5DFFE01F8CFE7EBF5E092
:109280008491EF012196882319F09BDFFE01F8CF2E
:10929000E6EAF5E08491EF012196882319F091DF49
:1092A000FE01F8CFE5E9F5E08491EF0121968823EE
:1092B00019F087DFFE01F8CFE6E8F5E08491EF01D1
:1092C0002196882319F07DDFFE01F8CFE1E7F5E074
:1092D0008491EF012196882319F073DFFE01F8CF06
:1092E000EBE5F5E08491EF012196882319F069DF21
:1092F000FE01F8CFE6E4F5E08491EF0121968823A2
:1093000019F05FDFFE01F8CFE9E2F5E08491EF01AB
:109310002196882319F055DFFE01F8CFE1E1F5E051
:109320008491EF012196882319F04BDFFE01F8CFDD
:10933000DF91CF9108953FB7F89420918F098091E4
:109340008E09821759F0E22FF0E0E25FF64F80813C
:1093500090E02F5F2F7720938F0902C08FEF9FEF50
:109360003FBF08958091FE049091FF04009731F073
:109370004AE050E060E070E00D94301860E070E08A
:10938000CB0108958091FE049091FF04009731F085
:109390004AE050E060E070E00D94FF1660E070E09D
:1093A000CB010895EFDF97FD0CC0ECDF6F3F710537
:1093B0008105910509F014F4E5DF01C06FEF862FF8
:1093C000089580E008958091FE049091FF04892B18
:1093D00039F0E8DF91E0811101C090E0892F089514
:1093E00081E008951F93CF93DF938091FE049091C5
:1093F000FF040097E1F0FC01EF011191212F2F7D77
:1094000079F0153411F01536B9F7188260E070E084
:109410000F9496151883562F472F382F292F0BC0DE
:1094200060E070E0DF91CF911F910D94961550E0B0
:1094300040E030E020E0652F742F832F922FDF91E2
:10944000CF911F910895149A0895179A1092EE0ED5
:10945000169A1092EF0E159A1092F00EF4CFCF924A
:10946000DF92EF92FF92C090C404D090C504E090C8
:10947000C604F090C7048091C904882321F120E03C
:1094800030E0A901C701B6010F94F0198823D9F083
:1094900020E030E040E05FE3C701B6010F94551AC9
:1094A0009B01AC010F94551A2BED3FE049E450E4C9
:1094B0000F94551A9B01AC0160E070E080E89FE3D7
:1094C0000F94301F04C060E070E080E89FE3609379
:1094D000BE107093BF108093C0109093C110FF9086
:1094E000EF90DF90CF900895CF92DF92EF92FF92AE
:1094F000CF93DF93EC0180917802882309F442C076
:10950000C0905602D0905702E0905802F090590255
:10951000A7019601688179818A819B810F947A20C5
:10952000181624F4C882D982EA82FB82C0905A02BB
:10953000D0905B02E0905C02F0905D02A701960182
:109540006C817D818E819F810F947A20181624F47E
:10955000CC82DD82EE82FF82C0905E02D0905F02FC
:10956000E0906002F0906102A7019601688579851C
:109570008A859B850F947A20181624F4C886D9868C
:10958000EA86FB86DF91CF91FF90EF90DF90CF903E
:10959000089580E1EEEFFEE0A0E4B4E001900D92CA
:1095A0008A95E1F7089580E1E0E4F4E0AEEFBEE0F3
:1095B00001900D928A95E1F70895AF92BF92CF92F4
:1095C000DF92EF92FF920F931F93CF93DF93C82FF9
:1095D000DD27C7FDD0958E01000F111F000F111F51
:1095E000F801EE50F14F20E030E0A9016081718177
:1095F000828193810F94541EF801E057F94F208126
:109600003181428153810F94541E6B017C01F8011A
:10961000E05BFB4F60837183828393830B501B4F0E
:10962000F80165917591859194918E01000F111F3C
:10963000000F111F980122583A4F5901A7019601B6
:109640000F94541EF50160837183828393830F5FAF
:109650001A4FF8016591759185919491CC0FDD1F9A
:10966000CC0FDD1FCA5ADD4FA70196010F94541E7F
:10967000688379838A839B83DF91CF911F910F91B8
:10968000FF90EF90DF90CF90BF90AF9008959091B2
:10969000B310E92FF0E0E25FF04F80839F5F9430DA
:1096A00018F49093B31002C01092B3108091B110CF
:1096B0008F5F8093B1100895CF93FC01C62F8081F6
:1096C0008B3399F08091B110843078F42091B310ED
:1096D00030E6239FC0011124BF01805D904F0F949D
:1096E0009A218C2FD4DF81E001C080E0CF910895D2
:1096F00081548A3148F5482F50E0FA01B3E0F595DE
:10970000E795BA95E1F7E45CFB4F208130E0877084
:1097100002C0359527958A95E2F720FF15C0FA011A
:10972000EE5DFB4F2081222339F08091ED04909172
:10973000EE04820F911D02C080E090E09093FF0440
:109740008093FE0481E0089580E00895CF93DF9335
:1097500085E4CEDF882369F036DE882351F0E3EE1E
:10976000F0E58491EF012196882319F02ADDFE01AE
:10977000F8CF81E4BDDF882369F025DE882351F02E
:10978000EDE0F5E08491EF012196882319F019DDD1
:10979000FE01F8CFC091B504D091B6048991882319
:1097A00011F00FDDFBCF8AE0DF91CF910ACD83E589
:1097B0009FDF882349F016DE6093A7067093A80602
:1097C0008093A9069093AA0684E592DF882349F046
:1097D00009DE6093A3067093A4068093A506909378
:1097E000A60682E485DF882349F0BCDD60938B0503
:1097F00070938C0580938D0590938E0588E578DFB6
:10980000882349F0EFDD609395047093960480936C
:1098100097049093980489E56BDF882349F0E2DD93
:109820006093990470939A0480939B0490939C0492
:109830008AE55EDF882349F0D5DD60939D0470934F
:109840009E0480939F049093A00485E451DF8823B5
:1098500049F0C8DD6093A1047093A2048093A3042F
:109860009093A40408950F931F93CF93DF93CFE1B8
:10987000D3E005E814E089913BDF882331F0B2DDC5
:10988000F80160837183828393830C5F1F4FF3E041
:10989000C332DF0781F7DF91CF911F910F910895B8
:1098A00027DF882339F081E02091FE043091FF0406
:1098B000232B09F480E0089583E5F2DF882329F063
:1098C00061DD7093A7026093A602089580914E1205
:1098D00090914F12891B8F7008958CE0EFEEF6E0A7
:1098E000AEEFBEE001900D928A95E1F708959FB723
:1098F000F894E2E0F1E080818B7F80839FBF089540
:109900000B96FC01849108950A96FC0184910895B8
:1099100068E04CC966E04AC9FC0184910895FCDF07
:10992000882311F0823011F486E0089583E00895D1
:10993000FB014181DC0112962C911297421760F0D5
:1099400013962C911397241738F0608115962C915B
:10995000621710F4248137C90895FC0120818281A7
:10996000820F82839181891760F484818F5F848361
:109970008381820F891710F08FEF890F838381E035
:10998000089580E00895FC011282808181508383D4
:109990001482089588E290E00197F1F708952EE986
:1099A0003FE0009729F0F9013197F1F70197F9CFDE
:1099B00008950F93FC010150040F84A996A99417F0
:1099C00018F0081728F402C0081750F0041740F4E4
:1099D0002150260F83A995A9961720F4281720F463
:1099E00080E007C0281720F481E0261710F0F8CF98
:1099F00081E00F910895DB01ED91FC911994EF92B4
:109A0000FF920F931F93CF93DF931F92CDB7DEB7D3
:109A10008C01DC011296ED90FC901397D196ED919C
:109A2000FC91D29782E0199520E030E04AE0B7013E
:109A3000C801E1DFF82ED801D196ED91FC91D297C3
:109A400083E01995D801D196ED91FC91D29780E0F1
:109A50001995FF2081F1F801628173819E012F5FCA
:109A60003F4F46E4C801C7DF8981D8018C93129625
:109A70006D917C9113979E012F5F3F4F47E4C80182
:109A8000BADF8981F80181836281738120E030E04F
:109A900048E4C801B0DFD8011B968C931B9798014E
:109AA0002D5C3F4F12966D917C91139747E1C80151
:109AB000A2DF81E001C080E00F90DF91CF911F9184
:109AC0000F91FF90EF9008958F929F92AF92BF9267
:109AD000CF92DF92EF92FF926B017C01FAD84B019B
:109AE0005C01C114D104E104F104D9F0F2D8681981
:109AF00079098A099B09683E73408105910588F3BD
:109B000021E0C21AD108E108F10888EE880E83E04E
:109B1000981EA11CB11CC114D104E104F10431F759
:109B2000E0CFFF90EF90DF90CF90BF90AF909F90ED
:109B30008F900895CF93DF93282F30E0F901EE5CEA
:109B4000F44D8491F901E451F54DD491F901EA55B0
:109B5000F54DC491CC2389F0811167D8EC2FF0E04A
:109B6000EE0FFF1FE552FB4FA591B4912C912D23D1
:109B700081E090E021F480E002C080E090E0DF919D
:109B8000CF9108950F931F93CF93DF931F92CDB77B
:109B9000DEB7282F30E0F901EE5CF44D8491F90135
:109BA000E451F54D1491F901EA55F54D0491002366
:109BB000C1F0882319F0698338D86981E02FF0E07B
:109BC000EE0FFF1FEE58F54DA591B4919FB7F89495
:109BD0008C91611103C01095812301C0812B8C935E
:109BE0009FBF0F90DF91CF911F910F91089561E07A
:109BF000FC018081C7CF2FB7F8946091C11170919B
:109C0000C2118091C3119091C4112FBF08950F9379
:109C10001F93CF93DF93EB01EEDF8B01CBDA8F3F06
:109C200041F0E9DF601B710B6C177D07B8F380E032
:109C300001C081E0DF91CF911F910F910895CF92E4
:109C4000DF92FF920F931F93CF93DF9300D01F9269
:109C5000CDB7DEB76C01F62EFC018281982F906A99
:109C600096959CBD80FD06C091E0863009F490E099
:109C7000892F01C080E08DBD60E0F60180812983DD
:109C80003A834B835C837EDF6CE271E0C601BFDF09
:109C90008F2D80648ADA08E110E05C814B813A8183
:109CA0002981DA01C901002E04C0B695A7959795C0
:109CB00087950A94D2F729833A834B835C8375DABC
:109CC0000850110929813A814B815C81083FFFEFDF
:109CD0001F0739F7FF2029F088E0F81621F08FEFF1
:109CE00003C085E901C087E860DAECE0FE1201C03C
:109CF00061DA10E05FDAF601838387FF04C01F3F5B
:109D000011F01F5FF7CF0F900F900F900F90DF9122
:109D1000CF911F910F91FF90DF90CF900895CF9238
:109D2000DF92EF92FF920F931F93CF93DF93EC019B
:109D300062DF0E811F8128853985011511052105F6
:109D4000310591F53C853323E1F12A8531503C877B
:109D500031E0320F3A874D85341301C01A86FE0177
:109D600034E0239FE00DF11D11240685178520891D
:109D700031890A831B832C833D836B017C01C00ED8
:109D8000D11EE11CF11CCE82DF82E886F9868C812F
:109D90009D81892BB1F09FB7F89480910201846076
:109DA000809302019FBF0DC06B017C01C01AD10AD4
:109DB000E20AF30AF7FC05C09ADD1E821F821886AC
:109DC0001986DF91CF911F910F91FF90EF90DF9057
:109DD000CF90089510DF60935C0470935D048093CE
:109DE0005E0490935F0408958091FA049091FB04BF
:109DF000A091FC04B091FD0480930A0290930B02A1
:109E0000A0930C02B0930D028091F8049091F90494
:109E10009093A7028093A602DDCF80910A029091D1
:109E20000B02A0910C02B0910D028093FA04909362
:109E3000FB04A093FC04B093FD048091A6029091D2
:109E4000A7029093F9048093F80484E690E090933D
:109E5000A7028093A602BECFFC011382128280EA81
:109E600093E09183808313AE14AE15AECF010496B8
:109E70001186108613861286158621E0248722E239
:109E80002687138A128A20E030E04FEFDC01A20F10
:109E9000B31F93964C932F5F3F4F2E303105B1F790
:109EA00041E044A324ED35E4328F218F438F148E9B
:109EB000158E20E4268F178E22EE35E436AB25ABC7
:109EC000778366839CCD07C9492F441F4427441FCD
:109ED00029F022273327281B390B01C09C01883E1B
:109EE0009340ACF0C90168EE73E00F943021CB01D0
:109EF000EAE0F0E0BF010F943021805D8093BF065F
:109F0000C90164E670E00F943021CB0112C0243601
:109F10003105B4F0442311F08DE201C080E280935A
:109F2000BF06C90164E670E00F943021CB01EAE07E
:109F3000F0E0BF010F943021805D8093C00611C016
:109F400080E28093BF068093C0062A3031059CF0E2
:109F5000442311F08DE201C080E28093C006EAE064
:109F6000F0E0C901BF010F943021CB01BF010F9474
:109F70003021805D05C0442311F08DE201C080E2F4
:109F80008093C106C9016AE070E00F943021805DC2
:109F90008093C2068FEB96E008959C0197FD0EC05A
:109FA0008436910584F064E670E00F943021CB0193
:109FB0006AE070E00F943021805D06C031952195F4
:109FC00031098DE201C080E28093C0062A3031055C
:109FD00064F0EAE0F0E0C901BF010F943021CB0149
:109FE000BF010F943021805D01C080E28093C106E3
:109FF000C9016AE070E00F943021805D8093C20651
:10A0000080EC96E008950F931F93CF93DF93EC01BC
:10A010008881813011F4EFDD04C069857A858B85F4
:10A020009C850D811E812F813885601B710B820BF1
:10A03000930B28EE33E040E050E00F94F61D898149
:10A040009A81AB81BC81280F391F4A1F5B1FCA014F
:10A05000B901DF91CF911F910F910895CF92DF92B7
:10A06000EF92FF920F931F93CF93DF93E091990E9E
:10A07000F0919A0E82819381A481B58118161906F8
:10A080001A061B06ACF58091980E90915D054091E3
:10A090005C0580FF10C083B186FB222720F99E7FDC
:10A0A000292B20935D05942F9170922309F18091C3
:10A0B0002F0F816018C086B1292F30E0992787FDC6
:10A0C0009095990F880B982F822793278071992755
:10A0D0008227932780935D05942F9071982341F0F8
:10A0E00080912F0F806180932F0F80E00E9458474E
:10A0F000E091990EF0919A0E86819781A085B185A5
:10A10000181619061A061B060CF040C09091980EFE
:10A1100080915D0520915C0591FF1AC033B190E0FC
:10A1200035FBCC24C0F8D12CD194C194D108C826D9
:10A13000D92632E0C322DD24C826D926C0925D0587
:10A14000822F82708C2111F180912F0F826019C0B3
:10A1500030B190E032FBEE24E0F8F12CF194E19480
:10A16000F108E826F92630E2E322FF24E826F92662
:10A17000E0925D05822F80728E2141F080912F0F39
:10A18000806280932F0F81E00E945847E091990EE2
:10A19000F0919A0E82859385A485B58518161906C7
:10A1A0001A061B060CF046C09091980E80915D0532
:10A1B00092FF21C09091F10E9923E1F123B190E03B
:10A1C00022952F7031E02327022F017010E01195A6
:10A1D0000195110908271927047011270827192745
:10A1E00000935D0580915C058470802319F1809156
:10A1F0002F0F84601AC020B190E026952170C22FE5
:10A2000020E0D22FD195C195D109C827D927C07494
:10A21000DD27C827D927C0935D0580915C05807430
:10A220008C2341F080912F0F806480932F0F82E068
:10A230000E94584780915D0580935C05DF91CF9126
:10A240001F910F91FF90EF90DF90CF9008954F9264
:10A250005F926F927F928F929F92AF92BF92CF92B6
:10A26000DF92EF92FF920F931F93CF93DF9300D073
:10A270001F92CDB7DEB78C01DC014D905D906D90E3
:10A280007C90139714968D909D90AD90BC901797ED
:10A2900018968D919D910D90BC91A02D89839A83E4
:10A2A000AB83BC83A3019201C301B2010F94551A81
:10A2B0006B017C01A5019401C501B4010F94551AED
:10A2C0009B01AC01C701B6010F94541E6B017C01C8
:10A2D00029813A814B815C81CA01B9010F94551AD9
:10A2E0009B01AC01C701B6010F94541E0F94BF200F
:10A2F0009B01AC0160E070E080E89FE30F94301FA9
:10A300006B017C019B01AC01C301B2010F94551A92
:10A31000F8016083718382839383A7019601C5014D
:10A32000B4010F94551AD80114966D937D938D93B3
:10A330009C931797A701960169817A818B819C81F3
:10A340000F94551AF80160877187828793870F9061
:10A350000F900F900F90DF91CF911F910F91FF9071
:10A36000EF90DF90CF90BF90AF909F908F907F90B5
:10A370006F905F904F9008954F925F926F927F928F
:10A380008F929F92AF92BF92CF92DF92EF92FF9205
:10A39000CF93DF93CDB7DEB728970FB6F894DEBF23
:10A3A0000FBECDBF2496AEADBFAD24978D919D91CC
:10A3B0000D90BC91A02D89839A83AB83BC83229698
:10A3C000EEADFFAD2297C080D180E280F380AEADCC
:10A3D000BFAD8D909D90AD90BC902E8D3F8D48A1CE
:10A3E00059A1C501B4010F94551A2B013C012AA5AE
:10A3F0003BA54CA55DA5C701B6010F94551A9B015D
:10A40000AC01C301B2010F94541E2B013C012EA9D3
:10A410003FA948AD59AD69817A818B819C810F94A8
:10A42000551A9B01AC01C301B2010F94541E6D83F8
:10A430007E838F8398872AA13BA14CA15DA1C50192
:10A44000B4010F94551A2B013C012EA53FA548A934
:10A4500059A9C701B6010F94551A9B01AC01C3015C
:10A46000B2010F94541E2B013C012AAD3BAD4CAD03
:10A470005DAD69817A818B819C810F94551A9B0116
:10A48000AC01C301B2010F94541E2B013C012A8D73
:10A490003B8D4C8D5D8DC501B4010F94551A4B0158
:10A4A0005C012EA13FA148A559A5C701B6010F9493
:10A4B000551A9B01AC01C501B4010F94541E6B01E8
:10A4C0007C012AA93BA94CA95DA969817A818B816C
:10A4D0009C810F94551A9B01AC01C701B6010F94E2
:10A4E000541EEEADFFAD60837183828393838D81B3
:10A4F0009E81AF81B8852296EEADFFAD2297808315
:10A500009183A283B3832496AEADBFAD24974D92C1
:10A510005D926D927C92139728960FB6F894DEBFE9
:10A520000FBECDBFDF91CF91FF90EF90DF90CF9026
:10A53000BF90AF909F908F907F906F905F904F9063
:10A5400008954F925F926F927F928F929F92AF92F7
:10A55000BF92CF92DF92EF92FF920F931F93CF9310
:10A56000DF93CDB7DEB7C454D1090FB6F894DEBF80
:10A570000FBECDBF8C0180919F06882309F43AC19C
:10A58000C0900A12D0900B12E0900C12F0900D12B5
:10A5900020910E1230910F12409110125091111211
:10A5A00029AB3AAB4BAB5CAB4090121250901312FC
:10A5B00060901412709015128091161290911712DB
:10A5C000A0911812B091191225968CAF9DAFAEAF25
:10A5D000BFAF259720911A1230911B1240911C1287
:10A5E00050911D122DAB3EAB4FAB58AF80901E1259
:10A5F00090901F12A0902012B09021124091221230
:10A60000509123126091241270912512809126128C
:10A6100090912712A0912812B091291289AF9AAF78
:10A62000ABAFBCAF8091061290910712A0910812B7
:10A63000B091091289839A83AB83BC834D825E8279
:10A640006F82788689869A86AB86BC86CD86DE86C2
:10A65000EF86F88A25968CAD9DADAEADBFAD259742
:10A66000898B9A8BAB8BBC8B4D8B5E8B6F8B788F72
:10A6700029A93AA94BA95CA9298F3A8F4B8F5C8FE6
:10A680008DA99EA9AFA9B8AD8D8F9E8FAF8FB8A3AE
:10A6900029AD3AAD4BAD5CAD29A33AA34BA35CA366
:10A6A0002091500430915104409152045091530430
:10A6B000D8016D917D918D919C910F94531E6DA742
:10A6C0007EA78FA798AB20915404309155044091F8
:10A6D000560450915704F8016481758186819781F1
:10A6E0000F94531E20E030E04FE353E40F94531EC9
:10A6F00069A77AA78BA79CA7209158043091590489
:10A7000040915A0450915B04D80118966D917D9147
:10A710008D919C911B970F94531E6DA37EA38FA3C5
:10A7200098A7CE0185969F938F9304969F938F93BE
:10A7300004969F938F93EDB7FEB7B4970FB6F89436
:10A74000FEBF0FBEEDBFADB7BEB7119684E2FE01EE
:10A75000319601900D928A95E1F70EDE20E030E00F
:10A76000A9016DA57EA58FA598A90F94541E2091CF
:10A7700050043091510440915204509153040F946D
:10A78000541ED8016D937D938D939C93139720E075
:10A7900030E04FE353E469A57AA58BA59CA50F94FF
:10A7A000541E209154043091550440915604509108
:10A7B00057040F94541EF80164837583868397832E
:10A7C000209158043091590440915A0450915B04EF
:10A7D0006DA17EA18FA198A50F94541ED801189643
:10A7E0006D937D938D939C931B970FB6F894DEBF6A
:10A7F0000FBECDBFCC5BDF4F0FB6F894DEBF0FBEF0
:10A80000CDBFDF91CF911F910F91FF90EF90DF901F
:10A81000CF90BF90AF909F908F907F906F905F9000
:10A820004F900895CF92DF92EF92FF920F931F9374
:10A83000CF93DF93CDB7DEB72C970FB6F894DEBF7A
:10A840000FBECDBF6C017B018A0180919F068823DA
:10A8500009F4A5C020915004309151044091520454
:10A8600050915304F60160817181828193810F942C
:10A87000531E69877A878B879C8720915404309177
:10A8800055044091560450915704F701608171813D
:10A89000828193810F94531E20E030E04FE353E414
:10A8A0000F94531E6D837E838F8398872091580465
:10A8B0003091590440915A0450915B04F801608131
:10A8C0007181828193810F94531E69837A838B8374
:10A8D0009C83CE0101969F938F9304969F938F93B1
:10A8E00004969F938F938DB79EB784970FB6F89475
:10A8F0009EBF0FBE8DBFADB7BEB7119684E2E6E036
:10A90000F2E101900D928A95E1F736DD20E030E02A
:10A91000A90169857A858B859C850F94541E2091A9
:10A9200050043091510440915204509153040F94BB
:10A93000541EF601608371838283938320E030E0AC
:10A940004FE353E46D817E818F8198850F94541E6F
:10A95000209154043091550440915604509157046D
:10A960000F94541EF7016083718382839383209137
:10A9700058043091590440915A0450915B04698104
:10A980007A818B819C810F94541EF80160837183BE
:10A99000828393830FB6F894DEBF0FBECDBF2C9693
:10A9A0000FB6F894DEBF0FBECDBFDF91CF911F91E0
:10A9B0000F91FF90EF90DF90CF9008950F931F932A
:10A9C0001AD90091690510916A0520916B053091A3
:10A9D0006C05601B710B820B930B97FD10C080916F
:10A9E00003018695817091E089279091030192FF80
:10A9F00082609091000196FF846080937D05809134
:10AA00007D05817090917D0591FD826090915B053F
:10AA1000891731F18130A9F028F0823041F083307C
:10AA200059F01CC0913089F0923099F017C09923E9
:10AA300061F0933071F012C0913059F0923071F49E
:10AA400004C0992331F0933049F4909175059150E9
:10AA500003C0909175059F5F9093750580935B058A
:10AA60001F910F910895EEE0F2E080E09191911135
:10AA700005C0282F482F421B50E204C0863181F4C4
:10AA800026E1F8CF822F90E0342F320FFC01E25FF5
:10AA9000FD4F363118F450832F5FF4CF10820895A4
:10AAA0008F5FE4CF2091EB0421110BC042E450E012
:10AAB000BC018EE092E00F94AF21D5DF83E080935C
:10AAC000A802089567FF03C01092EB0460E0209194
:10AAD000EB0430E0462F552747FD509542175307AA
:10AAE0006CF06093EB0442E450E0BC018EE092E035
:10AAF0000F946119B8DF83E08093A8020895CF9284
:10AB0000DF92EF92FF920F931F9375D80091570534
:10AB1000109158052091590530915A056B017C011F
:10AB2000C01AD10AE20AF30AF7FC13C020915605B5
:10AB3000209520935605DC01CB018A549C4FAF4FE2
:10AB4000BF4F8093570590935805A0935905B09334
:10AB50005A0581E090915605911101C080E01F9146
:10AB60000F91FF90EF90DF90CF900895CF92DF92FA
:10AB7000EF92FF92CF93C82F3ED86B017C0124EA5D
:10AB800030E74DE75FE36091080970910909809112
:10AB90000A0990910B090F94F01987FF04C040E057
:10ABA00050E0BA0104C04AEF50E060E070E04C0DA4
:10ABB0005D1D6E1D7F1D4093650550936605609376
:10ABC000670570936805C0935402CF91FF90EF9092
:10ABD000DF90CF900895209155052630D8F486E077
:10ABE000289FF0011124EF5CFA4F8091760290913A
:10ABF0007702918380838091B7119091B811A091D1
:10AC0000B911B091BA1182839383A483B5832F5F66
:10AC10002093550508956F927F928F929F92AF92E5
:10AC2000BF92CF92DF92EF92FF920F931F93CF9339
:10AC3000DF9300D01F92CDB7DEB76C013B01470117
:10AC4000580129833A834B835C83C5DF83E080937B
:10AC5000A802D092B806C092B7067092B60660926B
:10AC6000B50629813A814B815C81CA01B9010F94F3
:10AC7000981F6093B1067093B2068093B3069093C9
:10AC8000B4060F94F6196B017C019B01AC01C50160
:10AC9000B4010F94531E0F94981F6093AD067093E8
:10ACA000AE068093AF069093B006A7019601F3011C
:10ACB00060817181828193810F94531E0F949D1F37
:10ACC0006093B7117093B8118093B9119093BA1132
:10ACD00081E99AEC90937702809376020F900F901F
:10ACE0000F900F90DF91CF911F910F91FF90EF90F8
:10ACF000DF90CF90BF90AF909F908F907F906F909C
:10AD00000895209176023091770228173907D9F0FB
:10AD100090937702809376024093B7115093B811C5
:10AD20006093B9117093BA11895D984921F410921A
:10AD3000D8041092550582E08093A80281E08093A8
:10AD4000B511109276050895CF93DF931F921F924D
:10AD5000CDB7DEB789839A833EDF40E050E0BA0189
:10AD600089819A810F900F90DF91CF91CACF21E016
:10AD70002093D804609308097093090980930A0905
:10AD800090930B0940E050E0BA018091D906909170
:10AD9000DA06B7CF6DEC7CEC8CEC9DE3E8CF60E09D
:10ADA00070E080E89FE3E3CF60E070E080E291E450
:10ADB000DECF40E050E0BA0189ED98E9A2CFE09102
:10ADC0005505EE2381F0E150E093550586E0E89FBC
:10ADD000F0011124EF5CFA4F428153816481758147
:10ADE000808191818ECFE5CFCF93DF93EC016CE62C
:10ADF00072E032D884E993E099838883DF91CF9120
:10AE000008955A9887FD52C05B980000000000002A
:10AE100000005A9A5A98282F220F86FD53C05B983B
:10AE200000000000000000005A9A5A98922F990FD3
:10AE300026FD46C05B9800000000000000005A9A02
:10AE40005A98892F880F96FD39C05B980000000042
:10AE5000000000005A9A5A98982F990F86FD2CC02E
:10AE60005B9800000000000000005A9A5A98892F51
:10AE7000880F96FD1FC05B980000000000000000D6
:10AE80005A9A5A98982F990F86FD12C05B98000025
:10AE90000000000000005A9A5A9896FD15C05B9871
:10AEA00000000000000000005A9A08955B9AADCFA0
:10AEB0005B9AEDCF5B9AE0CF5B9AD3CF5B9AC6CF1C
:10AEC0005B9AB9CF5B9AACCF5B9AEACFFC0120E0EA
:10AED0003EE2DB014C91403241F0283011F43083E6
:10AEE0003196DB014C91408331962F5F6F5F7F4F2E
:10AEF0002B3079F710820895CF92DF92EF92FF9274
:10AF0000C0906D04D0906E04E0906F04F0907004D7
:10AF10006091A70E7091A80E68507109882777FD7F
:10AF20008095982F0F94F6199B01AC01C701B601CB
:10AF30000F94F01987FF1DC020E030E040E050E49E
:10AF4000C701B6010F94541E0F949D1F70937B117F
:10AF500060937A110E94FB4D605A75418F4F9F4F4D
:10AF600060937C1170937D1180937E1190937F117B
:10AF700008C010927C1110927D1110927E111092D7
:10AF80007F11FF90EF90DF90CF900895B5CFCF92D3
:10AF9000DF92EF92FF92C0906904D0906A04E09033
:10AFA0006B04F0906C046091AB0E7091AC0E6D5020
:10AFB0007109882777FD8095982F0F94F6199B01CA
:10AFC000AC01C701B6010F94F01987FF1DC020E046
:10AFD00030E040E050E4C701B6010F94541E0F94D6
:10AFE0009D1F70938111609380110E94FB4D605EE4
:10AFF000714B8F4F9F4F6093821170938311809399
:10B0000084119093851108C01092821110928311BF
:10B010001092841110928511FF90EF90DF90CF90E5
:10B02000089580E0B4CF4F925F926F927F928F929B
:10B030009F92AF92BF92CF92DF92EF92FF920F93C7
:10B040001F93CF93DF932C012BE837E081E090E052
:10B05000F90145915491441655060CF062C0AC01BB
:10B0600041505109DA01AA0FBB1FAA0FBB1FA757F6
:10B07000B84FFD0165917491440F551F440F551F42
:10B080004957584FFA0165907490FC01EE0FFF1F6D
:10B09000EE0FFF1FE757F84FA590B490FD01059103
:10B0A0001491F901C591D491FA0185909490882763
:10B0B00077FD8095982F0F94F6196B017C01B201F2
:10B0C00066197709882777FD8095982F0F94F619D0
:10B0D0002B013C01B501601B710B882777FD809522
:10B0E000982F0F94F6199B01AC01C301B2010F9484
:10B0F000551A2B013C01BE0168197909882777FD93
:10B100008095982F0F94F6199B01AC01C301B201F1
:10B110000F94301F9B01AC01C701B6010F94541E60
:10B1200011C001962C5F3F4F8A33910509F090CFF3
:10B13000EDE6F8E065917491882777FD8095982F6A
:10B140000F94F619DF91CF911F910F91FF90EF901F
:10B15000DF90CF90BF90AF909F908F907F906F9037
:10B160005F904F9008954F925F926F927F928F926F
:10B170009F92AF92BF92CF92DF92EF92FF92CF93C6
:10B18000DF93CDB7DEB72C970FB6F894DEBF0FBEB6
:10B19000CDBF80916D0490916E04A0916F04B09129
:10B1A000700489839A83AB83BC836091A70E7091EE
:10B1B000A80E882777FD8095982F0F94F61929817E
:10B1C0003A814B815C810F94531E6B017C0160932B
:10B1D0002D0570932E0580932F05909330052091B7
:10B1E000D2043091D3044091D4045091D5040F94EB
:10B1F000551A6D837E838F8398876093290570939A
:10B200002A0580932B0590932C05209125053091DC
:10B2100026054091270550912805C701B6010F94D6
:10B22000541E4B015C0160932505709326058093A5
:10B230002705909328052091CE043091CF044091AA
:10B24000D0045091D1040F94551A69877A878B875F
:10B250009C8760932105709322058093230590932A
:10B26000240520ED3CEC4CE45DE36091CA04709150
:10B27000CB048091CC049091CD040F94551A2B01EE
:10B280003C0120911D0530911E0540911F055091F4
:10B29000200569817A818B819C810F94531E9B01CB
:10B2A000AC01C301B2010F94551A2B013C0123E3F9
:10B2B00033E343E75FE36091190570911A058091CC
:10B2C0001B0590911C050F94551A9B01AC01C301FD
:10B2D000B2010F94541E2B013C0160931905709329
:10B2E0001A0580931B0590931C0589819A81AB8177
:10B2F000BC8180931D0590931E05A0931F05B093FC
:10B30000200529853A854B855C856D817E818F81FD
:10B3100098850F94541EA30192010F94531E2B0184
:10B320003C0120E030E04FE753E40F947A2020E026
:10B3300030E0A9011816ACF4C701B6010F947A20C9
:10B3400018166CF5A7019601C501B4010F94531EA0
:10B350006093250570932605809327059093280513
:10B360001EC0C301B2010F94F01987FF22C020E074
:10B3700030E0A901C701B6010F94F01987FF16C08C
:10B38000A7019601C501B4010F94531E60932505D2
:10B3900070932605809327059093280507C0412CBC
:10B3A000512C8FE7682E83E4782E03C0412C512C5A
:10B3B0003201C301B2012C960FB6F894DEBF0FBE66
:10B3C000CDBFDF91CF91FF90EF90DF90CF90BF90F6
:10B3D000AF909F908F907F906F905F904F90089567
:10B3E0004F925F926F927F928F929F92AF92BF9295
:10B3F000CF92DF92EF92FF920F931F93CF93DF9341
:10B4000000D01F92CDB7DEB70091AB0E1091AC0EFD
:10B410008090690490906A04A0906B04B0906C04D2
:10B42000B801882777FD8095982F0F94F619A5010C
:10B4300094010F94531E6B017C016093150570936A
:10B440001605809317059093180520ED3CEC4CE40D
:10B450005DE36091D40E7091D50E8091D60E9091DF
:10B46000D70E0F94551A2B013C01209111053091F4
:10B4700012054091130550911405C501B4010F94B4
:10B48000531E9B01AC01C301B2010F94551A2B014D
:10B490003C0123E333E343E75FE360910D057091E3
:10B4A0000E0580910F05909110050F94551A9B0180
:10B4B000AC01C301B2010F94541E69837A838B835C
:10B4C0009C8360930D0570930E0580930F059093F8
:10B4D00010058092110590921205A0921305B0926A
:10B4E00014058091DD04882321F081E080930C0510
:10B4F000B9C020E030E040E251E4C701B6010F944A
:10B500007A20181624F481E080930C05A4C020E072
:10B5100030E040E251ECC701B6010F94F01987FD0D
:10B52000E4CF012B11F380910C05882351F0109288
:10B5300008051092090510920A0510920B05109249
:10B540000C052091DC0E3091DD0E4091DE0E509105
:10B55000DF0EC701B6010F94551A2B013C01609311
:10B5600004057093050580930605909307052091C7
:10B5700008053091090540910A0550910B05C70156
:10B58000B6010F94541E4B015C0160930805709343
:10B59000090580930A0590930B052091D80E3091F0
:10B5A000D90E4091DA0E5091DB0E0F94551A9B0183
:10B5B000AC016093000570930105809302059093A0
:10B5C0000305C301B2010F94541E29813A814B81B6
:10B5D0005C810F94531E2B013C0120E030E04FE7CB
:10B5E00053E40F947A2020E030E0A9011816ACF45F
:10B5F000C701B6010F947A2018166CF5A7019601C1
:10B60000C501B4010F94531E60930805709309059A
:10B6100080930A0590930B051EC0C301B2010F94DD
:10B62000F01987FF22C020E030E0A901C701B60170
:10B630000F94F01987FF16C0A7019601C501B40148
:10B640000F94531E609308057093090580930A05B3
:10B6500090930B0507C0412C512C9FE7692E93E472
:10B66000792E03C0412C512C3201C301B2010F903D
:10B670000F900F900F90DF91CF911F910F91FF903E
:10B68000EF90DF90CF90BF90AF909F908F907F9082
:10B690006F905F904F90089560916D0470916E046B
:10B6A00080916F049091700408954F925F926F9211
:10B6B0007F928F929F92AF92BF92CF92DF92EF9242
:10B6C000FF920F931F93CF93DF932C012BE037E072
:10B6D00081E090E0F90145915491441655060CF033
:10B6E00062C0AC0141505109DA01AA0FBB1FAA0F79
:10B6F000BB1FA75FB84FFD0165917491440F551FA3
:10B70000440F551F495F584FFA0165907490FC0132
:10B71000EE0FFF1FEE0FFF1FE75FF84FA590B490ED
:10B72000FD0105911491F901C591D491FA0185901B
:10B730009490882777FD8095982F0F94F6196B01C8
:10B740007C01B20166197709882777FD8095982FCB
:10B750000F94F6192B013C01B501601B710B882772
:10B7600077FD8095982F0F94F6199B01AC01C301CA
:10B77000B2010F94551A2B013C01BE0168197909D9
:10B78000882777FD8095982F0F94F6199B01AC01BF
:10B79000C301B2010F94301F9B01AC01C701B60178
:10B7A0000F94541E11C001962C5F3F4F80329105BB
:10B7B00009F090CFE5E8F7E065917491882777FD6F
:10B7C0008095982F0F94F619DF91CF911F910F91CB
:10B7D000FF90EF90DF90CF90BF90AF909F908F90B1
:10B7E0007F906F905F904F9008951F93CF93DF935A
:10B7F0001092BB118091B7119091B811A091B9111D
:10B80000B091BA1181309048A105B10540F0109275
:10B81000B7111092B8111092B9111092BA11C091CB
:10B82000B71140916305141604F5842F992787FDFD
:10B83000909505972C2F332727FD3095281739072A
:10B84000A4F045301CF0CBEFC40F01C0C0E08C2F3A
:10B85000992787FD9095A92FB92F8093B7119093C1
:10B86000B811A093B911B093BA11C093B411D0E03C
:10B8700012E0C11109C08091A8028823D9F121E00A
:10B8800041E067EB79E020C0C13049F48091A80223
:10B89000882381F120E041E068EA79E015C0C230F8
:10B8A00049F48091A802882329F120E041E068E969
:10B8B00079E00AC0C33061F48091A8028823D1F0F6
:10B8C00020E041E061E979E08D2F0E9422A012C0C2
:10B8D000C43081F48091A802882351F021E040E037
:10B8E00066E879E08D2F0E9422A08D2F0E940BAA7E
:10B8F0001093A802DF5FCF5FD53009F0BACFD093A5
:10B900006305DF91CF911F9108951F93CF93DF932C
:10B910001092BB118091B7119091B811A091B911FB
:10B92000B091BA1181309048A105B10540F0109254
:10B93000B7111092B8111092B9111092BA11C091AA
:10B94000B71140916205141604F5842F992787FDDD
:10B95000909505972C2F332727FD30952817390709
:10B96000A4F045301CF0CBEFC40F01C0C0E08C2F19
:10B97000992787FD9095A92FB92F8093B7119093A0
:10B98000B811A093B911B093BA11C093B411D0E01B
:10B9900012E0C11109C08091A8028823D9F121E0E9
:10B9A00041E069E779E020C0C13049F48091A80204
:10B9B000882381F120E041E060E779E015C0C230E2
:10B9C00049F48091A802882329F120E041E060E653
:10B9D00079E00AC0C33061F48091A8028823D1F0D5
:10B9E00020E041E06EE579E08D2F0E9422A012C098
:10B9F000C43081F48091A802882351F021E040E016
:10BA000063E579E08D2F0E9422A08D2F0E940BAA62
:10BA10001093A802DF5FCF5FD53009F0BACFD09383
:10BA20006205DF91CF911F9108951F93CF93DF930C
:10BA30001092BB118091B7119091B811A091B911DA
:10BA4000B091BA1181309048A105B10540F0109233
:10BA5000B7111092B8111092B9111092BA11C09189
:10BA6000B71140916105141604F5842F992787FDBD
:10BA7000909505972C2F332727FD309528173907E8
:10BA8000A4F045301CF0CBEFC40F01C0C0E08C2FF8
:10BA9000992787FD9095A92FB92F8093B71190937F
:10BAA000B811A093B911B093BA11C093B411D0E0FA
:10BAB00012E0C11109C08091A8028823D9F121E0C8
:10BAC00041E066E479E020C0C13049F48091A802E9
:10BAD000882381F120E041E066E379E015C0C230BF
:10BAE00049F48091A802882329F120E041E065E231
:10BAF00079E00AC0C33061F48091A8028823D1F0B4
:10BB000020E041E066E179E08D2F0E9422A012C082
:10BB1000C43081F48091A802882351F021E040E0F4
:10BB20006BE079E08D2F0E9422A08D2F0E940BAA3E
:10BB30001093A802DF5FCF5FD53009F0BACFD09362
:10BB40006105DF91CF911F9108951F93CF93DF93EC
:10BB50001092BB118091B7119091B811A091B911B9
:10BB6000B091BA1181309048A105B10540F0109212
:10BB7000B7111092B8111092B9111092BA11C09168
:10BB8000B71140916005141604F5842F992787FD9D
:10BB9000909505972C2F332727FD309528173907C7
:10BBA000A4F045301CF0CBEFC40F01C0C0E08C2FD7
:10BBB000992787FD9095A92FB92F8093B71190935E
:10BBC000B811A093B911B093BA11C093B411D0E0D9
:10BBD00012E0C11109C08091A8028823D9F121E0A7
:10BBE00041E06EEF78E020C0C13049F48091A802B6
:10BBF000882381F120E041E065EF78E015C0C23094
:10BC000049F48091A802882329F120E041E067EE01
:10BC100078E00AC0C33061F48091A8028823D1F093
:10BC200020E041E065EE78E08D2F0E9422A012C056
:10BC3000C43081F48091A802882351F021E040E0D3
:10BC40006AED78E08D2F0E9422A08D2F0E940BAA12
:10BC50001093A802DF5FCF5FD53009F0BACFD09341
:10BC60006005DF91CF911F9108951F93CF93DF93CC
:10BC70001092BB118091B7119091B811A091B91198
:10BC8000B091BA1181309048A105B10540F01092F1
:10BC9000B7111092B8111092B9111092BA11C09147
:10BCA000B71140915F05141604F5842F992787FD7D
:10BCB000909505972C2F332727FD309528173907A6
:10BCC000A4F045301CF0CBEFC40F01C0C0E08C2FB6
:10BCD000992787FD9095A92FB92F8093B71190933D
:10BCE000B811A093B911B093BA11C093B411D0E0B8
:10BCF00012E0C11109C08091A8028823D9F121E086
:10BD000041E06DEC78E020C0C13049F48091A80298
:10BD1000882381F120E041E064EC78E015C0C23076
:10BD200049F48091A802882329F120E041E063EBE7
:10BD300078E00AC0C33061F48091A8028823D1F072
:10BD400020E041E061EB78E08D2F0E9422A012C03C
:10BD5000C43081F48091A802882351F021E040E0B2
:10BD600066EA78E08D2F0E9422A08D2F0E940BAAF8
:10BD70001093A802DF5FCF5FD53009F0BACFD09320
:10BD80005F05DF91CF911F9108951F93CF93DF93AC
:10BD90001092BB118091B7119091B811A091B91177
:10BDA000B091BA1181309048A105B10540F01092D0
:10BDB000B7111092B8111092B9111092BA11C09126
:10BDC000B71140915E05141604F5842F992787FD5D
:10BDD000909505972C2F332727FD30952817390785
:10BDE000A4F045301CF0CBEFC40F01C0C0E08C2F95
:10BDF000992787FD9095A92FB92F8093B71190931C
:10BE0000B811A093B911B093BA11C093B411D0E096
:10BE100012E0C11109C08091A8028823D9F121E064
:10BE200041E069E978E020C0C13049F48091A8027E
:10BE3000882381F120E041E069E878E015C0C23054
:10BE400049F48091A802882329F120E041E06CE7C1
:10BE500078E00AC0C33061F48091A8028823D1F051
:10BE600020E041E06AE778E08D2F0E9422A012C016
:10BE7000C43081F48091A802882351F021E040E091
:10BE80006FE678E08D2F0E9422A08D2F0E940BAAD2
:10BE90001093A802DF5FCF5FD53009F0BACFD093FF
:10BEA0005E05DF91CF911F9108950F931F93CF935C
:10BEB000DF931092BB118091B7119091B811A091AE
:10BEC000B911B091BA1181309048A105B10540F087
:10BED0001092B7111092B8111092B9111092BA11B4
:10BEE000C091B711409164051416D4F4842F99279A
:10BEF00087FD909501972C2F332727FD3095281724
:10BF0000390774F0CFEFC40F8C2F90E0A0E0B0E0C1
:10BF10008093B7119093B811A093B911B093BA114F
:10BF20001092B5118091B411C81714F4C093B411D4
:10BF30008091B411992787FD909504962C2F332773
:10BF400027FD30958217930724F48CEF8C0F809394
:10BF5000B4111091B411D0E081E002E0111123C0BE
:10BF60008823B9F01C16ACF04091B7115091B8116C
:10BF70006091B9117091BA114F5F5F4F6F4F7F4F52
:10BF80004093B7115093B8116093B9117093BA11DF
:10BF9000CF5F8091A802882309F469C021E041E0C5
:10BFA0006BEE79E04EC0113019F58823B9F0C2303C
:10BFB000ACF44091B7115091B8116091B9117091E2
:10BFC000BA114F5F5F4F6F4F7F4F4093B711509340
:10BFD000B8116093B9117093BA11CF5F8091A80224
:10BFE000882309F444C020E040E066ED79E029C0F0
:10BFF0001230E9F48091B311811105C08091A8023B
:10C000008823A9F109C0C230C9F70E94DF56809188
:10C01000B511882399F333C081E0C23009F080E084
:10C0200024E041ED59E06D2F0E94FBA120C01330A8
:10C0300061F48091A8028823D1F020E041E06FEC08
:10C0400079E08D2F0E9422A012C0143081F48091DB
:10C05000A802882351F021E040E064EC79E08D2FC4
:10C060000E9422A08D2F0E940BAA0093A802DF5FDE
:10C070001F5FD53011F080E071CFD0936405DF9160
:10C08000CF911F910F910895CF93DF93EC018B8196
:10C09000882391F1898187FF2BC06C857D858E85F2
:10C0A0009F8541E00E949F83882331F1E88980E2E7
:10C0B000E89FF0011124EE5FF84F3097E9F080819E
:10C0C000853ED1F08B81823040F449895A896B8951
:10C0D0007C89448F558F668F778F4D895E896F89F4
:10C0E000788D538F428F758B648B89818F7789838D
:10C0F000DF91CF910C94618381E0888380E0DF91B0
:10C10000CF910895CF93DF93EC01BEDF1B82DF91C7
:10C11000CF910895CF92DF92EF92FF921F93CF932A
:10C12000DF93109299128091F312882319F080EF17
:10C1300092E1E8DF109267141092641485E3809313
:10C1400063140E94FB4DEB01A895809163140E943B
:10C1500039A883E694E10E94F74D2398229A219A08
:10C16000209A289A85E08093651482E58CBD1DBCD9
:10C170001AE08FEF0E94D5481150D9F720E030E047
:10C18000A90160E083E694E10E941F4E182F80937E
:10C190006614813049F00E94FB4D6C1B7D0B613DA4
:10C1A000774060F381E054C02AEA31E040E050E09B
:10C1B00068E083E694E10E941F4E82FF03C0109363
:10C1C00067140EC014E00E94DA4880936614115080
:10C1D000D1F78A3A11F082E03BC082E08093671485
:10C1E00080916714823031F4C12CD12CE12C80E491
:10C1F000F82E03C0C12CD12C760120E030E0A9013B
:10C2000067E383E694E10E941F4EA701960169E26D
:10C2100083E694E10E941F4E80936614882349F0C0
:10C220000E94FB4D6C1B7D0B613D774030F38AE033
:10C230000FC080916714823011F520E030E0A90131
:10C240006AE383E694E10E941F4E882351F088E060
:10C250008093641483E694E10E94F74DE3EEF0E5E9
:10C260001AC00E94DA48807C803C19F483E08093F5
:10C2700067140E94DA480E94DA480E94DA4883E68E
:10C2800094E10E94F74D1092651481E00E9463AA28
:10C29000811132C015C08491EF012196882321F0CD
:10C2A0000E94E148FE01F7CFE5E7FAE08491EF0153
:10C2B0002196882309F457C00E94E148FE01F6CF79
:10C2C00080E00E9463AA811117C0ECEAF0E5849136
:10C2D000EF012196882321F00E94E148FE01F7CF6B
:10C2E000E1E6FAE08491EF012196882309F43BC04E
:10C2F0000E94E148FE01F6CF68E674E180EF92E12A
:10C300000E944886811116C0ECEAF0E58491EF01A5
:10C310002196882321F00E94E148FE01F7CFE0E555
:10C32000FAE08491EF0121968823E9F00E94E14828
:10C33000FE01F7CF81E080939912E3EEF0E584915E
:10C34000EF012196882321F00E94E148FE01F7CFFA
:10C35000E4E4FAE08491EF012196882321F00E9421
:10C36000E148FE01F7CF8BE1E0EFF2E1A1E1B3E1BB
:10C3700001900D928A95E1F78091EE129091EF1263
:10C380009093101380930F138CEE92E190930C1303
:10C3900080930B13DF91CF911F91FF90EF90DF906F
:10C3A000CF900895FC0123812111ACCE08952FE494
:10C3B00033E0FC01318320830496F4CF2F923F9227
:10C3C0004F925F926F927F928F929F92AF92BF92A5
:10C3D000CF92DF92EF92FF920F931F93CF93DF9351
:10C3E000CDB7DEB72B970FB6F894DEBF0FBECDBF2B
:10C3F0009E838D83DC0159962D903C905A97F101D4
:10C400004184528463847484FFEF4F1A5F0A6F0A79
:10C410007F0A1496CD90DD90ED90FC901797C11493
:10C42000D104E104F10439F02FEFC21AD20AE20A72
:10C43000F20A1B8607C0D101CD90DD90ED90FC90F3
:10C44000B1E0BB87460157011F82188619861A86FC
:10C45000F10181859285A385B4852F813885498531
:10C460005A85281739074A075B0708F08DC04C1416
:10C470005D046E047F0450F492E0C92ED12CE12CAF
:10C48000F12C22E0822E912CA12CB12C9E012F5F49
:10C490003F4FB701A601C1010E94D683882309F44A
:10C4A00073C089819A81AB81BC81892B8A2B8B2BAC
:10C4B00041F0460157013FEF831A930AA30AB30ADA
:10C4C00005C0C814D904EA04FB0489F08F8198855B
:10C4D000A985BA850196A11DB11D8F839887A9876B
:10C4E000BA879FEFC91AD90AE90AF90AB1CF0FEF43
:10C4F0001FEF2FEF3FE0B501A401C1010E94998613
:10C50000F82E882309F440C0ED81FE8144815581D5
:10C5100066817781411551056105710539F09501F5
:10C520008401C1010E949986882371F1AD81BE8189
:10C5300014968D929D92AD92BC921797BB85BB23AA
:10C5400051F0D501C4010196A11DB11DF1018083F7
:10C550009183A283B383ED81FE8185899689A78922
:10C56000B08D892B8A2B8B2B81F4AD81BE815596A2
:10C570008D929D92AD92BC92589711968C91119785
:10C58000806811968C9301C0F12C8F2D2B960FB6DD
:10C59000F894DEBF0FBECDBFDF91CF911F910F91F9
:10C5A000FF90EF90DF90CF90BF90AF909F908F90D3
:10C5B0007F906F905F904F903F902F900895CF9213
:10C5C000DF92EF92FF920F931F93CF93DF938C0133
:10C5D000EB016A0179010E94EB5523E02093A80248
:10C5E0001093B8060093B706D093B606C093B5066D
:10C5F000A601662757FD6095762F4093B1065093AC
:10C60000B2066093B3067093B406C701AA2797FDDC
:10C61000A095BA2F841B950BA60BB70B8093AD0684
:10C620009093AE06A093AF06B093B006888199812F
:10C63000AA2797FDA095BA2F841B950BA60BB70BC5
:10C640008093B7119093B811A093B911B093BA1118
:10C6500083EA9BEC9093770280937602DF91CF91EF
:10C660001F910F91FF90EF90DF90CF9008959091E0
:10C670009F06891781F080939F06811108C00E9450
:10C680007B478FEE96E00E94A1520C946D4C8EEF8A
:10C690009EE00C94A152089580E0E9DF80E090E0F4
:10C6A000A0E8BFE38093061290930712A0930812AC
:10C6B000B093091210920A1210920B1210920C12DF
:10C6C00010920D1210920E1210920F121092101260
:10C6D0001092111210921212109213121092141240
:10C6E000109215128093161290931712A09318129D
:10C6F000B093191210921A1210921B1210921C125F
:10C7000010921D1210921E1210921F1210922012DF
:10C7100010922112109222121092231210922412BF
:10C72000109225128093261290932712A09328121C
:10C73000B093291208951F93CF93DF9386E50E944B
:10C74000784B882321F087E29AE00E94A77C83E55A
:10C750000E94784B882321F00E94E349C82F01C032
:10C76000C0E083E50E94784B882311F08C2F7FDF97
:10C7700010919F06C11103C0E3EEF0E518C011113E
:10C78000FBCFECEAF0E58491EF012196882321F0BC
:10C790000E94E148FE01F7CFE8E0FAE08491EF0162
:10C7A0002196882349F30E94E148FE01F7CF849146
:10C7B000EF012196882321F00E94E148FE01F7CF86
:10C7C000112319F063E273E002C067E273E08AEFBD
:10C7D00099E00E940E8C8AE0DF91CF911F910C941A
:10C7E000E1488F929F92AF92BF92CF92DF92EF92E9
:10C7F000FF920F931F93CF93DF93882EB62EA42E14
:10C80000F22EE801242F220F220F220F0F2D462F88
:10C81000682F8CEC91E10E94D94C882351F10B2DAB
:10C820000F0DCA2CD12CB01621F17E019A2C182D97
:10C830009920D9F0F70184916091CE117091CF11B8
:10C840001093E811B092E9111092EB118093EA1164
:10C8500028EE31E14BE38CEC91E10E94FB4CFFEFC1
:10C86000EF1AFF0A9A94185FE3CFCC0DDD1DB39445
:10C87000DACFDF91CF911F910F91FF90EF90DF9072
:10C88000CF90BF90AF909F908F90089590914E124F
:10C8900080914F12981721F080E00F94F805F6CFA1
:10C8A00008952F923F924F925F926F927F928F9254
:10C8B0009F92AF92BF92CF92DF92EF92FF920F932F
:10C8C0001F93CF93DF9300D01F92CDB7DEB77B01CC
:10C8D0008A0119012091A5043091A6044091A70472
:10C8E0005091A804DC016D917D918D919C910F94E4
:10C8F000551A0F9485204B015C0160933E12709392
:10C900003F1280934012909341122091A9043091DC
:10C91000AA044091AB045091AC04F701608171818D
:10C92000828193810F94551A0F9485206B017C01AD
:10C930006093421270934312809344129093451275
:10C940002091AD043091AE044091AF045091B004F9
:10C95000D8016D917D918D919C910F94551A0F94F2
:10C9600085202B013C0160934612709347128093FF
:10C970004812909349122091B1043091B204409131
:10C98000B3045091B404F10160817181828193817B
:10C990000F94551A0F94852060934A1270934B128E
:10C9A00080934C1290934D1269837A838B839C837E
:10C9B0006DDF2FB7F8948092660E9092670EA0926A
:10C9C000680EB092690EC0926A0ED0926B0EE09221
:10C9D0006C0EF0926D0E40926E0E50926F0E609241
:10C9E000700E7092710E69817A818B819C81609347
:10C9F000720E7093730E8093740E9093750E2FBF0A
:10CA000010922A1210922B1210922C1210922D12A8
:10CA100080E1EEE2F2E1DF011D928A95E9F70F90E5
:10CA20000F900F900F90DF91CF911F910F91FF907A
:10CA3000EF90DF90CF90BF90AF909F908F907F90BE
:10CA40006F905F904F903F902F900895EF92FF92DC
:10CA50000F931F93CF93DF93CDB7DEB72C970FB60D
:10CA6000F894DEBF0FBECDBF05EA14E083E1E82EE7
:10CA70008FE0F82EF80121913191419151918F0170
:10CA800060E070E080E89FE30F94301FF70161934E
:10CA90007193819391937F01F4E0053B1F0751F758
:10CAA0008091FE0E9091FF0EA091000FB091010FAA
:10CAB00089839A83AB83BC838091020F9091030F8B
:10CAC000A091040FB091050F8D839E83AF83B8872B
:10CAD0008091060F9091070FA091080FB091090F58
:10CAE00089879A87AB87BC87AE01475F5F4FBE01DE
:10CAF0006B5F7F4FCE0101960E9412542AE03FE007
:10CB0000AE01475F5F4FBE016B5F7F4FCE01019665
:10CB1000C8DE0E946B482C960FB6F894DEBF0FBE9D
:10CB2000CDBFDF91CF911F910F91FF90EF900895AE
:10CB30000E946B488BDF0E942F4A80E00E94DD4AF2
:10CB400081E00E94DD4A82E00E94DD4A80E00E948E
:10CB50001C7B0C9492CF0F931F93CF93DF93CDB791
:10CB6000DEB72C970FB6F894DEBF0FBECDBF05EA37
:10CB700014E065E874E047E951E120E030E0F901B4
:10CB8000E35EF44F85919591A591B491F80181935D
:10CB90009193A193B1938F01F901E35FF44F8591D4
:10CBA0009591A591B491FB0181939193A193B19338
:10CBB000BF01F901E350F54F85919591A591B4918D
:10CBC000FA0181939193A193B193AF012C5F3F4FF1
:10CBD00020313105A1F680E090E0AAEFB4E4809323
:10CBE000AF119093B011A093B111B093B21140E086
:10CBF00050E86BE375E44093AB115093AC11609334
:10CC0000AD117093AE118093A7119093A811A093CA
:10CC1000A911B093AA111092A7061092A80610921B
:10CC2000A9061092AA0680E29EE4A0E0B0E08093FC
:10CC30008B0590938C05A0938D05B0938E05109273
:10CC4000A3061092A4061092A5061092A60680E0F4
:10CC500090E0A0E4B1E48093950490939604A093AF
:10CC60009704B09398048093990490939A04A093A6
:10CC70009B04B0939C048DEC9CECACECBEE38093E5
:10CC80009D0490939E04A0939F04B093A00480E021
:10CC900090E0A0E2B1E48093A1049093A204A09359
:10CCA000A304B093A4041CE0E2EFFEE0DF01812FB7
:10CCB0001D928A95E9F7F0DC89E891E4A0EBBFEBDF
:10CCC0008093E2069093E306A093E406B093E50612
:10CCD00084EB90E09093C1048093C00480EF90E0D7
:10CCE0009093C3048093C20486E490E09093B904C7
:10CCF0008093B8048EE690E09093BB048093BA04CE
:10CD00001092BD041092BC041092BF041092BE0495
:10CD100087ED93EAAEE9B1E48093DC0E9093DD0EEB
:10CD2000A093DE0EB093DF0E80E898E5A0E8BEE3A6
:10CD30008093D80E9093D90EA093DA0EB093DB0EA9
:10CD400081E09DECA3ECB3E48093D40E9093D50ED8
:10CD5000A093D60EB093D70E8DE39AE2A0ECB3E485
:10CD60008093D2049093D304A093D404B093D504B9
:10CD700087E790E3ADE3B1E48093CE049093CF04D2
:10CD8000A093D004B093D10489ED9CE2A3E4B5E470
:10CD90008093CA049093CB04A093CC04B093CD04A9
:10CDA0001092C90480E090E0A0E4B0E48093C40451
:10CDB0009093C504A093C604B093C70481E0809308
:10CDC000ED0E8093B704E9EAF2E0DE0111960190DE
:10CDD0000D921A95E1F713E01150C8F0A4E01A9FE4
:10CDE00090011124E1E0F0E0EC0FFD1FE20FF31FD2
:10CDF0006081718182819381F901E152FB4F6083EF
:10CE0000718382839383812F0E9452CFE5CF90DE7E
:10CE1000E3EEF0E584918F010F5F1F4F882321F02F
:10CE20000E94E148F801F6CFEAEDFAE084918F0123
:10CE30000F5F1F4F882321F00E94E148F801F6CFD1
:10CE40002C960FB6F894DEBF0FBECDBFDF91CF9109
:10CE50001F910F9108952F923F924F925F926F9280
:10CE60007F928F929F92AF92BF92CF92DF92EF927A
:10CE7000FF920F931F93CF93DF93CDB7DEB7C455C7
:10CE8000D1090FB6F894DEBF0FBECDBF2DB73EB7A8
:10CE900063963FAF2EAF639729961FAE1EAE2997BC
:10CEA00084E690E027969FAF8EAF27979E01295B7F
:10CEB0003F4F44E050E0BE01635C7F4FCE018B5B8F
:10CEC0009F4F0E94B9899E01295B3F4F42E050E08D
:10CED000BE016D5B7F4FCE018B5B9F4F0E94B98976
:10CEE00043E050E0BE01635C7F4F8BE393E00F941F
:10CEF000A121892B99F18DAD863519F08FE38DAF86
:10CF00001EAEE3EEF0E584918F010F5F1F4F882383
:10CF100021F00E94E148F801F6CFE6EAFBE08491B7
:10CF20008F010F5F1F4F882321F00E94E148F80115
:10CF3000F6CFBE01635C7F4F8DE99BE00E940E8CB3
:10CF4000EFE8FBE084918F010F5F1F4F882321F0F2
:10CF50000E94E148F801F6CFFEDD3EC46DB67EB614
:10CF600019AE1AAE1BAE1CAE29961FAE1EAE299787
:10CF70009E01295B3F4F41E050E0BE01615B7F4F66
:10CF8000CE018B5B9F4F0E94B98980E1E5EBF2E017
:10CF9000DE01919601900D928A95E1F780E1E5EC32
:10CFA000F2E0DE01519601900D928A95E1F780E161
:10CFB000E5EDF2E09E012F5F3F4F7901D90101902D
:10CFC0000D928A95E1F76096CFAC6097D12C33E053
:10CFD000C30ED11CCC0CDD1CCC0CDD1C8DB79EB758
:10CFE0008C199D090FB6F8949EBF0FBE8DBFEDB78B
:10CFF000FEB731964F012DB73EB72C193D090FB63C
:10D00000F8943EBF0FBE2DBF8DB79EB701965C0151
:10D01000EDB7FEB7EC19FD090FB6F894FEBF0FBED1
:10D02000EDBF0DB71EB70F5F1F4F9E01295B3F4F2E
:10D03000A601B401CE018B5B9F4F0E94B9899E016E
:10D04000295B3F4FA601B501CE018B5B9F4F0E942C
:10D05000B9899E01295B3F4FA601B801CE018B5BC8
:10D060009F4F0E94B98960964FAD609750E04E5F28
:10D070005F4F27E931E165963FAF2EAF659765E8D1
:10D0800074E0A5EAB4E080E090E020E030E04217F0
:10D09000530714F0640105C0F1E2CF2ED12CCC0E61
:10D0A000DD1EC80ED91EF6012080318042805380DB
:10D0B0002D923D924D925D924217530714F06501F7
:10D0C00005C0E1E1CE2ED12CCC0EDD1EC80ED91E3E
:10D0D000F6012080318042805380FB012192319201
:10D0E00041925192BF014217530714F0680101C0E9
:10D0F0006701C80ED91EF60120803180428053801E
:10D100006596EEADFFAD65972192319241925192B5
:10D110006596FFAFEEAF65972F5F3F4F04962430C3
:10D12000310509F0B4CF9E01295B3F4F44E050E048
:10D130006FEA71E1CE018B5B9F4F0E94B9899E011E
:10D14000295B3F4F44E050E06BEA71E1CE018B5B1D
:10D150009F4F0E94B9899E01295B3F4F44E050E0F8
:10D1600067EA71E1CE018B5B9F4F0E94B9899E01F6
:10D17000295B3F4F44E050E067EA76E0CE018B5BED
:10D180009F4F0E94B9899E01295B3F4F44E050E0C8
:10D1900063EA76E0CE018B5B9F4F0E94B9899E01C6
:10D1A000295B3F4F44E050E06BE875E0CE018B5BBC
:10D1B0009F4F0E94B9899E01295B3F4F40E150E09B
:10D1C00065E974E0CE018B5B9F4F0E94B9899E0197
:10D1D000295B3F4F4CE050E062EF7EE0CE018B5B7D
:10D1E0009F4F0E94B9899E01295B3F4F44E050E068
:10D1F000BE01675C7F4FCE018B5B9F4F0E94B98958
:10D200009E01295B3F4F41E050E0BE01625B7F4FD2
:10D21000CE018B5B9F4F0E94B9899E01295B3F4FD6
:10D2200044E050E0BE01675C7F4FCE018B5B9F4FB7
:10D230000E94B9899E01295B3F4F41E050E0BE0149
:10D24000635B7F4FCE018B5B9F4F0E94B9899E012C
:10D25000295B3F4F41E050E0BE01645B7F4FCE0150
:10D260008B5B9F4F0E94B9892E96EFAC2E972D961F
:10D270008FAD2D97E89E7001112400E010E00E158F
:10D280001F0581F09E01295B3F4F44E050E0BE0145
:10D29000675C7F4FCE018B5B9F4F0E94B9890F5F08
:10D2A0001F4FEDCF29960EAD1FAD299727968EAD56
:10D2B0009FAD279790936302809362029E01295B42
:10D2C0003F4F44E050E062EE76E0CE018B5B9F4F33
:10D2D0000E94B98929961FAF0EAF29979E01295B3D
:10D2E0003F4F44E250E066E072E1CE018B5B9F4F1E
:10D2F0000E94B9899E01295B3F4F41E050E0BE0189
:10D30000655B7F4FCE018B5B9F4F0E94B9899E0169
:10D31000295B3F4F41E050E0BE01665B7F4FCE018D
:10D320008B5B9F4F0E94B9899E01295B3F4F44E070
:10D3300050E0BE016B5C7F4FCE018B5B9F4F0E9424
:10D34000B9899E01295B3F4F44E050E0BE016F5C0C
:10D350007F4FCE018B5B9F4F0E94B9892C96EFAC1B
:10D360002C972B968FAD2B97E89E7001112400E02F
:10D3700010E09E01295B3F4F0E151F0569F044E048
:10D3800050E0BE01675C7F4FCE018B5B9F4F0E94D8
:10D39000B9890F5F1F4FEDCF41E050E0BE01605BE8
:10D3A0007F4FCE018B5B9F4F0E94B9899E01295B05
:10D3B0003F4F44E050E0BE01675C7F4FCE018B5B86
:10D3C0009F4F0E94B9899E01295B3F4F41E050E089
:10D3D000BE01675B7F4FCE018B5B9F4F0E94B98977
:10D3E00019AE1AAE1BAE1CAE1DE011509E01295B9A
:10D3F0003F4F44E050E0112349F0BE01675C7F4F8E
:10D40000CE018B5B9F4F0E94B989EFCF60EC74E037
:10D41000CE018B5B9F4F0E94B9899E01295B3F4FD4
:10D4200044E050E068EB74E0CE018B5B9F4F0E94BC
:10D43000B9899E01295B3F4F44E050E06CEB74E0FA
:10D44000CE018B5B9F4F0E94B9899E01295B3F4FA4
:10D4500044E050E0BE01675C7F4FCE018B5B9F4F85
:10D460000E94B989112311F004E03CC0C9ACDAACC8
:10D47000EBACFCAC20E030E84BE355E4C701B6016F
:10D480000F94F019882381F3C092DC0ED092DD0E48
:10D49000E092DE0EF092DF0E9E01295B3F4F44E0EA
:10D4A00050E068ED7EE0CE018B5B9F4F0E94B98912
:10D4B0009E01295B3F4F44E050E064ED7EE0CE01E9
:10D4C0008B5B9F4F0E94B9899E01295B3F4F44E0CF
:10D4D00050E0BE01675C7F4FCE018B5B9F4F0E9487
:10D4E000B98910C0015071F09E01295B3F4F44E0A3
:10D4F00050E0BE01675C7F4FCE018B5B9F4F0E9467
:10D50000B989F0CF1F5F153009F09FCF9E01295BCD
:10D510003F4F42E050E0BE016F5B7F4FCE018B5B1F
:10D520009F4F0E94B9899E01295B3F4F44E050E024
:10D53000BE01675C7F4FCE018B5B9F4F0E94B98914
:10D54000C9ACDAACEBACFCAC20E030E84BE355E422
:10D55000C701B6010F94F019882301F1C092D204DB
:10D56000D092D304E092D404F092D5049E01295BBA
:10D570003F4F44E050E06EEC74E0CE018B5B9F4F78
:10D580000E94B9899E01295B3F4F44E050E06AEC5C
:10D5900074E0CE018B5B9F4F0E94B9899E01295B8D
:10D5A0003F4F42E050E0BE016B5C7F4FCE018B5B92
:10D5B0009F4F0E94B9899E01295B3F4F41E050E097
:10D5C000BE01605B7F4FCE018B5B9F4F0E94B9898C
:10D5D00019E011509E01295B3F4F112359F044E09F
:10D5E00050E0BE01675C7F4FCE018B5B9F4F0E9476
:10D5F000B989EFCF41E050E069EC74E0CE018B5B7C
:10D600009F4F0E94B9899E01295B3F4F44E050E043
:10D61000BE01675C7F4FCE018B5B9F4F0E94B98933
:10D6200011110CC089AD9AADABADBCAD8093C404F3
:10D630009093C504A093C604B093C7041F5F153030
:10D6400011F71BE09E01295B3F4F42E050E0BE0115
:10D650006F5C7F4FCE018B5B9F4F0E94B989115049
:10D6600089F79E01295B3F4F44E050E0BE01675CB3
:10D670007F4FCE018B5B9F4F0E94B9899E01295B32
:10D680003F4F44E050E0BE01675C7F4FCE018B5BB3
:10D690009F4F0E94B98913E0115088F0F4E01F9F5A
:10D6A000B001112461527B4F9E01295B3F4F44E042
:10D6B00050E0CE018B5B9F4F0E94B989EDCF299638
:10D6C0002EAD3FAD299725968EAD9FAD2597281796
:10D6D000390709F039C02CDAE3EEF0E584918F01C7
:10D6E0000F5F1F4F811103C00BE313E004C00E94C2
:10D6F000E148F801F3CFF80181918F01882319F0F7
:10D700000E94E148F8CF27966EAD7FAD279764560B
:10D71000710982E79BE00E9420A829964EAD5FAD7B
:10D72000299760E070E085E69BE00E9417E0E2E662
:10D73000FBE084918F010F5F1F4F882309F447C0DE
:10D740000E94E148F801F5CFECEAF0E584918F0101
:10D750000F5F1F4F882321F00E94E148F801F6CFA8
:10D76000E2E4FBE084918F010F5F1F4F882321F0DB
:10D770000E94E148F801F6CF25966EAD7FAD259762
:10D7800080E090E04AE00E949FA6EDE3FBE08491F8
:10D790008F010F5F1F4F882321F00E94E148F8019D
:10D7A000F6CF29966EAD7FAD299780E090E04AE0F4
:10D7B0000E949FA6EDE2FBE084918F010F5F1F4F57
:10D7C000882321F00E94E148F801F6CFC4D90FB6B2
:10D7D000F8947EBE0FBE6DBE80E00E94E77C909103
:10D7E0008A0581E0892763962EAD3FAD63970FB61A
:10D7F000F8943EBF0FBE2DBFCC5ADF4F0FB6F89442
:10D80000DEBF0FBECDBFDF91CF911F910F91FF9073
:10D81000EF90DF90CF90BF90AF909F908F907F90D0
:10D820006F905F904F903F902F9008950F931F93AC
:10D83000CF93DF93CDB7DEB72C970FB6F894DEBF4A
:10D840000FBECDBF8091060F9091070FA091080FDA
:10D85000B091090F4091020F5091030F6091040F96
:10D860007091050F0091FE0E1091FF0E2091000F98
:10D870003091010F09831A832B833C834D835E8390
:10D880006F83788789879A87AB87BC87AE01475FAC
:10D890005F4FBE016B5F7F4FCE0101960E94125415
:10D8A0002AE03FE0AE01475F5F4FBE016B5F7F4FF5
:10D8B000CE0101960E9451642C960FB6F894DEBFFB
:10D8C0000FBECDBFDF91CF911F910F9108952F9281
:10D8D0003F924F925F926F927F928F929F92AF9200
:10D8E000BF92CF92DF92EF92FF920F931F93CF934D
:10D8F000DF9300D01F921F92CDB7DEB7B2EF8B2E11
:10D90000BEE09B2E1EEFA12E1EE0B12E0CE9202EB4
:10D9100006E0302E00E010E0822D80958D83F1012D
:10D9200081911F01882309F499C0F501408051803D
:10D9300062807380F801EA5AFD4F20813181428173
:10D940005381F801E258FA4F60817181828193819D
:10D950000F94541E20E030E040E05FE30F94551A2E
:10D960009B01AC01C301B2010F947A20181644F454
:10D97000F801EF5FFE4EC590D590E590F49003C09E
:10D98000C12CD12C7601F801E05BFB4F2081318165
:10D9900042815381C301B2010F94531E9B01AC011C
:10D9A000C701B6010F94531E6B017C0120E030E0EB
:10D9B00040EA51EC0F947A2087FD28C020E030E047
:10D9C00040EA51E4C701B6010F94F0191816F4F0BB
:10D9D000F4012081318142815381C701B6010F9446
:10D9E000531E9B01AC01C301B2010F94541EF501FB
:10D9F0006083718382839383F401C082D182E28247
:10DA0000F3828D81820D0E94DD4A28C0ECEAF0E5A8
:10DA100084918F010F5F1F4F882321F00E94E148FE
:10DA2000F801F6CFECEBFAE084918F010F5F1F4F06
:10DA3000882321F00E94E148F801F6CF61E08EEAE8
:10DA40009AE00E9462550E94D95688E290E09C8339
:10DA50008B8388EC90E09A83898329C0F4E08F0E51
:10DA6000911C0C5F1F4F84E0A80EB11C0C301105F7
:10DA700009F055CFDBDE0E94E87B60E08EE99AE09A
:10DA80000E94625583E992E09C838B8304E610E058
:10DA90001A830983BE016D5F7F4FCE0101960F94FB
:10DAA000AC0D8AEB92E09C838B831A830983BE01C1
:10DAB0006D5F7F4FCE0101960F94AC0D0F900F90CC
:10DAC0000F900F900F90DF91CF911F910F91FF90CA
:10DAD000EF90DF90CF90BF90AF909F908F907F900E
:10DAE0006F905F904F903F902F9008954F925F926C
:10DAF0006F927F928F929F92AF92BF92CF92DF925E
:10DB0000EF92FF920F931F93CF93DF93CDB7DEB7C2
:10DB10002E970FB6F894DEBF0FBECDBF1091540202
:10DB20001F3FE9F00E94FB4DC0906505D09066054F
:10DB3000E0906705F09068056C197D098E099F09D2
:10DB400097FD0DC020914F1280914E1230E090E071
:10DB500001968F7099272817390709F028C20E946B
:10DB6000DE5480917D0582FF3EC080917C0581114D
:10DB70003CC091E090937C0580910C0989278093AB
:10DB8000B31110920C0983E08093A80210927D05D6
:10DB90000E94FB4D6C507E4F8F4F9F4F60936905E5
:10DBA00070936A0580936B0590936C0588E893E108
:10DBB0009E878D8782E090E09A838983BE01635FB0
:10DBC0007F4FCE0101960F94AC0D16E0115069F015
:10DBD00080E592E10E948F4E62E070E080E090E08C
:10DBE0000E94644DF3CF10927C05109103011095B3
:10DBF0001170912F917080917B051817A9F09923CE
:10DC000009F428C20E948A6080917B05823029F045
:10DC100060E080E99AE00E94625510937B0583E002
:10DC20008093A8020E94F3CE0E94FB4D6B017C0101
:10DC30008091770590917805A0917905B0917A054A
:10DC4000A7019601281B390B4A0B5B0B57FF05C038
:10DC500080917605882309F449C2D701C6018C5901
:10DC60009F4FAF4FBF4F8093770590937805A09358
:10DC70007905B0937A058091750518162CF480917A
:10DC80007505823074F408C08091750599278195D7
:10DC90000CF4909502972CF48091B31181119DC0E2
:10DCA000ADC08091BB11882309F470C080917505C7
:10DCB00018165CF480917505992787FD909597FD5E
:10DCC0000196BC01759567950DC0809175059927E2
:10DCD00087FD909597FD01969595879566277727FF
:10DCE000681B790B8090921190909311A0909411E1
:10DCF000B090951181149104A104B10429F421E09C
:10DD000030E040E050E039C0882777FD8095982FBB
:10DD10000F94F6192B013C01C701B6016819790966
:10DD20008A099B090F94F4199B01AC01C301B2014C
:10DD30000F94301F20E030E04AE754E40F94551A66
:10DD40004B015C0120E030E040E253E40F947A2084
:10DD500087FF0FC020E030E046E952E4C501B4017E
:10DD60000F947A2087FDCBCF2AE030E040E050E0EE
:10DD700004C024E630E040E050E0C0929211D0921E
:10DD80009311E0929411F092951104C021E030E0DB
:10DD900040E050E0A0917505BB27A7FDB0950F941A
:10DDA0003E1E22E030E040E050E00F94181E8091CB
:10DDB000B7119091B811A091B911B091BA11820F19
:10DDC000931FA41FB51F8093B7119093B811A09310
:10DDD000B911B093BA1110927505D701C6018856D2
:10DDE000954CAF4FBF4F8093710590937205A093F0
:10DDF0007305B093740581E08093A80220917602A8
:10DE00003091770248E9293D340749F48091550261
:10DE10009FEF980F90935502882309F426C1295744
:10DE2000334779F480916E0590916D05891748F418
:10DE3000909155022FEF290F20935502992309F451
:10DE400024C12FB7F8948091920990919309A091E1
:10DE50009409B09195092FBF4091A802411105C0C6
:10DE600020917605222309F465C03AE0B695A7957E
:10DE7000979587953A95D1F7009721E0A207B105CC
:10DE800020F08FEF9FEFA0E0B0E096958795009788
:10DE900041F020916F05309170052817390708F07F
:10DEA00049C080917605811111C0423050F0443054
:10DEB00028F0443031F41092A80203C081E080932E
:10DEC000A8020E94D1A581E08093760584E00E949B
:10DED000AAA981E08093EC11E0917602F09177029B
:10DEE00019951092B31180917605882351F00E9404
:10DEF0001CA991E0811101C090E0909376059111E9
:10DF0000DCC080906F0590907005A12CB12C0E9410
:10DF1000FB4D6C197D098E099F0986169706A80688
:10DF2000B90640F40E94FB4D6C197D097093700591
:10DF300060936F058091760290917702895D984990
:10DF400021F08091D804882379F048E9C40E4AE38F
:10DF5000D41EE11CF11CC0927105D0927205E092B2
:10DF60007305F09274050FC0809171059091720550
:10DF7000A0917305B0917405C81AD90AEA0AFB0A80
:10DF8000F7FE0E94D956809176058111AFC080912D
:10DF9000A802813049F008F4A9C0843008F0A6C076
:10DFA00081E08093A802A2C01092A8029FC054E012
:10DFB0001502F0011124E55DFC4F20E030E040E760
:10DFC00052E460817181828193810F94301F4B01F3
:10DFD0005C018091FE0E9091FF0EA091000FB09118
:10DFE000010F89839A83AB83BC838091020F909148
:10DFF000030FA091040FB091050F8D839E83AF8313
:10E00000B8878091060F9091070FA091080FB091EB
:10E01000090F89879A87AB87BC87AE01475F5F4F3F
:10E02000BE016B5F7F4FCE0101960E941254C12C3E
:10E03000850174012AE03FE0AE01475F5F4FBE01FA
:10E040006B5F7F4FCE0101960E946BF48FEF809340
:10E05000540285CD1092981210929912823009F4D0
:10E06000DCCD60E083E89AE0D6CD8CE08093550269
:10E0700080916F0590917005019790937005809342
:10E080006F0581E08093A802CACE96E09093550276
:10E0900091E09093A8028F5F80936E05D701C6012F
:10E0A0008856954CAF4FBF4F809371059093720582
:10E0B000A0937305B0937405C4CE80906F059090C3
:10E0C0007005A12CB12C0E94FB4D6C197D098E09A5
:10E0D0009F0986169706A806B90640F40E94FB4DD4
:10E0E0006C197D097093700560936F052E960FB6BD
:10E0F000F894DEBF0FBECDBFDF91CF911F910F917E
:10E10000FF90EF90DF90CF90BF90AF909F908F9057
:10E110007F906F905F904F900895CF92EF92FF9213
:10E120000F931F93CF93DF93CDB7DEB72C970FB626
:10E13000F894DEBF0FBECDBFC090EC048091060FF7
:10E140009091070FA091080FB091090F4091020F15
:10E150005091030F6091040F7091050F0091FE0E16
:10E160001091FF0E2091000F3091010F09831A8347
:10E170002B833C834D835E836F83788789879A875F
:10E18000AB87BC87AE01475F5F4FBE016B5F7F4FC0
:10E19000CE0101960E941254E0900A02F0900B0208
:10E1A00000910C0210910D022AE03FE0AE01475FA2
:10E1B0005F4FBE016B5F7F4FCE0101960E946BF4F3
:10E1C0002C960FB6F894DEBF0FBECDBFDF91CF9176
:10E1D0001F910F91FF90EF90CF900895CF92DF9213
:10E1E000FF920F931F93CF93DF931F921F92CDB790
:10E1F000DEB76901DB0112960D911C911397423332
:10E2000009F471C0B8F4453109F47AC0473109F412
:10E210008BC0443109F0A1C0D80115962C911597F7
:10E220001696ED91FC911797CF01820F911D820FE9
:10E23000911D5EC0463409F487C0473409F488C094
:10E240004B3309F08AC0F90181819381913029F023
:10E25000933031F4282F885004C028E0280F01C0E3
:10E26000282F31E0D80113964C91481708F430E07C
:10E2700051E0F8014281241708F450E041E02817EA
:10E2800008F040E0832F842B85233423832B09F46B
:10E2900064C0D6011296FC90913039F070F0923043
:10E2A00039F0933041F020E001C021E030E007C0B8
:10E2B00020E03FEF04C02FEFF9CF20E031E0F7FE80
:10E2C00008C0B601C8012A8339830E94984C39815D
:10E2D0002A81F6018081830F80838181820F81836F
:10E2E000FF0C69F73AC0B901C8010E94984C35C0CB
:10E2F0001192E817F907E1F7C8010E94C34C2DC03D
:10E30000C8010E94AD4C882351F1F8012581068097
:10E31000F781E02DCF01820F911D820F911D119287
:10E32000E817F907E1F719C0D9011C92F8018281B9
:10E3300011968C9311978581815012968C93129728
:10E34000838113968C9309C0D80115968C9103C0D4
:10E35000D80111968C91F601808381E001C080E0A4
:10E360000F900F90DF91CF911F910F91FF90DF9051
:10E37000CF9008956F927F928F929F92AF92BF92AB
:10E38000CF92DF92EF92FF920F931F93CF93DF9381
:10E390005C017B01942E69018AE0481709F471C081
:10E3A000A5E14A134AC0DB011296ED91FC91139747
:10E3B0008280C681D7815D9A0E94CA4C80EE782EF9
:10E3C000780C90E1692E680C88EF0E9401570E943A
:10E3D000CA4CBFE1B81508F443C0882D8077806827
:10E3E0000E940157882D8295807F0E9401570E94CC
:10E3F000CA4C80E80E94015780E00E9401570E94A9
:10E40000CA4C8AEF0E9401570E94CA4C8E01005FDD
:10E410001F4F8881807F0E94015789918295807F5C
:10E420000E9401570C171D07A1F7E8010E94CA4C72
:10E43000839473948610C8CF5D989601492DB701D7
:10E44000C501DF91CF911F910F91FF90EF90DF9069
:10E45000CF90BF90AF909F908F907F906F90BECEE7
:10E46000872D807780680E940157872D8295807F55
:10E470000E9401570E94CA4C80E80E94015780E820
:10E48000BCCF559A5D98539A5B98529A5A9A5D9A66
:10E490000E94CA4C88E790E00E94CF4C88EF0E940F
:10E4A00001570E94CA4C80E00E94015780E80E94F8
:10E4B00001570E94CA4C80E00E94015780E10E94EF
:10E4C00001570E94CA4C8FE090E00E94CF4C80E33D
:10E4D0000E94015780EE0E9401570E94CA4CD0E072
:10E4E0008D2F807780680E9401578D2F8295807FC5
:10E4F0000E9401570E94CA4C80E80E94015780E0A8
:10E500000E9401570E94CA4C8AEF0E9401570E9444
:10E51000CA4CC0E280E00E94015780E00E9401578F
:10E520000E94CA4CC150B1F788EF0E9401570E9467
:10E53000CA4CDF5FD032A1F680E00E94015780EC28
:10E540000E9401570E94CA4C5D9877CF109291119A
:10E55000109290110F94DA090C94D956DF92EF9231
:10E56000FF920F931F93CF93DF93CDB7DEB76E97D4
:10E570000FB6F894DEBF0FBECDBF609190097091C9
:10E5800091096115710511F14DE150E08E010F5FA8
:10E590001F4FC8010F9461191E8EF8017F01E01A08
:10E5A000F10AD190DD2019F08AE0D812F7CFF801F6
:10E5B000EE0DFF1D108260E0C8010E945C4B8823B5
:10E5C00029F0C8010E94368C811109C081E0209198
:10E5D000900930919109232BA9F480E013C0DD202C
:10E5E00051F08FEFE81AF80A809190099091910903
:10E5F0008E0D9F1D02C080E090E090939109809362
:10E600009009E4CF6E960FB6F894DEBF0FBECDBF73
:10E61000DF91CF911F910F91FF90EF90DF900895C0
:10E6200086EB9CE0909391098093900997DF6FEFC0
:10E6300085EB9CE00C946255CF92DF92EF92FF92B3
:10E640000F931F93CF93DF93CDB7DEB7CDB6DEB672
:10E65000FC0101900020E9F7E81BF90B34962DB777
:10E660003EB72E1B3F0B0FB6F8943EBF0FBE2DBF1B
:10E670000DB71EB70F5F1F4F9F938F9386EC9CE0E3
:10E680009F938F931F930F930F948A19780134E00F
:10E69000E30EF11C0F900F900F900F900F900F90C2
:10E6A000F7018081882339F090E00F945321F7011E
:10E6B00081937F01F5CF60E0C8010E945C4B882305
:10E6C00019F0C8010E94368C82EC9CE0909391096D
:10E6D0008093900943DF0FB6F894DEBE0FBECDBE27
:10E6E000DF91CF911F910F91FF90EF90DF90CF902E
:10E6F0000895AF92BF92CF92DF92EF92FF920F9365
:10E700001F93CF93DF93CDB7DEB76F970FB6F89413
:10E71000DEBF0FBECDBF8091A802811105C08091E0
:10E72000B311882309F4ABC18DE093E190930C13EE
:10E7300080930B1381E0809344151092461510923C
:10E74000451540E050E0BA0181E193E10E9449851E
:10E7500080910B1390910C132BE1FC013496DE0198
:10E76000159601900D922A95E1F7FC018281938123
:10E770009C838B838FE493E09A83898340E050E00D
:10E78000BE016F5F7F4F8BEB93E00E946DC1CE01A6
:10E7900001960E94D761E0904515F09046151092C1
:10E7A000BB118091B7119091B811A091B911B0919E
:10E7B000BA1181309048A105B10540F01092B7110F
:10E7C0001092B8111092B9111092BA11D090B711DD
:10E7D00040918F061416DCF4842F992787FD9095BD
:10E7E00001972D2D332727FD3095281739077CF009
:10E7F000DD24DA94D40E8D2D90E0A0E0B0E080937B
:10E80000B7119093B811A093B911B093BA111092A7
:10E81000B5118091B411D81614F4D092B41180912E
:10E82000B411992787FD909504962D2D332727FD48
:10E8300030958217930724F48CEF8D0D8093B411DB
:10E84000C090B411B12C21E0E21AF108C1101BC034
:10E850008091B311811105C08091A802882399F09D
:10E8600009C0D110F9CF0E94DF568091B5118823DD
:10E8700099F305C181E0D11080E024E040EF5CE035
:10E880006B2D0E94FBA16BE972E181E193E10E9493
:10E8900088A580919B128F3209F181E0C8121CC0BB
:10E8A0008091B311811105C08091A8028823A1F045
:10E8B0000AC091E0D912F8CF0E94269F8091B5112D
:10E8C000882391F3DCC081E0D81280E020E24CEE96
:10E8D0005CE06B2D0E94FBA182E001C081E087011A
:10E8E000AA24A394AC0C0F3FFFEF1F0709F4C0C08C
:10E8F000C812BAC060E070E0C8010E9484C3909161
:10E900009A128091B311992309F492C0882309F4D3
:10E9100086C0DC1084C01D8218861C821B828FE496
:10E9200093E09A83898380911413811103C00CEEC4
:10E9300012E102C00DE013E17801E4E0EE0EF11CFB
:10E9400021E04BE952E1B701CE0105960E9475C066
:10E95000811127C0E3EEF0E584918F010F5F1F4F17
:10E96000882321F00E94E148F801F6CFE6EDFCE0B3
:10E9700084918F010F5F1F4F811103C00BE912E1DA
:10E9800004C00E94E148F801F3CFF80181918F01A2
:10E99000882319F00E94E148F8CF8AE00E94E148FC
:10E9A0002BC0809162148A30C0F491E0980F90934C
:10E9B0006214FFE18F9FC0011124845D9C4E2BE106
:10E9C000F701DC01149601900D922A95E1F7F80108
:10E9D00022813381FC01338322838BE1FE01359652
:10E9E000A1E1B3E101900D928A95E1F78B819C81C1
:10E9F0009093101380930F13CE0101960E94D7615C
:10EA00001092B7111092B8111092B9111092BA1158
:10EA100081E08093B51183E08093A80230C080919B
:10EA2000A8028823F9F081E0DC1080E041E017C003
:10EA3000811105C08091A8028823A1F00CC0DC10D0
:10EA4000F9CF8BE992E1F8DD0E94D9568091B5119A
:10EA5000882381F314C081E0DC1080E040E06B2D5E
:10EA60000E9484A18A2D01C08F5F015011093BCF04
:10EA7000B394C39425E0B212E9CE80938F066F96CB
:10EA80000FB6F894DEBF0FBECDBFDF91CF911F91BF
:10EA90000F91FF90EF90DF90CF90BF90AF900895CF
:10EAA0007F928F929F92AF92BF92CF92DF92EF921E
:10EAB000FF920F931F93CF93DF93CDB7DEB7AA9743
:10EAC0000FB6F894DEBF0FBECDBF8091EB128F93CF
:10EAD0008091EA128F938DEC9CE09F938F938E012F
:10EAE0000F5D1F4F1F930F930F948A190F900F9074
:10EAF0000F900F900F900F90D12CF80101900020F3
:10EB0000E9F73197E01BF10BDE1674F47801ED0C98
:10EB1000F11CD7FCFA94F701808190E00F94532107
:10EB2000F7018083D394E9CF40E050E0BA0180EF51
:10EB300092E10E944985912CCE0101967C0140E032
:10EB400050E0B70180EF92E10E94BEAB18168CF541
:10EB5000F70101900020E9F73197EE19FF09C12C68
:10EB6000D12C8E2E77247A947E0E872D8C198C14BE
:10EB700081F05701A80EB11C87FDBA94F501808180
:10EB800090E00F945321F5018083FFEFCF1ADF0A45
:10EB9000ECCF8A858E3799F245E050E0B801C70185
:10EBA0000F94A121892B59F6C80146DD992493942D
:10EBB000C6CF911003C08FEF9FEF05C08091EA127E
:10EBC0009091EB1201969093EB128093EA12AA9621
:10EBD0000FB6F894DEBF0FBECDBFDF91CF911F916E
:10EBE0000F91FF90EF90DF90CF90BF90AF909F90EC
:10EBF0008F907F9008958091F70483FD18C08091D5
:10EC0000D604811114C02091AB0E3091AC0E8091CE
:10EC1000510290915202281739074CF40E94EB558B
:10EC200040E050E0BA0185E59FE50C94815681E013
:10EC30008093D80440E050E0BA0185EF9BE50E9444
:10EC400081568AEB9CE0909391098093900986CC41
:10EC50006F927F928F929F92AF92BF92DF92EF92CC
:10EC6000FF920F931F93CF93DF93CDB7DEB7AD978E
:10EC70000FB6F894DEBF0FBECDBF7C01D62E8091BB
:10EC80009912882309F4F8C180918D14882309F41E
:10EC90009EC0442309F4C5C18091A514882329F19D
:10ECA000ECEAF0E584918F010F5F1F4F882321F07C
:10ECB0000E94E148F801F6CFE2E7FCE084918F0181
:10ECC0000F5F1F4F882321F00E94E148F801F6CF23
:10ECD00061E070E080E090E00E9410A78AE00E946E
:10ECE000E14889E69CE00F94FA098FE28093AA1428
:10ECF000B12C21E00BEA14E13FE1A32E80916214D4
:10ED0000B816B8F4AB9CC0011124B801805D9C4ECC
:10ED10002DA70E9488A5C8012DA58C010196F80198
:10ED20003081332321F02D3810F42F5FF6CFB394C8
:10ED3000E5CF27FD06C0B8018AE894E10E9488A5C6
:10ED400002C0F8011082E3EEF0E584918F010F5FBD
:10ED50001F4F882321F00E94E148F801F6CFB70148
:10ED600080E59CE00E940E8C6091A514FDE86F9FE9
:10ED7000B001112466557B4E85E49CE00E940E8C08
:10ED800040913B1550913C1560913D1570913E1599
:10ED90008FE39CE00E9417E08AE00E94E1488091A6
:10EDA000A51494E0899FF0011124EA55FB4E40918F
:10EDB0003B1550913C1560913D1570913E15408377
:10EDC0005183628373838F5F8093A5140DC010926B
:10EDD000A51422E0B22E27C1B70182E39CE00E9475
:10EDE0000E8C8AE00E94E1480E946DC51D82188643
:10EDF0001C821B828FE493E09A8389838CEE92E1DC
:10EE000090930C1380930B13F70180818F3209F0DC
:10EE10006DC087010F5F1F4FCE0101963C010115A8
:10EE2000110509F469C06FE270E0C8010F948F21E9
:10EE30005C01009709F461C00817190708F05DC06C
:10EE40004C01801A910AA401B801CE0180960F945A
:10EE5000AF21E0E2F0E0EC0FFD1FE80DF91D10829C
:10EE60008E01005E1F4FF80181918F01882319F0F8
:10EE70000E94E148F8CF8AE00E94E14860910B13BC
:10EE800070910C136115710519F06C5F7F4F02C012
:10EE900060E070E021E0AE01405E5F4FCE0105967C
:10EEA0000E9475C081111AC0EEE1FCE084918F01CF
:10EEB0000F5F1F4F811104C08E01005E1F4F04C001
:10EEC0000E94E148F801F2CFF80181918F01882377
:10EED00019F00E94E148F8CF8EE28CC070920C13BA
:10EEE00060920B1385010F5F1F4F99CF8DE093E167
:10EEF00090930C1380930B13870160910B13709107
:10EF00000C13DD2009F45DC06115710519F06C5F0B
:10EF10007F4F02C060E070E021E0A8018AE894E140
:10EF20000E9475C0882309F448C080919B14909179
:10EF30009C14A0919D14B0919E14809337159093CA
:10EF40003815A0933915B0933A15B80180E19CE0CB
:10EF50000E940E8C409137155091381560913915EB
:10EF600070913A1588E09CE00E9417E08AE00E94C8
:10EF7000E14810923B1510923C1510923D151092ED
:10EF80003E15E9EFFBE084917F019FEFE91AF90A52
:10EF9000882321F00E94E148F701F5CFB80180E015
:10EFA00090E00E9484C38091A812811102C0C80120
:10EFB00002C088EA92E160E02DC0B80185EE9BE0D6
:10EFC00013C06115710519F06C5F7F4F02C060E0DE
:10EFD00070E026E5A8018AE894E10E9475C08111DD
:10EFE0000CC0B80181ED9BE00E940E8C8EE20E9465
:10EFF000E1488AE00E94E1480FC081E080939612C8
:10F00000B7018FEB9BE00E940E8C8AE00E94E148E2
:10F0100060E0C8010E945255CE0101960E94D7615E
:10F020002BC0BB24B394E3EEF0E584918F010F5F16
:10F030001F4F882321F00E94E148F801F6CFEAE350
:10F04000FCE084918F010F5F1F4F882321F00E9405
:10F05000E148F801F6CFE1E0BE1203C005E413E099
:10F0600002C00FE313E0F80181918F01882309F4B6
:10F07000B3CE0E94E148F7CFAD960FB6F894DEBF4D
:10F080000FBECDBFDF91CF911F910F91FF90EF90F9
:10F09000DF90BF90AF909F908F907F906F9008957A
:10F0A0000F931F93CF93DF93CDB7DEB728970FB69B
:10F0B000F894DEBF0FBECDBF8823C9F083E992E08C
:10F0C00098878F8304E610E01A830983BE01695F85
:10F0D0007F4FCE0101960F94AC0D8AEB92E09E8398
:10F0E0008D831A830983BE016B5F7F4F0BC088EB52
:10F0F00091E09C838B8384E190E09A838983BE01B5
:10F100006D5F7F4FCE0101960F94AC0D28960FB620
:10F11000F894DEBF0FBECDBFDF91CF911F910F914D
:10F1200008950E9434E0BCCFCF92DF92EF92FF921D
:10F130000F931F93CF93DF93EB01FC0160817181EB
:10F14000828193812CE3C22ED12CE12CF12CA701DA
:10F1500096010F94F61D162F072FCA01B901A701BA
:10F1600096010F94F61DF62EE72ECA01B90128E18B
:10F1700030E040E050E00F94F61DFB01C9016DE660
:10F1800071E00F941C219B014F2D5E2D211531053F
:10F19000D9F00F931F93EF92FF92FF93EF939F93FA
:10F1A0008F933F932F9380EA90E19F938F93DF9308
:10F1B000CF930F948A198DB79EB70E960FB6F89419
:10F1C0009EBF0FBE8DBF5BC00097C9F00F931F930A
:10F1D000EF92FF92FF93EF939F938F9380E990E1DB
:10F1E0009F938F93DF93CF930F948A19EDB7FEB758
:10F1F0003C960FB6F894FEBF0FBEEDBF40C03097EF
:10F20000B9F00F931F93EF92FF92FF93EF9384E86F
:10F2100090E19F938F93DF93CF930F948A198DB7CB
:10F220009EB70A960FB6F8949EBF0FBE8DBF27C03B
:10F23000452BA9F00F931F93EF92FF928CE790E17B
:10F240009F938F93DF93CF930F948A19EDB7FEB7F7
:10F2500038960FB6F894FEBF0FBEEDBF10C00F93E7
:10F260001F9388E790E19F938F93DF93CF930F9441
:10F270008A190F900F900F900F900F900F90DF91C1
:10F28000CF911F910F91FF90EF90DF90CF90089555
:10F290002F923F924F925F926F927F928F929F92A6
:10F2A000AF92BF92CF92DF92EF92FF920F931F9394
:10F2B000CF93DF93CDB7DEB768970FB6F894DEBF74
:10F2C0000FBECDBF1C015B018A01DC01D7966D9199
:10F2D0007D918D919C91DA970F94F4196B017C01CB
:10F2E000F50120813181428153810F94551A0F9489
:10F2F0001A1F0F949D1F69877A878B879C87D80177
:10F300002D913D914D915C91C701B6010F94551A15
:10F310000F941A1F0F949D1F6D877E878F87988B80
:10F3200029853A854B855C8528373105410551058E
:10F3300040F488E790E0A0E0B0E089879A87AB8747
:10F34000BC872D853E854F85588928373105410575
:10F35000510540F488E790E0A0E0B0E08D879E87FB
:10F36000AF87B88B91012D5B3F4FD9018D919D9156
:10F370000D90BC91A02D8D839E83AF83B887BC0177
:10F38000CD010F94F61969837A838B839C836985F9
:10F390007A858B859C850F94F419698B7A8B8B8B7E
:10F3A0009C8B20E030E0A90169817A818B819C816E
:10F3B0000F94F019882339F1A7019601C701B6010E
:10F3C0000F94551A4B015C0129893A894B895C8954
:10F3D000CA01B9010F94551A9B01AC01C501B401D2
:10F3E0000F94531E4B015C0129813A814B815C8152
:10F3F000CA01B9010F94541E9B01AC01C501B401AF
:10F400000F94301F03C060E070E0CB010F941A1F0F
:10F410000F94981F2B013C016D817E818F8198850F
:10F4200090958095709561957F4F8F4F9F4F0F946A
:10F43000F6194B015C016D857E858F8598890F9447
:10F44000F4196D837E838F83988720E030E0A901D3
:10F45000C501B4010F94F019882349F12D813E8133
:10F460004F815885CA01B9010F94551A6D8B7E8B57
:10F470008F8B988FA7019601C701B6010F94551A7B
:10F480009B01AC016D897E898F89988D0F94531EE5
:10F490006B017C01A5019401C501B4010F94541EB8
:10F4A0009B01AC01C701B6010F94301F03C060E09F
:10F4B00070E0CB010F94C91FF10182889388A48862
:10F4C000B58875016401C418D508E608F7080F94DB
:10F4D000981FC61AD70AE80AF90AF7FE6BC020E09F
:10F4E00030E0A90169817A818B819C810F94F019A8
:10F4F000882309F447C029813A814B815C81CA0184
:10F50000B9010F94541E6B017C01C501B4010F9425
:10F51000F4199B01AC01C701B6010F94551A6B0198
:10F520007C0129893A894B895C89CA01B9010F9408
:10F53000551A9B01AC01C701B6010F94531E6B0114
:10F540007C012D813E814F815885CA01B9010F94FC
:10F55000551A9B01AC01C701B6010F94541E6B01F3
:10F560007C0120E030E040E850E469817A818B81C1
:10F570009C810F94551A9B01AC01C701B6010F94F1
:10F58000301F03C060E070E0CB010F941A1F0F948E
:10F59000981F2B013C0197FF03C0412C512C3201D5
:10F5A000481459046A047B0410F024013501C12C6D
:10F5B000D12C76018FB7F894D1019C9193FD22C094
:10F5C000F101468A578A608E718EC40CD51CE61CE8
:10F5D000F71C5A96CD92DD92ED92FC925D972985AB
:10F5E0003A854B855C85DB962D933D934D935C93DB
:10F5F000DE97FF962D853E854F8558892083318380
:10F60000428353838FBF68960FB6F894DEBF0FBE58
:10F61000CDBFDF91CF911F910F91FF90EF90DF90C1
:10F62000CF90BF90AF909F908F907F906F905F90A2
:10F630004F903F902F9008958F929F92AF92BF92DC
:10F64000CF92DF92EF92FF92CF93C82FC0907202B9
:10F65000D0907302E0907402F0907502A7019601B9
:10F66000C701B6010F9400218090E2069090E30656
:10F67000A090E406B090E506811129C0C11127C011
:10F6800080919F06882319F1A7019601C501B40155
:10F690000F94531E2091AD043091AE044091AF04FD
:10F6A0005091B0040F94551A0F948520719561956F
:10F6B00071098091F00E882351F08091A50E9091F0
:10F6C000A60E860F971F9093A60E8093A50E80928C
:10F6D000720290927302A0927402B0927502CF915E
:10F6E000FF90EF90DF90CF90BF90AF909F908F9062
:10F6F0000895CF92DF92EF92FF92E3EEF0E58491CE
:10F700007F019FEFE91AF90A882321F00E94E1485E
:10F71000F701F5CFEEE6F0E184917F019FEFE91A62
:10F72000F90A882321F00E94E148F701F5CF8AE524
:10F730000E94784B8823C9F10E94F2496B017C0139
:10F7400020E030E040E050EC0F947A2087FD20C0AC
:10F7500020E030E040EA50E4C701B6010F94F01910
:10F760001816B4F0C092E206D092E306E092E406E6
:10F77000F092E50680E060DF6091E2067091E306BA
:10F780008091E4069091E50642E00E949EE419C053
:10F79000E9E5F0E184917F019FEFE91AF90A8823F6
:10F7A00081F00E94E148F701F5CF4091E2065091C7
:10F7B000E3066091E4067091E50686E590E10E941B
:10F7C00030E58AE0FF90EF90DF90CF900C94E14815
:10F7D0004F925F926F927F928F929F92AF92BF9261
:10F7E000CF92DF92EF92FF92CF93DF93E3E5F0E1C8
:10F7F0008491EF012196882321F00E94E148FE01C7
:10F80000F7CF6091FE0E7091FF0E8091000F9091E6
:10F81000010F42E00E949EE4EFE4F0E18491EF01E9
:10F820002196882321F00E94E148FE01F7CF6091E4
:10F83000020F7091030F8091040F9091050F42E029
:10F840000E949EE4EBE4F0E18491EF01219688238D
:10F8500021F00E94E148FE01F7CF6091060F709100
:10F86000070F8091080F9091090F42E00E949EE4DB
:10F87000E7E4F0E18491EF012196882321F00E94D2
:10F88000E148FE01F7CF60910A0F70910B0F809154
:10F890000C0F90910D0F42E00E949EE48FB7F894F8
:10F8A0004090660E5090670E6090680E7090690EE2
:10F8B00080906A0E90906B0EA0906C0EB0906D0EC2
:10F8C000C0906E0ED0906F0EE090700EF090710EA2
:10F8D0008FBFEDE3F0E18491EF012196882321F0C1
:10F8E0000E94E148FE01F7CFC301B2010E9410A7B8
:10F8F000E9E3F0E18491EF012196882321F00E9451
:10F90000E148FE01F7CFC501B4010E9410A7E5E36D
:10F91000F0E18491EF012196882321F00E94E148D3
:10F92000FE01F7CFC701B6010E9410A78AE0DF9160
:10F93000CF91FF90EF90DF90CF90BF90AF909F90CE
:10F940008F907F906F905F904F900C94E1480F9351
:10F950001F93CF93DF93FC018491EF0121968111D6
:10F9600002C010E004C00E94E148FE01F5CF03E0B0
:10F97000010F84E0189FE0011124FE01EA5FFD4EB3
:10F9800020E030E0A90160817181828193810F9430
:10F990007A2087FD03C08BE20E94E148CA5FDD4EFA
:10F9A000688179818A819B8146E00E949EE480E2A1
:10F9B0000E94E1481F5F1013DCCF8AE00E94E148FB
:10F9C0001930A9F6DF91CF911F910F910895AF9251
:10F9D000BF92CF92DF92EF92FF920F931F93CF933C
:10F9E000C82F882319F0EDE1F0E10CC0E3EEF0E55B
:10F9F00084918F010F5F1F4F8823A9F30E94E14874
:10FA0000F801F6CF84918F010F5F1F4F882321F0FB
:10FA10000E94E148F801F6CFCC2319F0E0E0F0E1D4
:10FA20000CC0E3EEF0E584918F010F5F1F4F882338
:10FA3000A9F30E94E148F801F6CF84918F010F5F8E
:10FA40001F4F882321F00E94E148F801F6CF8AE099
:10FA50000E94E148C1112DC0E3EEF0E584918F01D1
:10FA60000F5F1F4F882321F00E94E148F801F6CF75
:10FA7000EDEEFFE084918F010F5F1F4F882321F08F
:10FA80000E94E148F801F6CF8091C904882321F053
:10FA90008AE00E94E14814C4E2EEFFE084918F0105
:10FAA0000F5F1F4F882309F40BC40E94E148F8013F
:10FAB000F5CF4091C4045091C5046091C604709183
:10FAC000C70489ED9FE00E9430E58AE00E94E1488A
:10FAD0008091C90481111BC0CC2319F0EEECFFE02A
:10FAE0000CC0E3EEF0E584918F010F5F1F4F882378
:10FAF000A9F30E94E148F801F6CF84918F010F5FCE
:10FB00001F4F882321F00E94E148F801F6CFC11170
:10FB100024C0E3EEF0E584918F010F5F1F4F88232F
:10FB200021F00E94E148F801F6CFEDEBFFE084916F
:10FB30008F010F5F1F4F882321F00E94E148F801D9
:10FB4000F6CFE3EEF0E584918F010F5F1F4F88231E
:10FB500021F00E94E148F801F6CF4091A5045091B0
:10FB6000A6046091A7047091A80485EB9FE00E9411
:10FB700030E54091A9045091AA046091AB047091C2
:10FB8000AC0482EB9FE00E9430E54091AD045091BF
:10FB9000AE046091AF047091B0048FEA9FE00E94C0
:10FBA00030E54091B1045091B2046091B30470917A
:10FBB000B4048CEA9FE00E9430E58AE00E94E148AC
:10FBC000C11124C0E3EEF0E584918F010F5F1F4F58
:10FBD000882321F00E94E148F801F6CFEEE8FFE02B
:10FBE00084918F010F5F1F4F882321F00E94E1480D
:10FBF000F801F6CFE3EEF0E584918F010F5F1F4F20
:10FC0000882321F00E94E148F801F6CF4091850455
:10FC100050918604609187047091880485E89FE084
:10FC20000E9430E54091890450918A0460918B04D0
:10FC300070918C0482E89FE00E9430E540918D0431
:10FC400050918E0460918F04709190048FE79FE033
:10FC50000E9430E540919104509192046091930488
:10FC6000709194048CE79FE00E9430E58AE00E9446
:10FC7000E148C11124C0E3EEF0E584918F010F5FEC
:10FC80001F4F882321F00E94E148F801F6CFEAE5F2
:10FC9000FFE084918F010F5F1F4F882321F00E94A6
:10FCA000E148F801F6CFE3EEF0E584918F010F5FB4
:10FCB0001F4F882321F00E94E148F801F6CF4091C0
:10FCC0009711509198116091991170919A1181E555
:10FCD0009FE00E9417E040919B1150919C11609110
:10FCE0009D1170919E118EE49FE00E9417E040915B
:10FCF0009F115091A0116091A1117091A2118BE4FC
:10FD00009FE00E9417E04091A3115091A4116091CF
:10FD1000A5117091A61188E49FE00E9417E08AE087
:10FD20000E94E148C11124C0E3EEF0E584918F0107
:10FD30000F5F1F4F882321F00E94E148F801F6CFA2
:10FD4000EEEFFEE084918F010F5F1F4F882321F0BB
:10FD50000E94E148F801F6CFE3EEF0E584918F01CF
:10FD60000F5F1F4F882321F00E94E148F801F6CF72
:10FD70004091AF115091B0116091B1117091B211D9
:10FD800085EF9EE00E9430E54091AB115091AC119F
:10FD90006091AD117091AE1182EF9EE00E9430E54E
:10FDA0004091A7115091A8116091A9117091AA11C9
:10FDB0008FEE9EE00E9430E58AE00E94E148C1118A
:10FDC00024C0E3EEF0E584918F010F5F1F4F88237D
:10FDD00021F00E94E148F801F6CFEBE7FEE08491C4
:10FDE0008F010F5F1F4F882321F00E94E148F80127
:10FDF000F6CFE3EEF0E584918F010F5F1F4F88236C
:10FE000021F00E94E148F801F6CF4091A7065091F9
:10FE1000A8066091A9067091AA0682E79EE00E945A
:10FE200030E54091A3065091A4066091A50670911B
:10FE3000A6068FE69EE00E9430E540918B0550912A
:10FE40008C0560918D0570918E058CE69EE00E9478
:10FE500017E0409195045091960460919704709139
:10FE6000980489E69EE00E9430E540919904509103
:10FE70009A0460919B0470919C0486E69EE00E9427
:10FE800030E540919D0450919E0460919F047091D3
:10FE9000A00483E69EE00E9430E54091A1045091C9
:10FEA000A2046091A3047091A40480E69EE00E94E5
:10FEB00030E58AE00E94E148C11124C0E3EEF0E59C
:10FEC00084918F010F5F1F4F882321F00E94E1482A
:10FED000F801F6CFE2E5FEE084918F010F5F1F4F3E
:10FEE000882321F00E94E148F801F6CFE3EEF0E527
:10FEF00084918F010F5F1F4F882321F00E94E148FA
:10FF0000F801F6CF4091F20E5091F30E6091F40E8D
:10FF10007091F50E89E49EE00E9430E54091F60E66
:10FF20005091F70E6091F80E7091F90E86E49EE004
:10FF30000E9430E54091FA0E5091FB0E6091FC0E4C
:10FF40007091FD0E83E49EE00E9430E58AE00E94FD
:10FF5000E148C11124C0E3EEF0E584918F010F5F09
:10FF60001F4F882321F00E94E148F801F6CFEFE20D
:10FF7000FEE084918F010F5F1F4F882321F00E94C4
:10FF8000E148F801F6CFE3EEF0E584918F010F5FD1
:10FF90001F4F882321F00E94E148F801F6CF6091BD
:10FFA0009F0670E086E29EE00E9420A88AE00E9400
:10FFB000E148CC2379F030ECA32E34E0B32E48EBAB
:10FFC000C42E44E0D42E5CEBE52E54E0F52E00E088
:10FFD00010E024C0E3EEF0E584918F010F5F1F4F26
:10FFE000882321F00E94E148F801F6CFE9E0FEE025
:10FFF00084918F010F5F1F4F882321F00E94E148F9
:020000021000EC
:10000000F801F6CFE3EEF0E584918F010F5F1F4F0B
:10001000882389F20E94E148F801F6CFB80180E018
:100020009EE00E9420A8F501619171915F018DEF22
:100030009DE00E9420A8F601619171916F018AEF05
:100040009DE00E9420A8F701619171917F0187EFE7
:100050009DE00E9420A88AE00E94E1480F5F1F4FA8
:1000600002301105D9F6C11124C0E3EEF0E5849108
:100070008F010F5F1F4F882321F00E94E148F80194
:10008000F6CFE8EEFDE084918F010F5F1F4F8823CC
:1000900021F00E94E148F801F6CFE3EEF0E584910B
:1000A0008F010F5F1F4F882321F00E94E148F80164
:1000B000F6CF4091DC0E5091DD0E6091DE0E709116
:1000C000DF0E8FED9DE00E9430E52CEA35EC47E233
:1000D0005EE36091D80E7091D90E8091DA0E909106
:1000E000DB0E0F94301FAB01BC018CED9DE00E9434
:1000F00014E52CEA35EC47E25EE36091D40E709192
:10010000D50E8091D60E9091D70E0F94551AAB0153
:10011000BC0189ED9DE00E9414E58AE00E94E1485F
:10012000C1110CC0E3EEF0E584918F010F5F1F4F0A
:10013000882321F00E94E148F801F6CF4091D204D3
:100140005091D3046091D4047091D50480ED9DE06A
:100150000E9430E52CEA35EC47E25EE36091CE0484
:100160007091CF048091D0049091D1040F94301FEE
:10017000AB01BC018DEC9DE00E9414E52CEA35EC4E
:1001800047E25EE36091CA047091CB048091CC0495
:100190009091CD040F94551AAB01BC018AEC9DE0FF
:1001A0000E9414E58AE00E94E148C11124C0E3EEF8
:1001B000F0E584918F010F5F1F4F882321F00E948B
:1001C000E148F801F6CFE4EBFDE084918F010F5F89
:1001D0001F4F882321F00E94E148F801F6CFE3EE9B
:1001E000F0E584918F010F5F1F4F882321F00E945B
:1001F000E148F801F6CF4091E2065091E3066091A4
:10020000E4067091E5068BEA9DE00E9430E58AE005
:100210000E94E148C11124C0E3EEF0E584918F0112
:100220000F5F1F4F882321F00E94E148F801F6CFAD
:10023000E2E9FDE084918F010F5F1F4F882321F0D9
:100240000E94E148F801F6CFE3EEF0E584918F01DA
:100250000F5F1F4F882321F00E94E148F801F6CF7D
:100260004091DF045091E0046091E1047091E20458
:1002700089E89DE00E9417E04091E3045091E40476
:100280006091E5047091E60486E89DE00E9417E025
:100290004091E7045091E8046091E9047091EA0408
:1002A00083E89DE00E9417E08AE0CF911F910F91B3
:1002B000FF90EF90DF90CF90BF90AF900C94E1480B
:1002C000E3EEF0E584918F010F5F1F4F882309F45F
:1002D000F0CB0E94E148F801F5CF83E50E94784B0E
:1002E0008823D9F00E94F249AB01BC014093AF11C1
:1002F0005093B0116093B1117093B2114093A71154
:100300005093A8116093A9117093AA118BE59DE0F9
:100310000E9430E58AE00E94E14880E50E94784B27
:10032000882399F00E94F249AB01BC014093AF11C0
:100330005093B0116093B1117093B2118EE39DE0B0
:100340000E9430E58AE00E94E14882E50E94784BF5
:10035000882399F00E94F249AB01BC014093AB1194
:100360005093AC116093AD117093AE118FE19DE08D
:100370000E9430E58AE00E94E14884E50E94784BC3
:10038000882399F00E94F249AB01BC014093A71168
:100390005093A8116093A9117093AA1181E09DE078
:1003A0000E9430E58AE00C94E1480895CF93DF93F2
:1003B00085E40E94504C811110C080E50E94784B6A
:1003C000882391F00E94F2496093DC0E7093DD0E59
:1003D0008093DE0E9093DF0E07C00E94D2498823DF
:1003E00061F3ECEAF0E56DC089E40E94784B882364
:1003F00081F00E94F2492CEA35EC47E25EE30F946B
:10040000551A6093D80E7093D90E8093DA0E90939C
:10041000DB0E84E40E94784B882381F00E94F2492D
:100420002CEA35EC47E25EE30F94301F6093D40E64
:100430007093D50E8093D60E9093D70EE3EEF0E531
:100440008491EF012196882321F00E94E148FE016A
:10045000F7CF4091DC0E5091DD0E6091DE0E709171
:10046000DF0E8DEF9CE00E9430E52CEA35EC47E290
:100470005EE36091D80E7091D90E8091DA0E909162
:10048000DB0E0F94301FAB01BC0189EF9CE00E9492
:1004900014E52CEA35EC47E25EE36091D40E7091EE
:1004A000D50E8091D60E9091D70E0F94551AAB01B0
:1004B000BC0185EF9CE00E9414E510C00E94E14859
:1004C000FE018491EF0121968111F8CFCEE0D3E0B7
:1004D0008991882319F00E94E148FACF8AE0DF91E0
:1004E000CF910C94E148FB014081FC0120813181D6
:1004F000342768E0A901440F551F37FD07C09A0152
:100500006150C1F7FC013183208308959A01F1E223
:100510002F27F0E13F27F4CFEF92FF920F931F9325
:10052000CF93DF93EC0189018C81833039F0E9E0CE
:10053000440F551F661F771FEA95D1F79A01AB014B
:1005400061E1CE010E941F4E882331F084E089834F
:10055000CE010E94F74D41C00E94FB4D7B010E94DD
:10056000DA488B838F3F49F40E94FB4D6E197F0957
:100570006D327140A0F381E103C08E3F49F08FE0FE
:100580008983CE010E94F74D8FEF0E94D54825C088
:100590008FEF8EBDF80180E090E02FEF0DB407FEE5
:1005A000FDCF3EB531932EBD01968F3F31E09307CD
:1005B000A9F70DB407FEFDCF8EB5F801E150FE4F4F
:1005C00080830E94DA480E94DA48CE010E94F74DEB
:1005D0008FEF0E94D54881E001C080E0DF91CF918C
:1005E0001F910F91FF90EF9008950F931F93CF935A
:1005F000DF93EC0189018C81833039F0F9E0440FFD
:10060000551F661F771FFA95D1F79A01AB0168E174
:10061000CE010E941F4E882311F086E034C08EEF79
:100620008EBD80E090E00DB407FEFDCFF801E80F2D
:10063000F91F20812EBD0DB407FEFDCF21812EBDF7
:100640000296811522E0920771F70DB407FEFDCFE7
:100650008FEF0E94D5488FEF0E94D5480E94DA485C
:100660008B838F71853031F083E18983CE010E94C5
:10067000F74D0AC068E572E0CE010E94074E182FC0
:10068000811107C087E18983CE010E94F74D10E0F8
:1006900012C020E030E0A9016DE0CE010E941F4EA3
:1006A000811104C00E94DA48882311F086E1EBCF63
:1006B000CE010E94F74D812FDF91CF911F910F91B5
:1006C0000895CF938091FD068823A9F14091FE06FD
:1006D0005091FF06609100077091010722E037E01A
:1006E0008091FB069091FC0680DFC82F882321F1C2
:1006F0004091DE065091DF066091E0067091E106C0
:10070000411551056105710589F022E037E08091BE
:10071000FB069091FC0669DF882359F01092DE06F3
:100720001092DF061092E0061092E1061092FD068C
:100730008C2FC82F01C0C1E08C2FCF910895CF928C
:10074000DF92EF92FF92CF936B017C01C42F8091D7
:10075000FE069091FF06A0910007B09101078C154D
:100760009D05AE05BF05C1F0ACDF811102C080E080
:1007700017C022E037E0B701A6018091FB069091F7
:10078000FC06CADE882399F3C092FE06D092FF06CB
:10079000E0920007F092010781E0C1118093FD060D
:1007A000CF91FF90EF90DF90CF9008958F929F921E
:1007B000AF92BF92CF92DF92EF92FF920F931F936F
:1007C000CF93DF93EC016A017B01890189859A85CA
:1007D000AB85BC850196A11DB11D84179507A607A1
:1007E000B70710F480E054C08F89803129F499272D
:1007F000872F762F652F0BC08032A1F7CB01BA016E
:1008000027E096958795779567952A95D1F78B88F8
:100810009C88AD88BE88680D791D8A1D9B1D8090BF
:10082000FE069090FF06A0900007B09001076815A3
:1008300079058A059B0581F48F89803191F4DD2447
:10084000EE24FF24F601EE0FFF1FEE5FF84F8081CC
:100850009181A0E0B0E016C040E071DF8111ECCFE3
:10086000C1CFE894C7F8DD24EE24FF24F601EE0F93
:10087000FF1FEE0FFF1FEE5FF84F80819181A28175
:10088000B381BF70F80180839183A283B38381E039
:10089000DF91CF911F910F91FF90EF90DF90CF905C
:1008A000BF90AF909F908F9008952F923F924F925C
:1008B0005F926F927F928F929F92AF92BF92CF92F0
:1008C000DF92EF92FF920F931F93CF93DF93EC0190
:1008D0005B016A018B81811103C08FEF9FEFC6C05E
:1008E000898180FFFACF49895A896B897C898885FB
:1008F0009985AA85BB852601612C712C8A019B01F3
:10090000081B190B2A0B3B0B04151505260537058B
:1009100018F46A01C81AD90A76013E0124E0620E71
:10092000711CE114F10409F476C0488559856A8583
:100930007B854A0181E098222B811A012B01E9E095
:100940005694479437942794EA95D1F7898D9A8DD8
:10095000FC01223049F4628D738D848D958D620D7A
:10096000731D841D951D3CC01481115012218114EA
:100970009104C1F4111116C0452B462B472B49F4A5
:100980008D899E89AF89B88D8C839D83AE83BF830B
:1009900009C04C815D816E817F81930107DF8823CF
:1009A00009F49BCFE98DFA8D6C817D818E819F81C9
:1009B0006250710981099109058404C0660F771F8F
:1009C000881F991F0A94D2F7268537854089518957
:1009D000620F731F841F951F610F711D811D911D73
:1009E00020E032E02819390987012E153F0508F467
:1009F00089010115F2E01F0761F52091FE06309193
:100A0000FF064091000750910107621773078407A2
:100A1000950719F41EC0C60129C09501AB01BC01A0
:100A20008091FB069091FC0677DD882309F455CF71
:100A3000A00EB11E88859985AA85BB85800F911F60
:100A4000A11DB11D88879987AA87BB87E01AF10A83
:100A500068CF40E074DE882309F43FCFB4016E5FB5
:100A6000784FA801C5010F946821E2CFDF91CF91A3
:100A70001F910F91FF90EF90DF90CF90BF90AF90BC
:100A80009F908F907F906F905F904F903F902F90AE
:100A900008954F925F926F927F92AF92BF92CF92E2
:100AA000DF92EF92FF920F931F93CF93DF93EC01AE
:100AB0006A017B012B81222349F089899A89AB89BC
:100AC000BC8984179507A607B70710F480E06BC0B0
:100AD000223009F463C0C114D104E104F10449F4E3
:100AE0001C821D821E821F82188619861A861B860A
:100AF00059C088859985AA85BB85E98DFA8DE585DC
:100B0000F0E03996AC01BD0141505109610971090C
:100B10000E2E04C076956795579547950A94D2F79F
:100B200097018601015011092109310904C0369548
:100B3000279517950795EA95D2F704171507260705
:100B4000370720F0892B8A2B8B2B49F48D899E89BE
:100B5000AF89B88D8C839D83AE83BF8304C0041B93
:100B6000150B260B370B280139015E0184E0A80E16
:100B7000B11C411451046104710481F04C815D8108
:100B80006E817F819501898D9A8D10DE91E0491AE1
:100B90005108610871088111ECCF05C0C886D9865B
:100BA000EA86FB8681E0DF91CF911F910F91FF9044
:100BB000EF90DF90CF90BF90AF907F906F905F905D
:100BC0004F9008954F925F926F927F92AF92BF9233
:100BD000CF92DF92EF92FF920F931F93CF93DF9309
:100BE00000D01F92CDB7DEB78C0149835A836B8347
:100BF0007C835901C12CD12C7601412CF2E05F2E6F
:100C0000612C712C49815A816B817C819E012F5FFF
:100C10003F4FC801CBDD882341F1D301C201F80168
:100C2000058404C0880F991FAA1FBB1F0A94D2F71E
:100C3000C80ED91EEA1EFB1E49815A816B817C8138
:100C40008789803139F481E0483F5F4F6105710544
:100C500038F4D8CF81E0483F5F4F6F4F7F4090F22C
:100C6000F501C082D182E282F3820F900F900F9043
:100C70000F90DF91CF911F910F91FF90EF90DF9038
:100C8000CF90BF90AF907F906F905F904F900895FE
:100C90000F931F93CF93DF93EC018B018B818823FC
:100CA00011F080E041C0FB018789803131F1803251
:100CB000C1F783E08B83F801428D538D648D758D70
:100CC0004D8B5E8B6F8B788F9E012F5E3F4FC801DF
:100CD00079DF882331F31A8F098F81E089831C82A1
:100CE0001D821E821F82188619861A861B861C8604
:100CF0001D861E861F86188A17C082E08B831D8A78
:100D00001E8A1F8A188EFB01408D518D60E070E0B5
:100D1000A5E0440F551F661F771FAA95D1F7498B91
:100D20005A8B6B8B7C8BD7CFDF91CF911F910F911B
:100D300008954F925F926F927F928F929F92AF929F
:100D4000BF92CF92DF92EF92FF920F931F93CF93B8
:100D5000DF93EC014A015B01280139014230510562
:100D60006105710508F462C049855A856B857C85EB
:100D70004F5F5F4F6F4F7F4F481559056A057B05E1
:100D800008F454C08F89803129F4FF24EB2CDA2C2D
:100D9000C92C0CC0803209F049C07501640107E01C
:100DA000F694E794D794C7940A95D1F74B895C8958
:100DB0006D897E89C40ED51EE61EF71E41E0C7016F
:100DC000B601BDDC882391F19F89903159F49924B3
:100DD000AA24BB24F401EE0FFF1FEE5FF84F5182EF
:100DE000408210C0E89487F89924AA24BB24F40117
:100DF000EE0FFF1FEE0FFF1FEE5FF84F4082518294
:100E0000628273829A89923090F04D815E816F8107
:100E100078854C0D5D1D6E1D7F1D4093DE06509341
:100E2000DF066093E0067093E10601C080E0DF9189
:100E3000CF911F910F91FF90EF90DF90CF90BF90D7
:100E4000AF909F908F907F906F905F904F9008959C
:100E5000AF92BF92CF92DF92EF92FF920F931F93C8
:100E6000CF93DF9300D01F92CDB7DEB75C016A014C
:100E70007B0182E090E0A0E0B0E0F5018083918307
:100E8000A283B3839E012F5F3F4FB701A601C50127
:100E90008DDC811102C080E023C000E010E09801E9
:100EA000B701A601C50145DF8823A9F3C980DA800F
:100EB000EB80FC80F5018789803149F481E0F8EF0F
:100EC000CF16FFEFDF06E104F10450F4DBCF81E041
:100ED00098EFC9169FEFD906E9069FE0F90690F250
:100EE0000F900F900F900F90DF91CF911F910F9166
:100EF000FF90EF90DF90CF90BF90AF900895CF9389
:100F0000DF93CDB7DEB78091EB04811110C09E0155
:100F1000275F3F4F4F81588562E470E08EE092E09A
:100F20000F94B8190E94335583E08093A802DF9193
:100F3000CF910895FF920F931F93CF93DF93C091AA
:100F40009C0681E0C827D0919D06D827F0909E0688
:100F5000F826C11102C0DD2319F0E3EEF0E504C06C
:100F6000F110FBCF80E077C084918F010F5F1F4F9E
:100F7000882321F00E94E148F801F6CFEBEFF0E181
:100F800084918F010F5F1F4F882321F00E94E14859
:100F9000F801F6CFCC2361F0E9EFF0E184918F0105
:100FA0000F5F1F4F882321F00E94E148F801F6CF20
:100FB000DD2361F0E7EFF0E184918F010F5F1F4FB8
:100FC000882321F00E94E148F801F6CFF11003C018
:100FD000EDEEF0E10CC0E5EFF0E184918F010F5FE1
:100FE0001F4F8823A9F30E94E148F801F6CF8491AE
:100FF0008F010F5F1F4F882321F00E94E148F80105
:10100000F6CFFF2019F047E553E002C04BEB53E069
:10101000DD2319F029E533E002C02BEB33E0CC23CC
:1010200019F08BE593E002C08BEB93E05F934F9355
:101030003F932F939F938F938BED90E19F938F938B
:101040001F925DDF8DB79EB709960FB6F8949EBFCD
:101050000FBE8DBF81E0DF91CF911F910F91FF9067
:101060000895CF92DF92EF92FF92C0900A0FD09036
:101070000B0FE0900C0FF0900D0F2091B104309108
:10108000B2044091B3045091B404C701B6010F9467
:10109000551A0F94852060934A1270934B128093D7
:1010A0004C1290934D12C701B6010F94981F2FB7A1
:1010B000F8946093720E7093730E8093740E9093F5
:1010C000750E2FBF10923A1210923B1210923C12E2
:1010D00010923D12FF90EF90DF90CF900895CF9245
:1010E000DF92EF92FF920F931F93CF93DF939FE1D5
:1010F000E92E93E0F92E00E414E0CEEFDEE02FEECF
:10110000C22E24E0D22EF70181917F010E94784BFC
:101110008823D1F00E94F249F6012081211104C0F8
:101120002091F304222329F0288139814A815B81AF
:1011300003C020E030E0A9010F94541EF801608341
:1011400071838283938309C088819981AA81BB813D
:10115000F80180839183A283B3830C5F1F4F249691
:10116000FFEFCF1ADF0A83E2E81683E0F80659F6AC
:1011700086E40E94504C8823C9F00E94F24920E086
:1011800030E0A9010F947A20181684F40E94F249E5
:1011900020E030E040E752E40F94301F60930A02F1
:1011A00070930B0280930C0290930D028091F704D0
:1011B00083FD2AC060914C0470914D0480914E04CF
:1011C00090914F0420910A0F30910B0F40910C0F1A
:1011D00050910D0FE0919512EE23B1F00F94531E34
:1011E0009B01AC01609187127091881280918912E5
:1011F00090918A120F94541E6093871270938812F4
:101200008093891290938A12DF91CF911F910F9151
:10121000FF90EF90DF90CF90089580916E12813013
:1012200079F482E080936E120E94FB4D60937712F6
:10123000709378128093791290937A1281E00895D6
:1012400080E00895E82FF0E0EE5CF44D849190E0AA
:10125000FC013797EC30F105F8F4EC57FF4F0D9493
:1012600043218091B100887F84608093B10008950C
:1012700080919100887F846080939100089580918F
:10128000A100887F84608093A1000895809121014E
:10129000887F84608093210108958F929F92AF92FE
:1012A000BF92CF92DF92EF92FF920F931F93CF9353
:1012B000DF931F921F92CDB7DEB77C014901809169
:1012C0008A05811147C08B015B01A40EB51E0A156A
:1012D0001B0509F43FC0F701C080D180F80161917E
:1012E0008F016983C6016A830F94B61C6A816817EF
:1012F00029F1C6010F94DF1CC6010F94B61C998119
:101300008917E1F0E3EEF0E584918F010F5F1F4F45
:10131000882321F00E94E148F801F6CFE1ECF0E1EA
:1013200084918F010F5F1F4F882321F00E94E148B5
:10133000F801F6CF81E080938A050CC0BE016F5F93
:101340007F4FC401D0D8F7018081918101969183AC
:101350008083BDCF0F900F90DF91CF911F910F91A0
:10136000FF90EF90DF90CF90BF90AF909F908F90C5
:101370000895AF92BF92CF92DF92EF92FF920F93B8
:101380001F93CF93DF931F92CDB7DEB78C016B0114
:101390007A01590180918A0581111BC0F801808171
:1013A00091810F94B61C8983F60181936F01BE0170
:1013B0006F5F7F4FC50197D8F801408151814F5F22
:1013C0005F4F51834083F1E0EF1AF108E114F1041B
:1013D00029F70F90DF91CF911F910F91FF90EF9020
:1013E000DF90CF90BF90AF900895CF92DF92EF92B1
:1013F000FF920F931F93CF93DF937C018B016A01C0
:10140000E9010E94EB5583E08093A802F092B806B0
:10141000E092B7061093B6060093B5061092B10697
:101420001092B2061092B3061092B406A601662777
:1014300057FD6095762F4093AD065093AE066093AE
:10144000AF067093B006F80180819181AA2797FDBD
:10145000A095BA2F8093B7119093B811A093B911AA
:10146000B093BA118AE99BEC90937702809376024D
:10147000D0936B11C0936A1110926911DF91CF91D3
:101480001F910F91FF90EF90DF90CF900895CF9232
:10149000DF92EF92FF920F931F93CF93DF9300D0D1
:1014A0001F92CDB7DEB77C018B01CA01B901298338
:1014B0007A838B839C830E94EB5523E02093A802C0
:1014C000F092B806E092B7061093B6060093B50600
:1014D0002AE037ED43E25CE369817A818B819C816C
:1014E0000F94551A0F94981F6093B1067093B2062B
:1014F0008093B3069093B4060F94F6196B017C01A8
:101500009B01AC0160E070E887E794E40F94531E00
:101510000F94981F6093AD067093AE068093AF064C
:101520009093B0062AE037ED43E25CE3F801608176
:101530007181828193810F94551AA70196010F94AE
:10154000531E0F949D1F6093B7117093B811809331
:10155000B9119093BA118FED99EC90937702809323
:1015600076020F900F900F900F90DF91CF911F9107
:101570000F91FF90EF90DF90CF9008950F931F93FE
:10158000CF93DF938C01EB010E94EB5583E08093B6
:10159000A8021093B8060093B706D093B606C0937E
:1015A000B50684EF91E0A0E0B0E08093B10690939F
:1015B000B206A093B306B093B40688EE9FE3AFE003
:1015C000B0E08093AD069093AE06A093AF06B093C3
:1015D000B00620E030E048EC52E4688179818A81ED
:1015E0009B810F94551A20E030E04AEF53E40F94AA
:1015F000531E0F949D1F6093B7117093B811809381
:10160000B9119093BA1182E798EC90937702809386
:1016100076028FE29DEE90936B1180936A11109287
:101620006911DF91CF911F910F910895CF92DF92B1
:10163000EF92FF920F931F93CF93DF9300D01F92EF
:10164000CDB7DEB77C018B0129833A834B835C8362
:101650000E94EB5583E08093A802F092B806E092D6
:10166000B7061093B6060093B50629813A814B81DF
:101670005C81CA01B9010F94F4192AE037ED43E205
:101680005CE30F94551A0F94981F6093B106709302
:10169000B2068093B3069093B4060F94F6196B01CB
:1016A0007C019B01AC0160E070E887E794E40F9453
:1016B000531E0F94981F6093AD067093AE068093EF
:1016C000AF069093B006F8016081718182819381A9
:1016D0000F94F4192AE037ED43E25CE30F94551AB6
:1016E000A70196010F94531E0F949D1F6093B7118D
:1016F0007093B8118093B9119093BA118CED90E06A
:10170000909377028093760283E69FE490936B1127
:1017100080936A11109269110F900F900F900F90A3
:10172000DF91CF911F910F91FF90EF90DF90CF90BD
:1017300008958F929F92AF92BF92CF92DF92EF92D5
:10174000FF92CF9320E030E04AE754E4FC0160814F
:101750007181828193810F94551A0F94981F6B01A8
:101760007C01611571058105910561F097FF0AC043
:10177000F094E094D094C094C11CD11CE11CF11CE5
:101780008DE201C080E28093BD06C701B60128EE5C
:1017900033E040E050E00F94181E6AE0862E912C52
:1017A000A12CB12CCA01B901A50194010F94181EF6
:1017B000605D6093BE068EE28093BF06C701B601EE
:1017C00024E630E040E050E00F94181ECA01B90151
:1017D000A50194010F94181E605D6093C006C701B7
:1017E000B601A50194010F94181EC62FCA01B901B4
:1017F000A50194010F94181E605D6093C106C05D41
:10180000C093C2068DEB96E0CF91FF90EF90DF90F2
:10181000CF90BF90AF909F908F9008950F931F939C
:10182000CF93DF931F921F92CDB7DEB7FC01849157
:101830008F010F5F1F4F811102C08B0108C06983A8
:101840007A830E94E148F80169817A81F0CFD8015A
:101850008D918D01882319F00E94E148F8CF0F90F7
:101860000F90DF91CF911F910F9108950F931F93C8
:10187000CF93DF938C01E3EEF0E58491EF012196A5
:10188000882321F00E94E148FE01F7CFB80184EBE4
:1018900090E1C4DF82E20E94E1488AE00E94E148D0
:1018A00081E0DF91CF911F910F9108958F929F92C8
:1018B000AF92BF92CF92DF92EF92FF92CF93FC0153
:1018C000C080D180E280F38020E030E0A901C70130
:1018D000B6010F94F01987FF08C0C701B6019058F0
:1018E00020E030E048EC52E406C020E030E048EC74
:1018F00052E4C701B6010F94551A0F94981F6B015B
:101900007C01603AF6E87F07F1E08F07910584F0EB
:1019100020EA36E841E050E00F94181ECA01B901F0
:101920002AE030E040E050E00F94181E605D01C0F6
:1019300060E26093BC0680E1C81687E2D806E10445
:10194000F10494F0C701B60120E137E240E050E035
:101950000F94181ECA01B9012AE030E040E050E0BF
:101960000F94181E605D01C060E26093BD06E8EE52
:10197000CE16E3E0DE06E104F10494F0C701B601FF
:1019800028EE33E040E050E00F94181ECA01B90180
:101990002AE030E040E050E00F94181E605D01C086
:1019A00060E26093BE06C701B60124E630E040E085
:1019B00050E00F94181E7AE0872E912CA12CB12CA8
:1019C000CA01B901A50194010F94181E605D6093CE
:1019D000BF068EE28093C006C701B601A50194013F
:1019E0000F94181EC62FCA01B901A50194010F94C6
:1019F000181E605D6093C106C05DC093C2068CEB8B
:101A000096E0CF91FF90EF90DF90CF90BF90AF9096
:101A10009F908F9008958F929F92AF92BF92CF9296
:101A2000DF92EF92FF92CF9320E030E048EC52E457
:101A3000FC0160817181828193810F94551A0F940A
:101A4000981F6B017C0197FF0AC0F094E094D0943A
:101A5000C094C11CD11CE11CF11C8DE201C08BE2C1
:101A60008093BC06C701B60120E137E240E050E0B8
:101A70000F94181EEAE08E2E912CA12CB12CCA01D5
:101A8000B901A50194010F94181E605D6093BD0615
:101A9000C701B60128EE33E040E050E00F94181E75
:101AA000CA01B901A50194010F94181E605D6093ED
:101AB000BE06C701B60124E630E040E050E00F94D6
:101AC000181ECA01B901A50194010F94181E605D8A
:101AD0006093BF068EE28093C006C701B601A501E0
:101AE00094010F94181EC62FCA01B901A5019401D3
:101AF0000F94181E605D6093C106C05DC093C2065E
:101B00008CEB96E0CF91FF90EF90DF90CF90BF905D
:101B1000AF909F908F9008958F929F92AF92BF92B7
:101B2000CF92DF92EF92FF92FC01C080D180E280E1
:101B3000F38020E030E0A901C701B6010F94F0194D
:101B400087FF04C0C701B601905802C0C701B601A3
:101B50000F94981F6B017C016031F7E27F078105CC
:101B6000910584F020E137E240E050E00F94181E28
:101B7000CA01B9012AE030E040E050E00F94181E9D
:101B8000605D01C060E26093BE0688EEC81683E027
:101B9000D806E104F10494F0C701B60128EE33E061
:101BA00040E050E00F94181ECA01B9012AE030E06D
:101BB00040E050E00F94181E605D01C060E2609349
:101BC000BF06E4E6CE16D104E104F10494F0C701A7
:101BD000B60124E630E040E050E00F94181ECA0140
:101BE000B9012AE030E040E050E00F94181E605D3B
:101BF00001C060E26093C006FAE0CF16D104E104B0
:101C0000F1049CF0FAE08F2E912CA12CB12CC7018D
